:100000000C944C160C947D160C947D160C947D1655
:100010000C947D160C947D160C947D160C947D1614
:100020000C947D160C947D160C947D160C947D1604
:100030000C947D160C944E590C947D160C947D16E0
:100040000C947D160C9421C40C947D160C947D1692
:100050000C947D160C947D160C9479760C940459AE
:100060000C947D160C94B74B0C947D160C947D1655
:100070000C947D160C947D160C947D160C947D16B4
:100080000C947D160C947D160C947D160C947D16A4
:100090000C947D160C947D160C947D160C947D1694
:1000A0000C947D160C947D160C947D160C947D1684
:1000B0000C947D160C947D160C947D160C947D1674
:1000C0000C947D160C947D160C947D160C947D1664
:1000D0000C947D160C947D160C9469580C942A5837
:1000E0000C947D168D31AA31DB31F8310D32363268
:1000F000A3320933B233FA370838013828382C389C
:100100004638A13C5B38A738CE38F5381E397439EB
:1001100085399639A739B839C939A13CAC3BA13CDE
:10012000B73B273C2D3C4D3CD0B0D3B0C2B0C6B09D
:10013000CCB00AB1D7B0DBB0E1B0E5B0E9B0EFB018
:10014000F3B0F7B00AB1FDB001B105B16AB66FB650
:1001500074B67EB688B601B792B69AB6A2B6ACB6F9
:10016000B6B6C0B6CFB6D9B601B7E3B6EDB6F7B6F8
:10017000084AD73B3BCE016E84BCBFFDC12F3D6C0E
:1001800074319ABD56833DDA3D00C77F11BED9E474
:10019000BB4C3E916BAAAABE000000803F05A84C54
:1001A000CDB2D44EB93836A9020C50B99186880820
:1001B0003CA6AAAA2ABE000000803F004E414E493C
:1001C0004E495459494E46CDCCCC3D0AD7233C1715
:1001D000B7D13877CC2B329595E6241FB14F0A0062
:1001E0000020410000C84200401C4620BCBE4CCA52
:1001F0001B0E5AAEC59D74434F4D4D554E4943415C
:1002000054494F4E0044525952554E004552524F98
:10021000525300494E464F004543484F0047322F46
:1002200047332062616420706172616D657465722C
:10023000730A00206F6620004D424C20473239205F
:10024000706F696E74200059206F7574206F66207E
:1002500072616E67652028312D35292E0A005820DD
:100260006F7574206F662072616E67652028312D6E
:1002700035292E0A004D6573682070726F62696EB1
:100280006720646F6E652E0A005374617274206D6E
:100290006573682070726F62696E67207769746831
:1002A0002022473239205331222066697273742E1E
:1002B0000A004732380A47323920533200537461FA
:1002C00074653A20004D65736820626564206C6532
:1002D00076656C696E6720686173206E6F2064615B
:1002E00074612E0A0053206F7574206F662072614E
:1002F0006E67652028302D35292E0A004D657368FC
:1003000020706F696E742063616E6E6F7420626519
:10031000207265736F6C7665640A00456E642066B2
:10032000696C65206C6973740A00426567696E20A8
:1003300066696C65206C6973740A00286E6F2066AC
:10034000696C6529005344207072696E74696E6728
:10035000206279746520004E6F74205344207072BF
:10036000696E74696E670A0043757272656E7420F7
:1003700066696C653A20002569730025696D202542
:100380006973002569682025696D2025697300253A
:100390006964202569682025696D20256973002519
:1003A000697920256964202569682025696D2025E3
:1003B0006973005072696E742074696D653A20002B
:1003C0006F6E2E0A006F66662E0A00473236204492
:1003D000656275672000180213020C020502F7011E
:1003E0006F66660044454255473A004B494C4C45C0
:1003F000442E20004D3131332053006F6B002C20F0
:10040000002C2000544845524D414C5F50524F54EF
:10041000454354494F4E004155544F5245504F5259
:10042000545F53445F53544154555300454D455216
:1004300047454E43595F5041525345520043415343
:10044000455F4C494748545F4252494748544E45DE
:10045000535300544F47474C455F4C49474854530A
:1004600000534F4654574152455F504F5745520035
:100470004255494C445F50455243454E54004C450B
:1004800056454C494E475F44415441005A5F5052D3
:100490004F4245004155544F4C4556454C00505233
:1004A000494E545F4A4F420050524F4752455353B2
:1004B000004155544F5245504F52545F54454D5092
:1004C00000564F4C554D45545249430045455052F6
:1004D0004F4D0053455249414C5F584F4E5F584F66
:1004E0004646004649524D574152455F4E414D45A3
:1004F0003A4D61726C696E20312E312E39202847B9
:1005000069746875622920534F555243455F434FC4
:1005100044455F55524C3A68747470733A2F2F6794
:1005200069746875622E636F6D2F4D61726C696EB0
:100530004669726D776172652F4D61726C696E20CC
:1005400050524F544F434F4C5F56455253494F4EB4
:100550003A312E30204D414348494E455F54595061
:10056000453A3344205072696E7465722045585480
:1005700052554445525F434F554E543A31205555DC
:1005800049443A63656465326132662D34316132C3
:100590002D343734382D396231322D633535633699
:1005A000326633363766660A002F2F20002054004B
:1005B000205200416363656C65726174696F6E3AC5
:1005C0002050005741524E494E4721204C6F772012
:1005D0005A204A65726B206D6179206C65616420D8
:1005E000746F20756E77616E7465642070617573C9
:1005F00065732E0A00546F6F206661722066726FF9
:100600006D207265666572656E636520706F696ED8
:10061000740A0020466C6F773A20000001363726B6
:10062000032BFFFFFF3C3D382AFFFFFFFF2E303E2C
:1006300012FFFFFFFFFFFFFF0809FF2C071A1C181E
:10064000FFFFFF08440A2C4324221E20643A0020A6
:10065000693A0020703A00496E76616C69642065E1
:10066000787472756465720A0043290A0061626CCD
:10067000656420286D696E2074656D702000436F7D
:100680006C6420657874727564657320617265208E
:100690000020643A0020693A0020703A004E6F2032
:1006A00063617365206C696768740A004545505240
:1006B0004F4D204F4B0A00205A004475616C204575
:1006C0006E6473746F702041646A7573746D656EC7
:1006D0007420286D6D293A20003F4B2076616C759F
:1006E00065206F7574206F662072616E67652028C3
:1006F000302D3130292E0A00416476616E63652009
:100700004B3D004163746976652045787472756469
:1007100065723A2000496E76616C69642065787470
:1007200072756465720A0043616E6E6F7420656E47
:10073000746572207375626469723A2000473931BA
:100740000A4731205A2D302E310A47393000537074
:10075000656369616C204D656E753A205A20446F5F
:10076000776E20302E310A004739310A4731205A3E
:100770002D302E30320A473930005370656369617D
:100780006C204D656E753A205A20446F776E20308C
:100790002E30320A004739310A4731205A2B302E89
:1007A00030320A473930005370656369616C204DFF
:1007B000656E753A205A20557020302E30320A006E
:1007C0004739310A4731205A2B302E310A47393008
:1007D000005370656369616C204D656E753A205AEF
:1007E00020557020302E310A004732392053320014
:1007F0005370656369616C204D656E753A204E6576
:100800007874204D65736820506F696E740A0047D4
:100810003239205331005370656369616C204D6536
:100820006E753A205374617274204D657368204C64
:100830006576656C696E670A004D31343020533639
:1008400030005370656369616C204D656E753A20A8
:1008500050726568656174204265640A004D3530E8
:1008600031005370656369616C204D656E753A2087
:100870004C6F61642046572044656661756C7473E3
:100880000A004D353030005370656369616C204D4E
:10089000656E753A205361766520454550524F4D3F
:1008A0000A004D33303320452D312053363020435C
:1008B00036205531005370656369616C204D656E5B
:1008C000753A204175746F2054756E6520486F74B9
:1008D000626564205069640A004D3130362053311E
:1008E00037380A4D333033204530205332313020F1
:1008F0004336205531005370656369616C204D6546
:100900006E753A204175746F2054756E6520486F7E
:1009100074656E64205049440A003C5370656369F5
:10092000616C5F4D656E753E003C53706563696137
:100930006C5F4D656E753E002F002F002F002F2E2F
:100940002E0A002F2E2E002F2E2E003C5370656392
:1009500069616C5F4D656E753E0A003C537065635E
:1009600069616C204D656E753E003C53706563692E
:10097000616C204D656E753E003C4C6F6164204695
:10098000572044656661756C74733E003C4C6F6122
:10099000642046572044656661756C74733E003C64
:1009A0004175746F2054756E6520486F746265647C
:1009B000205049443E003C4175746F2054756E656B
:1009C00020486F74626564205049443E003C417584
:1009D000746F2054756E6520486F74656E64205086
:1009E00049443E003C4175746F2054756E65204843
:1009F0006F74656E64205049443E003C45786974CC
:100A00003E003C457869743E003C53617665204564
:100A10004550524F4D3E003C536176652045455050
:100A2000524F4D3E003C4E657874204D65736820F2
:100A3000506F696E743E003C4E657874204D65734E
:100A40006820506F696E743E003C5374617274206C
:100A50004D657368204C6576656C696E673E003C39
:100A60005374617274204D657368204C6576656CB3
:100A7000696E673E003C507265686561742062650E
:100A8000643E003C50726568656174206265643E36
:100A9000003C5A20446F776E20302E313E003C5A85
:100AA00020446F776E20302E313E003C5A20446F38
:100AB000776E20302E30323E003C5A20446F776EE5
:100AC00020302E30323E003C5A20557020302E30DF
:100AD000323E003C5A20557020302E30323E003CD1
:100AE0005A20557020302E313E003C5A205570203F
:100AF000302E313E0056313136004A333320004D1E
:100B00003530300A4D3432302053310A4731205AC3
:100B1000313020463234300A4731205830205930A5
:100B2000204636303030004A3232004A32320047F6
:100B300031205A3520463234300A47312058313975
:100B400030205932302046363030300A4731205A72
:100B5000302046323430004731205A352046323476
:100B6000300A473120583139302059313930204648
:100B7000363030300A4731205A3020463234300087
:100B80004731205A3520463234300A473120583117
:100B90003930205932302046363030300A47312043
:100BA0005A302046323430004739310A4731205A12
:100BB000313020463234300A4739300A4732380A59
:100BC0004732390A473120583230205932302046D6
:100BD000363030300A4731205A3020463234300027
:100BE0004A3032004A3132004731205A3130004F0A
:100BF0004B004731205A313000473930004731200F
:100C00004525694635303000473120452D302E319D
:100C10004625690047312045302E31462569004779
:100C200031205A2569462569004731205A2D302E3A
:100C300031462569004731205A302E31462569005A
:100C400047312059256946256900473120592D3003
:100C50002E314625690047312059302E314625690D
:100C60000047312058256946256900473120582D15
:100C7000302E314625690047312058302E31462527
:100C800069004739310047323800473238205A006E
:100C90004732382059004732382058004132305608
:100CA00020004731205A3130004A3034004A323176
:100CB000004A3230004B494C4C45442E20004A300B
:100CC0003400454E4400464E20004A303200393947
:100CD000393A393939004D00480041375620004132
:100CE0003656202D2D2D004A303200413656200038
:100CF0005A3A2000593A2000583A2000413556000F
:100D000041345620004133562000413256200041E4
:100D10003156200041305620004D3834004A3136DB
:100D2000004A3138004739310A4731205A313020E2
:100D3000463234300A473930004A3134004A3030C4
:100D4000004A3031004A31300024F4D43050C38E90
:100D500020C2A24017828B7011127A910D816CD93A
:100D60000AA861E108C7586607615143061E4B5D3A
:100D700005C145A7041A411104093D980371393191
:100D8000034036DB0265339102D4305402802E1DBD
:100D900002632CEE01752AC501B028A0011027813D
:100DA000018F2564012B244B01E0223401AC211F6B
:100DB000018D200D01801FFC00841EED00971DDFBA
:100DC00000B81CD200E61BC600201BBC00641AB28F
:100DD00000B219A8000A19A0006A189900D1179149
:100DE0000040178B00B516840031167E00B31579CC
:100DF000003A157300C7146F0058146A00EE1366AA
:100E0000008813630025135E00C7125B006C125745
:100E10000015125400C111510070114F0021114BE7
:100E200000D61049008D10470046104400021042C1
:100E300000C00F4000800F3E00420F3C00060F3BF9
:100E400000CB0E3800930E37005C0E3500270E34B1
:100E500000F30D3200C10D3100900D3000600D2EF9
:100E600000320D2D00050D2C00D90C2B00AE0C29E5
:100E700000850C29005C0C2700350C27000E0C2681
:100E800000E80B2400C40B2400A00B23007D0B23DF
:100E9000005A0B2100390B2100180B2000F80A1F03
:100EA00000D90A1E00BB0A1E009D0A1D00800A1DF3
:100EB00000630A1C00470A1B002C0A1B00110A1AB7
:100EC00000F7091A00DD091900C4091900AB091956
:100ED00000920917007B091800630917004C0916D6
:100EE0000036091600200916000A091500F5081534
:100EF00000E0081400CC081400B8081400A408147A
:100F000000900813007D0812006B081300580812A7
:100F100000460812003408110023081100120811BD
:100F20000001081100F0071000E0071000D00710C2
:100F300000C0071000B0070F00A107100091070EB6
:100F40000083070F0074070F0065070E0057070E98
:100F50000049070E003B070D002E070E0020070D6D
:100F60000013070D0006070D00F9060C00ED060D35
:100F700000E0060C00D4060C00C8060C00BC060CF1
:100F800000B0060C00A4060B0099060C008D060BA1
:100F90000082060B0077060B006C060B0061060A48
:100FA0000057060B004C060A0042060A0038060AE3
:100FB000002E060A0024060A001A060A0010060976
:100FC0000007060A00FD050900F4050900EB050904
:100FD00000E2050900D9050900D0050900C7050987
:100FE00000BE050900B5050800AD050800A5050906
:100FF000009C050800940508008C0508008405087D
:10100000007C050800740508006C050700650508EC
:10101000005D050700560508004E05070047050757
:10102000004005080038050700310507002A0507BC
:1010300000230507001C050600160507000F05071D
:10104000000805060002050700FB040600F504077A
:1010500000EE040600E8040600E2040700DB0406D4
:1010600000D5040600CF040600C9040600C3040628
:1010700000BD040600B7040600B1040500AC040678
:1010800000A6040600A00405009B040600950405C4
:1010900000900406008A040500850405008004060B
:1010A000007A04050075040500700405006B040552
:1010B0000066040500610405005C04050057040592
:1010C00000520405004D04050048040500430405D2
:1010D000003E0404003A0405003504050030040411
:1010E000002C04050027040400230405001E04044A
:1010F000001A04040016040500110404000D040481
:1011000000090405000404040000040400FC0304B6
:1011100000F8030400F4030400F0030400EC0304EB
:1011200000E8030400E4030400E0030400DC03041B
:1011300000D8030400D4030400D0030400CC03044B
:1011400000C8030300C503030024F404D9201BC412
:101150000C5C0E9804C4095F0265077101F405F97F
:1011600000FB04B30048048700C10369005803551D
:101170000003034500BE023A008402310053022AF4
:10118000002902250004022000E4011C00C8011906
:1011900000AF0117009801140084011300710110C1
:1011A000006101100051010E0043010D0036010BDA
:1011B000002B010B0020010B00150109000C010997
:1011C0000003010800FB000800F3000800EB000723
:1011D00000E4000600DE000600D8000600D200068B
:1011E00000CC000500C7000500C2000500BD0004DA
:1011F00000B9000400B5000400B1000400AD000413
:1012000000A9000400A5000300A20003009F000441
:10121000009B000300980003009500020093000368
:1012200000900003008D0002008B00030088000284
:10123000008600020084000300810002007F00029B
:10124000007D0002007B00020079000200770001AF
:1012500000760002007400020072000100710002BA
:10126000006F0002006D0001006C0002006A0001C6
:1012700000690002006700010066000100650001CE
:1012800000640002006200010061000100600001D2
:10129000005F0002005D0001005C0001005B0001D6
:1012A000005A0001005900010058000100570001D8
:1012B00000560001005500010054000100530000D9
:1012C00000530001005200010051000100500001D4
:1012D000004F0001004E0000004E0001004D0001D3
:1012E000004C0001004B0000004B0001004A0001CF
:1012F00000490001004800000048000100470001CB
:1013000000460000004600010045000000450001C5
:1013100000440001004300000043000100420000BF
:1013200000420001004100000041000100400001B6
:10133000003F0000003F0001003E0000003E0001B1
:10134000003D0000003D0001003C0000003C0000AA
:10135000003C0001003B0000003B0001003A00009F
:10136000003A000100390000003900010038000097
:10137000003800000038000100370000003700018D
:101380000036000000360000003600010035000085
:10139000003500000035000100340000003400007A
:1013A000003400010033000000330000003300016E
:1013B0000032000000320000003200010031000065
:1013C000003100000031000100300000003000005A
:1013D00000300001002F0000002F0000002F00004F
:1013E000002F0001002E0000002E0000002E000142
:1013F000002D0000002D0000002D0000002D000138
:10140000002C0000002C0000002C0000002C00012B
:10141000002B0000002B0000002B0000002B00011F
:10142000002A0000002A0000002A0000002A000113
:101430000029000000290000002900000029000008
:1014400000290001002800000028000000280000FA
:1014500000280000002800010027000000270000ED
:1014600000270000002700000027000100260000E0
:1014700000260000002600000026000000260001D3
:1014800000250000002500000025000000250000C8
:1014900000250000002500010024000000240000B9
:1014A00000240000002400000024000100230000AC
:1014B00000230000002300000023000000230000A0
:1014C0000023000000230001002200000022000091
:1014D0000022000000220000002200000022000183
:1014E0000021000000210000002100000021000078
:1014F0000021000000210000002100010020000068
:10150000002000000020000000200000002000005B
:10151000002000000020000000200001001F00004B
:10152000001F0000001F0000001F0000001F00003F
:10153000001F0000001F0001001E0000001E000030
:10154000001E0000001E000000232C0000B8220036
:1015500000561800003A0F0000B8080000B104005F
:1015600000710200003E010000696E206D6F76651B
:101570005F746F282920666565645F76616C7565A8
:1015800020666F722058593A002C2065793D002959
:10159000202D3E202865783D002C2073793D0020C9
:1015A000436F6E6E656374696E6720776974682037
:1015B000766572746963616C206C696E652028734E
:1015C000783D002C2065793D0029202D3E2028659E
:1015D000783D002C2073793D0020436F6E6E65636B
:1015E00074696E67207769746820686F72697A6FB2
:1015F0006E74616C206C696E65202873783D003FC5
:1016000053706563696669656420582C5920636F5F
:101610006F7264696E617465206F7574206F6620E7
:10162000626F756E64732E0A003F285229657065DB
:1016300061742076616C7565206E6F7420706C61CA
:10164000757369626C653B206D75737420626520EB
:101650006174206C6561737420312E0A003F28523A
:10166000296570656174206D7573742062652073DF
:101670007065636966696564207768656E206E6F62
:1016800074207573696E6720616E204C43442E0A86
:10169000003F537065636966696564206E6F7A7A8E
:1016A0006C652074656D7065726174757265206E0D
:1016B0006F7420706C61757369626C652E0A003FEF
:1016C0005370656369666965642066696C616D6500
:1016D0006E742073697A65206E6F7420706C61750A
:1016E0007369626C652E0A003F53706563696669B1
:1016F0006564207072696D65206C656E6774682022
:101700006E6F7420706C61757369626C652E0A006F
:101710003F5072696D65206C656E677468206D75E9
:1017200073742062652073706563696669656420FF
:101730007768656E206E6F74207573696E672061BF
:101740006E204C43442E0A003F53706563696669FE
:101750006564206E6F7A7A6C652073697A65206E95
:101760006F7420706C61757369626C652E0A003F3E
:10177000537065636966696564205265747261635C
:1017800074696F6E204D756C7469706C6965722038
:101790006E6F7420706C61757369626C652E0A00DF
:1017A0003F52657472616374696F6E204D756C741D
:1017B00069706C696572206D757374206265207341
:1017C00070656369666965642E0A003F53706563DE
:1017D0006966696564206C6179657220686569670E
:1017E0006874206E6F7420706C61757369626C65CB
:1017F0002E0A003F537065636966696564206265FF
:10180000642074656D7065726174757265206E6FA9
:101810007420706C61757369626C65202834302D9A
:1018200031343043292E0A0047323620636F6D6D04
:10183000616E6420737461727465642E20576169EF
:1018400074696E6720666F722068656174657228BE
:1018500073292E0A00024A3135004A3132004A31DA
:1018600037002020506C616E6E6572427566666549
:101870007242797465733A20002046726565204D86
:10188000656D6F72793A2000436F6D70696C6564A5
:101890003A2044656320323720323031380A002044
:1018A0007C20417574686F723A202864617669649F
:1018B00072616D69726F2C20666F7220416E796360
:1018C00075626963206933204D656761290A0032BA
:1018D0003031382D31322D323400204C6173742078
:1018E000557064617465643A2000312E312E390AD6
:1018F000004D61726C696E0020536F66747761727F
:10190000652052657365740A0020576174636864CA
:101910006F672052657365740A002042726F776E9C
:10192000206F75742052657365740A0020457874C1
:1019300065726E616C2052657365740A00506F7732
:10194000657255700A0073746172740A004D323406
:10195000004D3233202573006175746F25692E6741
:10196000006572726F722077726974696E67207495
:101970006F2066696C650A00205A3A0020593A00C7
:1019800020583A00656E6473746F707320686974D0
:101990003A2000446F6E6520736176696E67206639
:1019A000696C652E0A004D32390020746F6F206C0F
:1019B0006F6E6720657874727573696F6E207072D0
:1019C0006576656E7465640A0020636F6C642065DB
:1019D0007874727573696F6E2070726576656E7457
:1019E00065640A00454550524F4D2064617461732F
:1019F000697A65206572726F722E0A00290A0020CA
:101A000062797465733B206372632000536574745C
:101A1000696E67732053746F726564202800290A09
:101A2000002062797465733B206372632000207329
:101A3000746F7265642073657474696E6773207265
:101A40006574726965766564202800202863616C7E
:101A500063756C6174656429210A0020213D2000B2
:101A6000454550524F4D20435243206D69736D617F
:101A7000746368202D202873746F726564292000B8
:101A80002053697A653A2000496E6465783A2000EF
:101A9000204D61726C696E3D563535290A00284526
:101AA0004550524F4D3D00454550524F4D207665B3
:101AB0007273696F6E206D69736D61746368200065
:101AC0001000C90210012C0140012201700118010F
:101AD000B0010E01F00104015002FA00B002F00062
:101AE0003003E600D003DC009004D2007005C8008B
:101AF000A006BE000008B400B009AA00D00BA000E8
:101B0000600E960060118C0000158200201978008C
:101B1000C01D6E00A0226400B0275A00902C500017
:101B200000314600E0343C0010383200903A280082
:101B3000603C1E00A03D1400803E0A00203F0000D3
:101B40002CFFFFFFFFFF0001010101016265640A34
:101B5000002C2073797374656D2073746F707065D9
:101B60006421204865617465725F49443A200042EF
:101B700065642068656174696E67206661696C657B
:101B8000640048656174696E67206661696C6564AC
:101B90000045312048656174696E67206661696C33
:101BA00065640048656174696E67206661696C658B
:101BB000640070012C0190012701B0012201C001D5
:101BC0001D01F00118011002130130020E01600224
:101BD000090190020401C002FF000003FA00400363
:101BE000F5008003F000D003EB002004E600700451
:101BF000E100E004DC004005D700C005D20040064B
:101C0000CD00D006C8008007C3003008BE00F00831
:101C1000B900C009B400B00AAF00B00BAA00D00CE4
:101C2000A500000EA000500F9B00C010960050129F
:101C3000910000148C00C0158700B0178200B01905
:101C40007D00D01B7800001E730040206E009022A3
:101C50006900F024640040275F0090295A00E02BBF
:101C60005500102E500020304B0010324600E0335B
:101C7000410090353C001037370070383200A039F1
:101C80002D00B03A2800A03B2300603C1E00103D10
:101C90001900903D1400103E0F00703E0A00C03E37
:101CA0000500003F0000403FFBFF803FF6FFC03FC4
:101CB000F1FF453120544845524D414C2052554E7C
:101CC000415741590042454420544845524D414CEA
:101CD0002052554E4157415900546865726D616CF0
:101CE0002052756E61776179004531204572723AF4
:101CF000204D415854454D50004572723A204D4197
:101D00005854454D5020424544004D415854454D8E
:101D100050207472696767657265640045312045BB
:101D200072723A204D494E54454D50004572723AF8
:101D3000204D494E54454D5020424544004D494E9A
:101D400054454D5020747269676765726564004D33
:101D5000383420582059205A204500202F00204296
:101D6000403A0020403A006F70656E206661696CF1
:101D700065642C2046696C653A200043616E6E6F85
:101D800074206F70656E2073756264697220004AFA
:101D90003035004A3233004739310A4731205A2D55
:101DA000313020463234300A473930005344206302
:101DB000617264206F6B0A006F70656E526F6F7492
:101DC000206661696C65640A00766F6C756D652EBE
:101DD000696E6974206661696C65640A0045727297
:101DE0006F723A00534420696E6974206661696CB1
:101DF0000A006563686F3A00656E7175657565699F
:101E00006E672022004B494C4C45442E20005072F6
:101E1000696E7465722073746F7070656420647588
:101E20006520746F206572726F72732E2046697818
:101E300020746865206572726F7220616E6420750F
:101E40007365204D39393920746F20726573746160
:101E500072742E202854656D706572617475726598
:101E60002069732072657365742E20536574206930
:101E7000742061667465722072657374617274692E
:101E80006E67290A004E6F20436865636B73756D3A
:101E90002077697468206C696E65206E756D626567
:101EA000722C204C617374204C696E653A20004E90
:101EB0006F20436865636B73756D20776974682064
:101EC0006C696E65206E756D6265722C204C617355
:101ED00074204C696E653A2000636865636B7375A6
:101EE0006D206D69736D617463682C204C6173742F
:101EF000204C696E653A20004C696E65204E756D08
:101F0000626572206973206E6F74204C6173742057
:101F10004C696E65204E756D6265722B312C204CBC
:101F2000617374204C696E653A20004D3131300088
:101F30004D33310053442072656164206572726FC5
:101F4000720A00446F6E65207072696E74696E6704
:101F50002066696C650A00205A3A0020593A002030
:101F6000436F756E7420583A0020453A00205A3A63
:101F70000020593A00583A003A004361703A002074
:101F80005A00205900580020204D61783A20002046
:101F90005A00205900580020204D696E3A20004F09
:101FA0006E20004F666600536F667420656E647322
:101FB000746F70733A20004B642000236465666977
:101FC0006E652044454641554C545F004B692000E6
:101FD00023646566696E652044454641554C545FEF
:101FE000004B70200023646566696E652044454699
:101FF00041554C545F00504944204175746F7475CD
:102000006E652066696E6973686564212050757419
:1020100020746865206C617374204B702C204B69B0
:1020200020616E64204B6420636F6E7374616E7404
:10203000732066726F6D2062656C6F7720696E74B5
:102040006F20436F6E66696775726174696F6E2E7B
:10205000680A00504944204175746F74756E65209C
:102060006661696C6564212074696D656F75740AB9
:1020700000453120544845524D414C2052554E4167
:102080005741590042454420544845524D414C2047
:1020900052554E4157415900546865726D616C202C
:1020A00052756E61776179004531204865617469C8
:1020B0006E67206661696C656400426564206865CE
:1020C0006174696E67206661696C6564004865616A
:1020D00074696E67206661696C65640050494420CC
:1020E0004175746F74756E65206661696C656421F5
:1020F0002054656D706572617475726520746F6FC0
:1021000020686967680A00204B643A2000204B6908
:102110003A2000204B703A20000A20436C61737310
:10212000696320504944200A002054753A20002059
:102130004B753A2000206D61783A2000206D696E61
:102140003A200020643A200020626961733A20003E
:10215000504944204175746F74756E6520666169DD
:102160006C656421204261642065787472756465D1
:1021700072206E756D6265720A0050494420417587
:10218000746F74756E652073746172740A004F66A3
:10219000660A0046616465204865696768742000C6
:1021A000426564204C6576656C696E672000466107
:1021B000696C656420746F20656E61626C65204295
:1021C0006564204C6576656C696E670A004D6573C1
:1021D0006820426564204C6576656C20646174619A
:1021E0003A0A004D65736820706F696E74206361F0
:1021F0006E6E6F74206265207265736F6C766564B5
:102200000A004D34323120696E636F7272656374F7
:1022100020706172616D65746572207573616765A8
:102220000A007C3C3E5E2B3D3F2F5B5D3B2C2A220F
:102230005C00627573793A2070617573656420661D
:102240006F7220696E7075740A00627573793A2036
:1022500070617573656420666F7220757365720AAC
:1022600000627573793A2070726F63657373696E7B
:10227000670A004A3135004B494C4C45442E20003A
:102280004B494C4C20636175736564206279204B27
:10229000494C4C20627574746F6E2F70696E0A0021
:1022A0004B494C4C45442E20004B494C4C2063611B
:1022B0007573656420627920746F6F206D75636833
:1022C00020696E6163746976652074696D65202D7F
:1022D0002063757272656E7420636F6D6D616E64DC
:1022E0003A20004A3131005072696E74657220687C
:1022F000616C7465642E206B696C6C2829206361A5
:102300006C6C6564210A000000A0C00000000000A1
:102310000000005761726E696E673A20486F6D6900
:102320006E672042756D702044697669736F722004
:102330003C20310A000202040000A0400000A0403E
:10234000000000400000614300005C4300004D437A
:10235000FFFFFF20496E76616C69642065787472B6
:102360007564657220000000A0C00000000000003D
:10237000000000005C4300005C4300004D43486FD8
:102380006D696E67206661696C656400206E6F74AC
:1023900020656E74657265642E0A0046696C65205E
:1023A00064656C657465643A0044656C6574696F56
:1023B0006E206661696C65642C2046696C653A2004
:1023C0000050726F7465637465642050696E0A0012
:1023D0004A3036004A3034004A30370020573A003D
:1023E0004A3038004A30390020573A0000002100B6
:1023F000240027002A002D003000330001010000D6
:10240000040107010A0100002200250028002B001A
:102410002E003100340002010000050108010B010B
:10242000000020002300260029002C002F0032008D
:102430000001000003010601090105050505070566
:1024400008080808020202020A0A08080404040430
:10245000010101010101010103030303030303035C
:10246000040707070C0C0C0C0C0C0C0C02020202EB
:1024700006060606060606060B0B0B0B0B0B0B0BD4
:102480000102102020080810204010204080020186
:10249000020108040201010204081020408080406B
:1024A000201008040201800402018040201008046A
:1024B0000201080402010102040810204080010208
:1024C00004081020408000000A0B02090C0D0E08C1
:1024D00007030401000000000000000000000000ED
:1024E00000000000000000000000000000000000EC
:1024F00000001211100000000000000000000000A9
:10250000000000000000000000000000556E6B6E2F
:102510006F776E20636F6D6D616E643A20220020CC
:1025200066697273740A005A0059005800486F6D4A
:102530006520000000484200004842000080400042
:10254000000000545249474745524544006F7065AA
:102550006E003A20007A325F6D696E007A5F6D69B5
:102560006E00795F6D696E00785F6D696E0052650F
:10257000706F7274696E6720656E6473746F70201B
:102580007374617475730A000A4D656173757265C1
:102590006420706F696E74733A0A005A206F666621
:1025A0007365743A20004E756D20582C593A2035C9
:1025B0002C350A000000000100000001000080002E
:1025C000555555000000400033333300AAAA2A00B5
:1025D0004992240000002000C7711C00999919003D
:1025E000D1451700555515003BB113002449120081
:1025F00011111100000010000F0F0F00E3380E0042
:1026000043790D00CCCC0C00C3300C00E8A20B00C9
:1026100064210B00AAAA0A00703D0A009DD8090097
:10262000427B090092240900DCD308008888080056
:102630001042080000000800F0C10700878707006B
:1026400075500700711C07003EEB0600A1BC060098
:102650006990060066660600703E06006118060076
:1026600017F4050074D105005BB00500B2900500B9
:10267000627205005555050078390500B81E050041
:10268000050505004EEC040087D40400A1BD04003C
:1026900090A7040049920400C17D0400EE69040083
:1026A000C7560400444404005C32040008210400BE
:1026B00041100400000004003FF00300F8E00300B4
:1026C00026D20300C3C30300CCB503003AA803001D
:1026D0000A9B0300388E0300C08103009F7503002E
:1026E000D0690300505E03001D530300344803000B
:1026F000913D03003333030016290300381F030004
:1027000097150300300C0300030303000BFA0200CB
:1027100049F10200BAE802005CE002002DD8020094
:102720002DD0020059C80200B0C0020031B9020029
:10273000DAB10200AAAA0200A0A30200BC9C020017
:10274000FA9502005C8F0200DF880200828202009C
:10275000457C02002776020027700200436A0200CF
:102760007C640200D05E02003F590200C8530200A0
:1027700048617264636F6465642044656661756C6A
:10278000742053657474696E6773204C6F6164655F
:10279000640A00D0070000D00700003C00000010D1
:1027A0002700000000FA430000FA430000C0400088
:1027B0000070420000A0420000A0420000C8433365
:1027C00033B94220286D6D290020204D393030204A
:1027D0004B004C696E65617220416476616E636581
:1027E0003A0A0020440020490020204D3330342094
:1027F000500020440020490020204D33303120502B
:10280000005049442073657474696E67733A0A0016
:10281000205A0020204D36363600456E6473746FA2
:10282000702061646A7573746D656E743A0A002075
:102830005A002059002020473239205333205800B5
:10284000205A0020204D3432302053004D657368EB
:1028500020426564204C6576656C696E673A0A00B3
:10286000205A0020590020204D3230362058004890
:102870006F6D65206F66667365743A0A00204500C7
:10288000205A0020590020580020540020530020D6
:10289000204D32303520510020453C6D61785F6518
:1028A0005F6A65726B3E0020583C6D61785F785FAF
:1028B0006A65726B3E20593C6D61785F795F6A652D
:1028C000726B3E205A3C6D61785F7A5F6A65726B0D
:1028D0003E00416476616E6365643A20513C6D69E7
:1028E0006E5F7365676D656E745F74696D655F7546
:1028F000733E20533C6D696E5F66656564726174FA
:10290000653E20543C6D696E5F74726176656C5FE4
:1029100066656564726174653E0020540020520053
:1029200020204D323034205000416363656C657265
:102930006174696F6E2028756E6974732F73322904
:102940003A20503C7072696E745F616363656C3EDF
:1029500020523C726574726163745F616363656C7D
:102960003E20543C74726176656C5F616363656C94
:102970003E0A00204500205A0020590020204D32F8
:1029800030312058004D6178696D756D2041636369
:10299000656C65726174696F6E2028756E697473F9
:1029A0002F7332293A0A00204500205A002059008E
:1029B00020204D3230332058004D6178696D756D9F
:1029C000206665656472617465732028756E69742C
:1029D000732F73293A0A00204500205A002059001D
:1029E00020204D3932205800537465707320706573
:1029F0007220756E69743A0A0020204D3230302002
:102A000044300A0020204D323030204400204469F8
:102A10007361626C65640A0046696C616D656E7411
:102A20002073657474696E67733A002020473231F1
:102A3000202020203B00FFFDFCFAF8F6F4F2F0EE37
:102A4000ECEAE9E7E5E3E1E0DEDCDAD9D7D5D4D298
:102A5000D0CFCDCBCAC8C7C5C3C2C0BFBDBCBAB931
:102A6000B7B6B4B3B2B0AFADACAAA9A8A6A5A4A29C
:102A7000A1A09E9D9C9A99989795949392908F8EE1
:102A80008D8B8A8988878684838281807F7E7D7B07
:102A90007A797877767574737271706F6E6D6C6B0E
:102AA0006A696867666564636261605F5E5D5C5BFE
:102AB0005A5958585756555453525150504F4E4DDD
:102AC0004C4B4A4A494847464645444342424140A6
:102AD0003F3E3E3D3C3B3B3A39383837363535345E
:102AE0003332323130302F2E2E2D2C2B2B2A292908
:102AF00028272726252524232322212120201F1EA5
:102B00001E1D1C1C1B1B1A19191818171616151533
:102B100014131312121111100F0F0E0E0D0D0C0CB9
:102B20000B0A0A0909080807070606050504040335
:102B3000030202010000526573656E643A20006F63
:102B40006B0020746F6F206C6F6E672065787472F5
:102B50007573696F6E2070726576656E7465640A50
:102B60000020636F6C6420657874727573696F6E92
:102B70002070726576656E7465640A004572726FC6
:102B8000722077726974696E6720746F20454550B2
:102B9000524F4D210A0057726974696E6720746F35
:102BA0002066696C653A20006F70656E2066616909
:102BB0006C65642C2046696C653A20006F70656E08
:102BC000206661696C65642C2046696C653A20005A
:102BD00046696C652073656C65637465640A0020E2
:102BE00053697A653A200046696C65206F70656E9E
:102BF00065643A20002066696C653A2000646F695C
:102C00006E67006672657368004E6F772000454EF0
:102C10004420535542524F5554494E450A002220F4
:102C2000706F73002220706172656E743A220053D7
:102C30005542524F5554494E452043414C4C207407
:102C400061726765743A22004B494C4C45442E2012
:102C500000747279696E6720746F2063616C6C20F8
:102C60007375622D67636F64652066696C65732098
:102C70007769746820746F6F206D616E79206C6560
:102C800076656C732E204D4158206C6576656C20FE
:102C900069733A0095DF4BE111241FBECFEFD1E2FB
:102CA000DEBFCDBF00E00CBF14E0A0E0B2E0E0E585
:102CB000FCED01E00BBF02C007900D92A831B107F7
:102CC000D9F728E1A8E1B4E001C01D92AC3CB207FD
:102CD000E1F716E1CBE4D6E100E006C02197010957
:102CE000802FFE010E9480EDCA34D10780E00807E2
:102CF000A9F70E94F5D90C9417EE0C9400002F92BE
:102D00003F924F925F926F927F928F929F92AF927B
:102D1000BF92CF92DF92EF92FF920F931F93CF93C8
:102D2000DF93CDB7DEB7CA58D1090FB6F894DEBF2E
:102D30000FBECDBF21E020934310809119188D3430
:102D400011F40C947D21843511F40C94A52E873454
:102D500011F00C94F12E80911718909118188A3167
:102D6000910509F4BEC79CF4843091053CF482308F
:102D70009105B4F597FF2DC00C947921843091050D
:102D800009F4D2C1059709F40EC20C9479218A3254
:102D9000910511F40C9470204CF48C31910509F4D8
:102DA000A4C74D9709F4A6C70C9479218B359105DA
:102DB00011F40C94FB208C35910511F40C94FF2038
:102DC0008A35910511F00C94792110922B040C9402
:102DD000F32E8091270281110C94F82E0C94F32E7F
:102DE00020912702222311F40C94F32E11E0029774
:102DF00009F010E00E94A6AA19821A821B821C8286
:102E00001D821E821F82188682E50E94914C8823B3
:102E100009F43AC10E94114C4B015C0120E030E002
:102E2000A9010E9438E6882309F444C1C090360401
:102E3000D0903704E0903804F0903904CCAADDAA91
:102E4000EEAAFFAAC0903A04D0903B04E0903C0464
:102E5000F0903D04C8AED9AEEAAEFBAEC090B21061
:102E6000D090B310E090B410F090B510CCAEDDAEC1
:102E7000EEAEFFAEC090B610D090B710E090B81094
:102E8000F090B9102496CCAEDDAEEEAEFFAE249736
:102E90002CAD3DAD4EAD5FAD6CA97DA98EA99FA9AE
:102EA0000E9438E681110BC0A701960168AD79AD8B
:102EB0008AAD9BAD0E9438E6882309F4FBC020E070
:102EC00030E0A901C501B4010E9438E6881F8827B7
:102ED000881F181739F0C12CD12C80E8E82E8FEB11
:102EE000F82E06C0C12CD12C00E8E02E0FE3F02E06
:102EF0002C96CCAEDDAEEEAEFFAE2C972CA93DA944
:102F00004EA95FA96CAD7DAD8EAD9FAD0E9483EAE9
:102F100028966CAF7DAF8EAF9FAF289728AD39ADA7
:102F20004AAD5BAD24966CAD7DAD8EAD9FAD249763
:102F30000E9483EA6B017C0128962CAD3DAD4EAD1D
:102F40005FAD2897CA01B9010E949DE62B013C01A3
:102F5000A7019601C701B6010E949DE69B01AC0145
:102F6000C301B2010E9484EA0E94EFEC2B013C01F4
:102F700020E030E040E05FE30E949DE660966CAFA9
:102F80007DAF8EAF9FAF6097A5019401C501B401DD
:102F90000E949DE64B015C0160962CAD3DAD4EADAF
:102FA0005FAD6097CA01B9010E949DE69B01AC012B
:102FB000C501B4010E9483EA0E94EFEC2C962CAD6F
:102FC0003DAD4EAD5FAD2C970E949DE64B015C017F
:102FD000C701B6019058A30192010E9460EBA501C0
:102FE00094010E949DE66B017C012CAD3DAD4EAD80
:102FF0005FAD6CA97DA98EA99FA90E9484EA20E0FB
:1030000030E040E05FE30E949DE69B01AC01C70118
:10301000B6010E9484EA2CA93DA94EA95FA90E948D
:1030200083EA69837A838B839C8324962CAD3DADA0
:103030004EAD5FAD249768AD79AD8AAD9BAD0E9472
:1030400084EA20E030E040E05FE30E949DE66B010F
:103050007C01A301920128966CAD7DAD8EAD9FAD34
:1030600028970E9460EBA50194010E949DE69B01B8
:10307000AC01C701B6010E9484EA28AD39AD4AAD62
:103080005BAD0E9483EA12C089E40E94914C8823C0
:1030900031F00E94114C69837A838B839C838AE48C
:1030A0000E94914C882331F00E94114C6D837E83E5
:1030B0008F83988720E030E0A90169817A818B8134
:1030C0009C810E9438E681110EC020E030E0A90109
:1030D0006D817E818F8198850E9438E6811103C0C1
:1030E000EDEDFDE10DC0412FBE016F5F7F4F82EB23
:1030F00090E10E94C8A40C94F32E0E94C689F801A6
:1031000084918F010F5F1F4F8111F7CFEDE1F2E046
:1031100084918F010F5F1F4F882311F40C94F32EBD
:103120000E94C689F801F4CF80E50E94914C882363
:1031300079F08091250490912604009749F04AE0A7
:1031400050E060E070E00E94B7E46B017C0103C0D6
:10315000C12CD12C760183E50E94914C882361F02B
:103160000E94114C20E030E04AE754E40E949DE6C2
:103170000E94CDEB6B017C010E94186A0E94F858F6
:10318000C60ED71EE81EF91E0E94F858DC01CB01BE
:103190008C199D09AE09BF09B7FD02C00C94F32E2E
:1031A0000E94FCA0F1CF80912702882311F40C9497
:1031B000F32E0E94A6AA89E40E94914C882329F04C
:1031C0000E94114C2B013C0103C0412C512C3201B7
:1031D0008AE40E94914C882329F00E94114C4B01F3
:1031E0005C0103C0812C912C540180E50E94914C1C
:1031F000882329F00E94114C6B017C0103C0C12C73
:10320000D12C760181E50E94914C882339F00E94EF
:10321000114C6CAB7DAB8EAB9FAB04C01CAA1DAA3E
:103220001EAA1FAA20914210C657DF4F2883CA58F2
:10323000D0406091020270910302072E000C880BAF
:10324000990B0E943EE6209130023091310240916C
:103250003202509133020E949DE62AE037ED43E2AC
:103260005CE30E949DE668AB79AB8AAB9BAB409177
:10327000360450913704609138047091390448AF96
:1032800059AF6AAF7BAF9A01AB01C301B2010E9493
:1032900084EAA1966CAF7DAF8EAF9FAFA1974090AF
:1032A0003A0450903B0460903C0470903D04A301AC
:1032B0009201C501B4010E9484EAA5966CAF7DAF6E
:1032C0008EAF9FAFA5972091B2103091B31040916F
:1032D000B4105091B510C701B6010E9484EAA996B6
:1032E0006CAF7DAF8EAF9FAFA9972091B610309194
:1032F000B7104091B8105091B9106CA97DA98EA952
:103300009FA90E9484EAAD966CAF7DAF8EAF9FAF50
:10331000AD97C8ACD9ACEAACFBACC982DA82EB821F
:10332000FC824D825E826F8278860E94F8589B01F3
:10333000AC0128533F4F4F4F5F4FCB57DF4F288390
:1033400039834A835B83C558D040BDEC8B2EBCECDF
:103350009B2EA92CBDE3BB2E25961FAE2597299643
:103360001FAE29972D961FAE2D9761961FAE6197C0
:103370000E94C97B0E94F8588B019C01CB57DF4FFC
:10338000C880D980EA80FB80C558D0400C191D093F
:103390002E093F0937FD10C09B01AC0128533F4F58
:1033A0004F4F5F4FCB57DF4F288339834A835B836F
:1033B000C558D0400E94FCA025967FAD2597299640
:1033C0006FAD29972D969FAD2D9761968FAD619723
:1033D000272F362F492F582FC501B4010E9484EAA8
:1033E0006CAB78AF8CAF21969FAF219720E030E097
:1033F00040E85FE30E94AAEC181644F41CAA18AE39
:1034000030E83CAF4FE321964FAF21976091B21067
:103410007091B3108091B4109091B510E1966CAF9B
:103420007DAF8EAF9FAFE1978091360490913704C6
:10343000A0913804B0913904E5968CAF9DAFAEAF42
:10344000BFAFE59721969FAD21979F93ACADAF930A
:10345000B8ADBF93ECA9EF93E196ACACBDACCEACEC
:10346000DFACE197A996ECACFDAC0EAD1FADA99712
:10347000A1962CAD3DAD4EAD5FADA197E5966CAD7F
:103480007DAD8EAD9FADE5970E9483C50F900F90E7
:103490000F900F9062966FAF629763967FAF6397BE
:1034A00064968FAF649765969FAF6597C090B6108E
:1034B000D090B710E090B810F090B910E996CCAE6B
:1034C000DDAEEEAEFFAEE99720913A0430913B04B9
:1034D00040913C0450913D04ED962CAF3DAF4EAF72
:1034E0005FAFED9721963FAD21973F934CAD4F9342
:1034F00058AD5F936CA96F93E996ACACBDACCEAC04
:10350000DFACE997AD96ECACFDAC0EAD1FADAD9761
:10351000A5962CAD3DAD4EAD5FADA597ED966CADCE
:103520007DAD8EAD9FADED970E9483C50F900F903E
:103530000F900F9066966FAF669767967FAF67970D
:1035400068968FAF689769969FAF699789819A81CE
:10355000AB81BC81C358DF4F88839983AA83BB8327
:10356000CD57D040CD80DE80EF80F884CF57DF4F3D
:10357000C882D982EA82FB82C158D0406A961FAEC7
:103580006A9725967FAD259729966FAD29972D9639
:103590009FAD2D9761968FAD6197272F362F492FBD
:1035A000582FBCA9A8ADFCAD2196EFAD21976B2F8C
:1035B0007A2F8F2F9E2F0E9483EA2FE632E143E07D
:1035C0005BE30E9438E687FD29C125967FAD2597EC
:1035D00029966FAD29972D969FAD2D9761968FAD4A
:1035E0006197272F362F492F582FBCA9A8ADFCADC6
:1035F0002196EFAD21976B2F7A2F8F2F9E2F0E9450
:1036000084EA20E030E040E05FE30E949DE6662E21
:10361000972E882E792E9F938F937F936F93E196A9
:10362000ACACBDACCEACDFACE197A996ECACFDACDC
:103630000EAD1FADA997A1962CAD3DAD4EAD5FADC2
:10364000A197E5966CAD7DAD8EAD9FADE5970E94DF
:1036500083C50F900F900F900F906B966FAF6B9785
:103660006C967FAF6C976D968FAF6D97C757DF4F96
:103670009883C958D0407F928F929F926F92E9961B
:10368000ACACBDACCEACDFACE997AD96ECACFDAC70
:103690000EAD1FADAD97A5962CAD3DAD4EAD5FAD5A
:1036A000A597ED966CAD7DAD8EAD9FADED970E946B
:1036B00083C50F900F900F900F90162F072FB82EE5
:1036C000A92E66962FAD669767963FAD6797689669
:1036D0004FAD689769965FAD6997CF57DF4F6881A7
:1036E00079818A819B81C158D0400E9484EA20E080
:1036F00030E040E05FE30E949DE61B012C016296F2
:103700002FAD629763963FAD639764964FAD649714
:1037100065965FAD6597C358DF4F688179818A816F
:103720009B81CD57D0400E9484EA20E030E040E009
:103730005FE30E949DE69B01AC016B966FAD6B97BA
:103740006C967FAD6C976D968FAD6D97C757DF4FB9
:103750009881C958D0400E9483EA6B017C0120E027
:1037600030E0A9010E94AAEC87FF04C0F7FAF094A8
:10377000F7F8F094A2019101612F702F8B2D9A2DF3
:103780000E9483EA1B012C0120E030E0A9010E9485
:10379000AAEC87FF04C057FA509457F85094A2013E
:1037A0009101C701B6010E9484EA2DEC3CEC4CEC7F
:1037B0005DE30E9438E618168CF566961FAF669793
:1037C00067960FAF67976896BFAE68976996AFAE7A
:1037D00069976B96DFAC6B976296DFAE62976C96DB
:1037E000EFAC6C976396EFAE63976D96FFAC6D97F9
:1037F0006496FFAE6497C757DF4F2881C958D04001
:1038000065962FAF65976CAA98AE8CAE21967FAE69
:10381000219731E06A963FAF6A97B3CE6A964FAD73
:103820006A97411144C125967FAD259729966FADC2
:1038300029972D969FAD2D9761968FAD6197272F74
:10384000362F492F582FBCA9A8ADFCAD2196EFAD5E
:1038500021976B2F7A2F8F2F9E2F0E9483EA6B0167
:103860007C012DEC3CEC4CEC5DE30E94AAEC1816BC
:103870000CF41DC1A7019601C701B6010E9484EA9C
:103880002596EFAD25972996BFAD29972D96AFAD1B
:103890002D976196FFAD61972E2F3B2F4A2F5F2FFB
:1038A0000E9484EA662E972E882E792E20E030E042
:1038B00040E85FE30E94AAEC87FFF9C07F928F92F5
:1038C0009F926F92E196ACACBDACCEACDFACE19711
:1038D000A996ECACFDAC0EAD1FADA997A1962CAD91
:1038E0003DAD4EAD5FADA197E5966CAD7DAD8EADB6
:1038F0009FADE5970E9483C50F900F900F900F909A
:103900006A966FAF6A976B967FAF6B976C968FAF27
:103910006C976D969FAF6D977F928F929F926F92EB
:10392000E996ACACBDACCEACDFACE997AD96ECACF7
:10393000FDAC0EAD1FADAD97A5962CAD3DAD4EAD1A
:103940005FADA597ED966CAD7DAD8EAD9FADED975E
:103950000E9483C50F900F900F900F90162F072F86
:10396000B82EA92E262F372F482F592FCF57DF4F8C
:10397000688179818A819B81C158D0400E9484EA04
:1039800020E030E040E05FE30E949DE66B017C01B7
:103990006A962FAD6A976B963FAD6B976C964FAD5D
:1039A0006C976D965FAD6D97C358DF4F68817981D5
:1039B0008A819B81CD57D0400E9484EA20E030E08C
:1039C00040E05FE30E949DE69B01AC0162966FAD13
:1039D000629763967FAD639764968FAD64976596A3
:1039E0009FAD65970E9483EA1B012C0120E030E027
:1039F000A9010E94AAEC87FF04C057FA509457F817
:103A00005094A701960166966FAD669767967FAD55
:103A1000679768968FAD689769969FAD69970E9482
:103A200083EA6B017C0120E030E0A9010E94AAEC4E
:103A300087FF04C0F7FAF094F7F8F094A20191011F
:103A4000C701B6010E9484EA2DEC3CEC4CEC5DE32E
:103A50000E94AAEC18165CF166961FAF66976796EF
:103A60000FAF67976896BFAE68976996AFAE6997D4
:103A70006A965FAD6A9762965FAF62976B966FAD1D
:103A80006B9763966FAF63976C967FAD6C976496F8
:103A90007FAF64976D968FAD6D9765968FAF659785
:103AA0006CAA98AE8CAE21967FAE2197BCCE25969F
:103AB0007FAD259729966FAD29972D969FAD2D97B0
:103AC00061968FAD6197272F362F492F582FBCA9AC
:103AD000A8ADFCAD2196EFAD21976B2F7A2F8F2FDC
:103AE0009E2F0E9483EA4B015C0162968FAD629724
:103AF00063969FAD63976496AFAD64976596BFADCF
:103B0000659789839A83AB83BC8366968FAD6697EE
:103B100067969FAD67976896AFAD68976996BFAD9A
:103B200069978D839E83AF83B8877CA968AD9CAD70
:103B300021968FAD2197272F362F492F582F60E0E0
:103B400070E080E89FE30E9483EA6B017C01209192
:103B50003E0430913F0440914004509141040E9442
:103B60009DE62B013C012091BA103091BB10409191
:103B7000BC105091BD10BCA9A8ADFCAD2196EFAD15
:103B800021976B2F7A2F8F2F9E2F0E949DE69B01EE
:103B9000AC01C301B2010E9484EA69877A878B87EE
:103BA0009C872091420430914304409144045091F9
:103BB0004504C701B6010E949DE66B017C0120917E
:103BC000BE103091BF104091C0105091C110BCA9DF
:103BD000A8ADFCAD2196EFAD21976B2F7A2F8F2FDB
:103BE0009E2F0E949DE69B01AC01C701B6010E9479
:103BF00084EA6D877E878F87988BCE0101960E941D
:103C0000C0C91CA61DA61EA61FA689819A81AB81CC
:103C1000BC8188A399A3AAA3BBA38D819E81AF81F8
:103C2000B8858CA39DA3AEA3BFA389859A85AB85D8
:103C3000BC8588A799A7AAA7BBA7AE01485D5F4F1F
:103C4000BE016C5D7F4FCE0180960E94C2BCDE013A
:103C50009C966D01C657DF4FE880CA58D0408E0150
:103C6000005D1F4F9E01235F3F4FAE01485D5F4FD8
:103C7000BE016C5D7F4FCE0180960E94F45988236F
:103C800029F120E030E040E85FE3BCA9A8ADFCAD3D
:103C90002196EFAD21976B2F7A2F8F2F9E2F0E94A9
:103CA00038E687FF13C03CA925963FAF259748AD5E
:103CB00029964FAF29975CAD2D965FAF2D97219632
:103CC0006FAD219761966FAF619752CB80E1E2EBC8
:103CD000F0E1A6E3B4E001900D928A95E1F70C942F
:103CE000F32E0E942E4E0C94F32E80E00E9446ACE0
:103CF0000C94F32E83E50E94914C882321F10E94BD
:103D0000F14B182F863070F0E5EEF2E084918F01D0
:103D10000F5F1F4F882311F40C94F32E0E94C68965
:103D2000F801F4CF833009F44AC130F4813091F1C5
:103D3000823009F43FC008C0843009F49FC1853047
:103D400009F4ACC101C010E00E94F9AB811103C0BD
:103D5000E5ECF2E013C080918010882319F063E154
:103D600073E002C067E173E08DEB92E00E9468C5EA
:103D70008AE00E94C6890E94FCBC96C184917F01A2
:103D8000BFEFEB1AFB0A882309F48EC10E94C68993
:103D9000F701F4CF0E94AFBD109201021092000211
:103DA00082EB92E09093A8078093A7070E94F28984
:103DB0000C94F32E809100029091010297FF0EC0A7
:103DC000E9E8F2E084918F010F5F1F4F882311F41F
:103DD0000C94F32E0E94C689F801F4CF0097A1F449
:103DE0008091520280932C0419821A821B821C82B9
:103DF00018A219A21AA21BA2BE016F5F7F4FCE01AB
:103E000080960E9445B427C0815065E00E944CED29
:103E100080FF03C024E0291B922F25E09202F001CD
:103E20001124E80FF11D87FDFA95EE0FFF1FEE0F2D
:103E3000FF1FE653FF4E80913E0490913F04A091F6
:103E40004004B091410480839183A283B383809125
:103E50002C048093520280910002909101028931DA
:103E600091050CF067C0109252029C012F5F3F4FEA
:103E7000309301022093000265E00E944CED80FF28
:103E800003C024E0291B922F40913E0450913F042F
:103E9000609140047091410448A359A36AA37BA395
:103EA00019821A821B821C8244E084029001112430
:103EB000B9016351764F4B01DB012D913D914D913D
:103EC0005C91B4E09B02C0011124FC01EF5FF54F4F
:103ED0005F016081718182819381DE0111966D01A4
:103EE000E12CF12C00EA10E40E9478B319821A82C6
:103EF0001B821C82B601CE0180960E9445B4F5015A
:103F000080819181A281B38180933604909337049C
:103F1000A0933804B0933904F40180819181A28187
:103F2000B38180933A0490933B04A0933C04B093F4
:103F30003D04BCC080E090E0A0EAB0E480933E0481
:103F400090933F04A0934004B09341040E9439AD84
:103F50000E94186A8FEF9FEF9093010280930002F6
:103F6000E5E7F2E084918F010F5F1F4F882321F076
:103F70000E94C689F801F6CF83E992E09A8389838B
:103F800004E610E019A308A3BE016F5F7F4FCE01C6
:103F900080960E9460B58AEB92E09A83898319A388
:103FA00008A3BE016F5F7F4FCE0180960E9460B56F
:103FB00081E00E9446AC81E00E9426AC77C088E593
:103FC0000E94914C8823A1F00E94E14B1FEF160F35
:103FD0001530A8F0EEE5F2E084918F010F5F1F4FDE
:103FE000882311F40C94F32E0E94C689F801F4CFB3
:103FF00088E50E94C6890E9487E10C94F32E89E52A
:104000000E94914C8823A1F00E94E14B0FEF060F14
:104010000530A8F0E7E4F2E084918F010F5F1F4FB5
:10402000882311F40C94F32E0E94C689F801F4CF72
:1040300089E50E94C6890E9487E10C94F32E8AE5E7
:104040000E94914C882399F00E94114C25E0129F08
:10405000F0011124E00FF11DEE0FFF1FEE0FFF1F07
:10406000E653FF4E608371838283938335C08AE574
:104070000E94C6890E9487E10C94F32E8AE50E9473
:10408000914C8823A1F30E94114C6093C610709349
:10409000C7108093C8109093C9101EC080E00E9482
:1040A00026AC0E94AFBD18C01230B1F4609100027E
:1040B000709101026931710514F069E170E088E3E3
:1040C00092E00E944FC569E170E083E392E00E94B4
:1040D0004FC58AE00E94C6890E9445950C94F32E34
:1040E00080912702882311F40C94F32E89E40E9416
:1040F000914CE82E882321F00E94E14B062F01C04D
:1041000000E08AE40E94914CF82E882321F00E945E
:10411000E14B162F01C010E0EE2011F0053020F425
:10412000FF2081F0153070F0ECEFF2E084918F0108
:104130000F5F1F4F882311F40C94F32E0E94C68941
:10414000F801F4CF0E949D4CEE2091F034E0030280
:10415000F0011124EF5FF54F80819181A281B3813D
:104160008093B2109093B310A093B410B093B51095
:10417000FF2091F044E01402F0011124E351F64FC6
:1041800080819181A281B3818093B6109093B71002
:10419000A093B810B093B91080E50E94914C882389
:1041A00019F00E94024C03C080E50E94484C86E44E
:1041B0000E94914C8823D9F00E94114C6B017C0124
:1041C00020E030E0A9010E94AAEC181684F420E057
:1041D00030E040E752E4C701B6010E9460EB609313
:1041E00030027093310280933202909333020E9426
:1041F00057CA0C94F32E20932B040C94F32E97E5BE
:10420000292E92E0392E21E5E22E20E1F22E66E3FE
:1042100074E07DAB6CAB38E1C32E34E0D32E00E00C
:1042200010E0D1018D911D010E94914C882309F469
:104230004BC00E94114C2B013C01133049F0F60198
:1042400020813181428153810E9483EA2B013C010C
:10425000ACA9BDA92D913D914D915C91C301B201D5
:104260000E9483EA4B015C012DEB37E346E855EBF6
:104270000E94AAEC87FD0AC02DEB37E346E855E320
:10428000C501B4010E9438E61816F4F4133051F455
:104290004092420450924304609244047092450458
:1042A00001E012C0A5019401F70160817181828152
:1042B00093810E9484EAD7016D937D938D939C93A3
:1042C0001397812F0E9490AD1F5FB4E0EB0EF11C9D
:1042D000ECA9FDA93496FDABECABF4E0CF0ED11CFC
:1042E000143009F09ECF002309F4F6CE0E9414B3D7
:1042F000F3CE0E9494B50C94F32E809117189091F0
:1043000018188537910511F40C94F32E0CF0C0C0E9
:104310008C34910509F43CC40CF058C08A319105E5
:1043200009F42EC224F58531910509F4E7C184F41E
:104330008231910509F4A9C58431910509F49EC122
:10434000419711F00C94A22E0E94BDA40C94F32E60
:104350008731910509F4DCC10CF4D4C18831910591
:1043600009F4ECC1499709F4F4C10C94A22E8F31E1
:10437000910509F401C39CF48C31910509F4A6C29E
:104380000CF40CC28D31910511F40C94F32E4E9760
:1043900011F00C94A22E0E940FB00C94F32E8A32CE
:1043A000910509F49CC32CF4809709F499C20C94EC
:1043B000A22E8133910509F4C6C38B34910511F007
:1043C0000C94A22E0E94BD780C94F32E8A3691058F
:1043D00009F40AC5B4F58435910509F456C5E4F429
:1043E0008135910509F42CC54CF48D34910511F0FB
:1043F0000C94A22E0E94F4780C94F32E8235910531
:1044000009F440C58335910511F00C94A22E81E08A
:1044100080932A040C94F32E8C35910509F47BC506
:1044200034F48535910509F45DC50C94A22E8836C7
:10443000910509F4B1C38936910509F475C40C944A
:10444000A22E8F36910509F4E3C384F48C369105CE
:1044500009F431C40CF4E4C48D36910509F4A6C402
:104460008E36910509F4C1C30C94A22E81379105B3
:1044700009F42DC40CF423C48237910509F4D3C583
:104480008337910511F00C94A22EE3EEF4E008C6F8
:104490008E3221E0920711F40C94DE2C0CF071C0E6
:1044A0008B3C910509F416C7CCF58C38910509F4BD
:1044B00081C4ACF48737910509F49AC60CF44BC655
:1044C0008837910509F497C68937910511F00C9446
:1044D000A22E10923B0510923A050C94F32E8E3BBF
:1044E000910509F47DC434F48B39910509F437C47E
:1044F0000C94A22E883C910509F483C6893C910551
:1045000011F00C94A22EF7E5EF2EF2E0FF2E03E55A
:1045100011E1A3E6CA2EA1E1DA2EC3C68C3D9105B6
:1045200011F40C94712B9CF48D3C910509F463C734
:104530000CF4ECC68E3C910509F4EAC7833D910565
:1045400011F00C94A22E0E9431940C94F32E823E12
:10455000910511F40C94EC2B3CF48D3D910511F474
:104560000C947E2B0C94A22E8C3241E0940711F413
:104570000C94152C8D32914011F40C943E2C0C941B
:10458000A22E853F61E0960711F40C94CB2DDCF54B
:104590008A39A1E09A0709F496C3BCF48033E1E0BC
:1045A0009E0711F40C94352D14F40C94322D83369F
:1045B00021E0920709F45EC08039914011F00C941B
:1045C000A22E0E94186A0C94F32E853A41E09407BB
:1045D00011F40C94C82D4CF4843A914011F00C94D1
:1045E000A22E0E940F960C94F32E8C3A71E097073E
:1045F00009F4B1C7843F914011F00C94A22E0E949F
:104600005F700C94F32E8A39B2E09B0711F40C947E
:104610000A2EB4F4873FF1E09F0711F40C94D12DDA
:1046200014F40C94CE2D883F31E0930711F40C94D0
:10463000DD2D8C30924011F40C94012E0C94A22E9E
:104640008B3853E0950711F40C94F32E3CF4843826
:10465000934011F40C94372E0C94A22E803AA3E0D0
:104660009A0709F47CC1873E934011F40C948F2E75
:104670000C94A22EEDEDFDE10C94B52DEAE2F3E0F1
:1046800084918F010F5F1F4F882321F00E94C689FC
:10469000F801F6CF1092B30C86E69AE00E94369AA3
:1046A0008BE1E6E6FAE0DE01159601900D928A951F
:1046B000E1F78091640A9091650A9C838B838DEE6B
:1046C00092E09A83898340E050E0BE016F5F7F4FA4
:1046D00080E090E00E94E382CE0101960E9492A0C9
:1046E000EBE1F3E084918F010F5F1F4F882311F4FA
:1046F0000C94F32E0E94C689F801F4CF0E94B58075
:104700000C94F32E1092350A1092360A0C94F32E64
:10471000E0911518F09116188081882329F08032D5
:1047200009F410823196F8CF40E061E080911518CD
:10473000909116180E9486D50C94F32E8091360A1B
:10474000882319F081E08093350A0E94BD780C948B
:10475000F32E1092350A80912F07813011F00C94BE
:10476000F32E82E080932F070E94F85860932B0766
:1047700070932C0780932D0790932E070C94F32EA3
:104780008091360A882311F40C94F32E83E50E945D
:10479000914C81110C94FD2E0C94F32E83E40E9415
:1047A000484C882309F450C0E8E6F3E084918F0177
:1047B0000F5F1F4F882321F00E94C689F801F6CFB2
:1047C0008091010C811103C0EBE3F3E012C0BE0144
:1047D0006F5F7F4F8EEF9BE00E94FE988E010F5F10
:1047E0001F4FF80181918F01882349F10E94C689EA
:1047F000F8CF84918F010F5F1F4F882301F10E9432
:10480000C689F801F6CF06EDC02E03E0D02EE12CCC
:10481000F12C20E08091140790E00E2C02C09595B9
:1048200087950A94E2F780FD23C2BFEFEB1AFB0ADB
:10483000E2E0CE0ED11CF5E0EF16F10459F78AE064
:104840000E94C6890C94F32E8091360A882339F091
:104850008091350A882319F0E5E4F3E003C0E7E529
:10486000F3E028C084918F010F5F1F4F882321F050
:104870000E94C689F801F6CF6091AF0C7091B00C20
:104880008091B10C9091B20C4AE00E94E98C8FE2C9
:104890000E94C6896091AB0C7091AC0C8091AD0CFC
:1048A0009091AE0C4AE00E94E98C8AE00E94C68991
:1048B0000C94F32E84918F010F5F1F4F882311F406
:1048C0000C94F32E0E94C689F801F4CF40E060E01A
:1048D00080911518909116180E9486D50C94F32E8D
:1048E0008091350A81110E94186A8091360A8823C6
:1048F00011F40C94F32E80E50E94914C882319F05A
:104900000E94024C03C080E50E94484C182F482F9B
:1049100061E080911518909116180E9486D583E564
:104920000E94914C882381F00E94E14BAB01BC01B5
:104930004093AF0C5093B00C6093B10C7093B20CD9
:104940008EEF9BE00E94EF978091360A882319F042
:1049500081E08093350A11110C94F32EF6CE8091EC
:1049600015189091161821E02093340A40E060E079
:104970000E9486D50C94F32E0E946E787B018C01E8
:1049800020E831E541E050E00E9426EAC9016DE6E9
:1049900071E00E9459ED4B015C01C801B70120E1B3
:1049A0003EE040E050E00E9426EACA01B90128E159
:1049B00030E040E050E00E9426EA762E672EC62EB8
:1049C000D72E8CE3282E312C412C512CC801B70155
:1049D000A20191010E9426EAF62EE72ECA01B90132
:1049E000A20191010E9426EACB018E010F5F1F4FA9
:1049F00081149104D1F0EF92FF927F936F936F92A5
:104A00007F92BF92AF929F928F928FE993E09F9394
:104A10008F931F930F930E940AE60FB6F894DEBFA0
:104A20000FBECDBFE2EFFDE145C0A114B10489F096
:104A3000EF92FF927F936F936F927F92BF92AF92AC
:104A40008FE893E09F938F931F930F930E940AE642
:104A5000E4CFCD2879F0EF92FF927F936F936F921E
:104A60007F9283E893E09F938F931F930F930E940D
:104A70000AE6D3CF892B69F0EF92FF927F936F9371
:104A80008BE793E09F938F931F930F930E940AE607
:104A9000C4CFEF92FF9287E793E09F938F931F938A
:104AA0000F930E940AE60F900F900F900F900F90B7
:104AB0000F90B8CF84917F019FEFE91AF90A8823FC
:104AC00021F00E94C689F701F5CFB80183EB93E08E
:104AD0000E9468C58AE00E94C6890C94F32E83E583
:104AE0000E94914C882311F40C94F32E0E94F14BF8
:104AF000E82E80E50E94914C882339F00E94F14B0A
:104B0000182F87FF03C00C94F32E1DE089E40E9448
:104B1000914C882341F00E94024C81110C94792F12
:104B2000EBE1F6E00BC089E40E94484CF6CF3196E9
:104B3000A6E0EB34FA0711F40C94792F8491181342
:104B4000F6CF0C944E2FF090240481E0F826F092DA
:104B50002404EBECF3E084918F010F5F1F4F882357
:104B600021F00E94C689F801F6CFFF2019F0E0EC91
:104B7000F3E002C0E5ECF3E084918F010F5F1F4F7B
:104B8000882311F40C94F32E0E94C689F801F4CF07
:104B90000E94DF780C94F32E88E690E00E94D0AD5E
:104BA00081110C94F32E8091140783FF02C00C94A2
:104BB000F32E83E50E94914C882399F00E94114CBA
:104BC0000E94C8EBCB010E94ED590E94114C20E0DD
:104BD00030E044EB52E40E9438E6181614F00E94CC
:104BE000F4780E9492C70C94F32E8EE40E94914CAC
:104BF000882311F40C94F32E0E94E14B6093C218A9
:104C00007093C3188093C4189093C5180C94F32E16
:104C100083E50E94484C882359F083E50E94914C1B
:104C2000882319F00E94F14B01C080E080931407A3
:104C3000E2EFFDE184918F010F5F1F4F811103C0EF
:104C4000E4EEF3E004C00E94C689F801F3CF84913A
:104C50008F010F5F1F4F882321F00E94C689F80142
:104C6000F6CF809114078111CECDE0EEF3E018C0AD
:104C7000BB24B394B20E222319F08CE20E94C689A1
:104C8000F60185919491FC0184918F010F5F1F4F74
:104C9000882321F00E94C689F801F6CF2B2DC5CDBF
:104CA00084918F010F5F1F4F882309F4C8CD0E94A4
:104CB000C689F801F5CF109220020C94F32E8BEEEA
:104CC00093E00E94B5A00E94C68E0C94F32E83E55B
:104CD0000E94914C811103C0E2EFFDE10DC00E94E2
:104CE000F14B8D3320F480932B020C94F32E8CE344
:104CF00080932B020C94F32E84918F010F5F1F4F32
:104D0000882321F00E94C689F801F6CF40912B023A
:104D100050E060E070E084EF93E00E9415C58AE007
:104D20000E94C6890C94F32E89E690E00E94D0ADD3
:104D3000811111C0EBEFF3E084918F010F5F1F4FE2
:104D4000882321F00E94C689F801F6CF0E94F675EB
:104D50008AE00E94C689109243100C948E2F83E53E
:104D60000E94914C882311F40C94F32E0E94F14B75
:104D7000182F8D3308F01CE3109350100E94F85840
:104D80006B017C01212F30E0A8EEB3E00E9474EAB1
:104D9000C60ED71EE81EF91EC0924C10D0924D10C0
:104DA000E0924E10F0924F100C94F32E0E9412AE2F
:104DB0000C94F32E8091140783FF02C00C94F32E01
:104DC00083E50E94914C882311F40C94F32E0E94E9
:104DD000114C0E94C8EBCB010E94204E0C94F32E84
:104DE0000E94D6A80C94F32E80E50E94914C81116C
:104DF00006C083E50E94914C882359F005C00E94AB
:104E0000F14B8111F0C7F5CF0E94E14B6F3F710567
:104E100010F06FEF70E07093470460934604E3C7AF
:104E200080E50E94914C811105C0109247041092B8
:104E30004604D9C70E94E14B672B09F0D4C7F5CFD0
:104E40000E9409790E94A4B7109247041092460468
:104E500000E010E062E370E080E090E00E940AB7BA
:104E60000E94C97B0F5F1F4F0331110599F762E361
:104E700070E080E090E00E940AB70E94C97B0E9427
:104E8000A82FB1C710922A04AEC783E50E94914CA7
:104E9000882399F00E94114C20E030E04AE754E466
:104EA0000E949DE60E94CDEB60932C0270932D0230
:104EB00080932E0290932F0296C788E50E94484C5B
:104EC0008111ACC789E50E94484C8111A7C78AE5CA
:104ED0000E94484C8111A2C785E40E94484C811170
:104EE0009DC7CEC783E50E94484C882309F47BC741
:104EF0000E94114C20E030E04AE754E40E949DE615
:104F00000E94CDEB609348107093491080934A1033
:104F100090934B1068C7B7E5CB2EB2E0DB2E16E9B5
:104F2000E12E10E1F12E10E0D6018D916D010E946D
:104F3000484C882309F46DC0133009F063C00E9407
:104F4000114C4B015C0120E030E040EA51E40E944A
:104F500038E687FF4EC0A50194016091A2107091C0
:104F6000A3108091A4109091A5100E9460EB2B01DA
:104F70003C019B01AC016091E3067091E4068091D5
:104F8000E5069091E6060E949DE66093E306709325
:104F9000E4068093E5069093E606A30192016091F2
:104FA00003077091040780910507909106070E94FE
:104FB0009DE6609303077093040780930507909321
:104FC000060760914F11709150118091511190918D
:104FD00052110E943CE6A30192010E949DE60E94AC
:104FE000CDEB60934F1170935011809351119093BA
:104FF00052118092A2109092A310A092A410B0928D
:10500000A51007C00E94114CF70160837183828351
:1050100093831F5FF4E0EF0EF11C143009F084CF8E
:105020000E9433C9E0C60E94186A83E50E94914C31
:10503000882309F451C80E94E14B6230710509F0E0
:105040004BC80E94A4C98BE50E94C6896091A8182C
:105050007091A9188091AA189091AB1842E00E9413
:105060006E8D4091AC185091AD186091AE18709152
:10507000AF1881E094E00E9432C54091B018509181
:10508000B1186091B2187091B3188EEF93E00E943E
:1050900032C58DE50E94C6898AE00E94C689A3C6F2
:1050A00084918F010F5F1F4F882321F00E94C689D2
:1050B000F801F6CF60E083ED94E00E940F9561E087
:1050C0008CEC94E00E940F9561E081EC94E00E94EA
:1050D0000F9561E081EB94E00E940F9560E088EA13
:1050E00094E00E940F9561E08EE994E00E940F9594
:1050F00060E084E994E00E940F9560E08CE894E021
:105100000E940F9561E08EE794E00E940F9560E0A9
:1051100080E794E00E940F9560E081E694E00E94B1
:105120000F9560E083E594E00E940F9560E08DE3C9
:1051300094E00E940F9560E08CE294E00E940F954D
:1051400060E087E194E00E940F9561E084E094E0E4
:105150000E940F9548C6009115181091161883E00B
:10516000D12C40E08150E9F0D8019C91292F2B7F70
:105170002134C1F711962C912133A1F7913421F0FC
:10518000953421F441E002C0DD24D39498012E5FD0
:105190003F4F89012F5F3F4FF80190819032C9F353
:1051A000E1CF442369F0E2EFFDE184917F012FEF2D
:1051B000E21AF20A882321F00E94C689F701F5CF8E
:1051C000DD2069F0E9EAF5E084917F013FEFE31A21
:1051D000F30A882321F00E94C689F701F5CFD80190
:1051E0008D918D01882309F42ACB0E94C689F7CFBF
:1051F0000E9447BEF8C581E080933B0580933A0545
:10520000F2C588EC90E00E94D0AD8111ECC584E439
:105210000E94484C882309F441C00E94114C6B0144
:105220007C0111E020E030E0A9010E9438E6811104
:1052300001C010E010932E1120E030E0A901C70159
:10524000B6010E9438E6882349F10E94114CE09192
:105250005207B4E0EB9FF0011124ED5CFE4E608339
:1052600071838283938320E030E0A9016091331140
:105270007091341180913511909136110E9438E669
:1052800081110CC080E090E0A0EEBFE38093331169
:1052900090933411A0933511B09336110E94E2B768
:1052A000A2C5F70181917F010E94484C882351F0EB
:1052B0000E94114C0E94CDEBD8016D937D938D938C
:1052C0009C9313970C5F1F4FC016D10651F70E9495
:1052D000C2C789C5E7E5EE2EE2E0FE2E07EF16E035
:1052E000F70181917F010E94484C882341F00E9480
:1052F000114CD8016D937D938D939C9313970C5F04
:105300001F4FB7E007301B0759F76DC583E50E94B3
:10531000914C8823A1F00E94114C6093EF0670938A
:10532000F0068093F1069093F2066093EB0670937B
:10533000EC068093ED069093EE0610E001C011E0BC
:1053400080E50E94914C882359F00E94114C609393
:10535000EF067093F0068093F1069093F20610E04A
:1053600082E50E94914C882359F00E94114C609371
:10537000F3067093F4068093F5069093F60610E01A
:1053800084E50E94914C882359F00E94114C60934F
:10539000EB067093EC068093ED069093EE0623C522
:1053A000112309F420C54091EF065091F006609159
:1053B000F1067091F20683EB95E00E9432C54091B0
:1053C000F3065091F4066091F5067091F60680EBB5
:1053D00095E00E9432C54091EB065091EC06609139
:1053E000ED067091EE068DEA95E00E9432C58AE0E6
:1053F0000E94C689F8C481E50E94484C8823C1F008
:105400008091250490912604009739F04AE050E0FD
:1054100060E070E00E94B7E403C060E070E0CB01A0
:1054200060930707709308078093090790930A0712
:1054300083E50E94484C882351F00E94114C6093F0
:105440000F0770931007809311079093120784E55C
:105450000E94484C882351F00E94114C60930B0726
:1054600070930C0780930D0790930E0788E50E94B8
:10547000484C882351F00E94114C6093D7067093DA
:10548000D8068093D9069093DA0689E50E94484CA5
:10549000882351F00E94114C6093DB067093DC0668
:1054A0008093DD069093DE068AE50E94484C8823AF
:1054B000F1F00E94114C6093DF067093E006809338
:1054C000E1069093E2062DEC3CEC4CEC5DE30E948F
:1054D00038E6181664F0E3ECF5E084918F010F5F75
:1054E0001F4F882321F00E94C689F801F6CF85E47A
:1054F0000E94484C882309F476C40E94114C6093A2
:10550000E3067093E4068093E5069093E6066BC489
:1055100067E5C62E62E0D62E7CE3E72E75E0F72E17
:1055200010E0F60181916F010E94484C882359F0E8
:105530000E94114CD7016D937D938D939C9313978B
:10554000812F0E9490AD1F5FB4E0EB0EF11C133071
:1055500041F70C946C200E9463B4811144C407E0AD
:1055600013E2E6E3F4E0FDABECAB9E012F5F3F4FAF
:10557000590150E5852E53E2952E1901F8016591E8
:10558000759185919491ACA9BDA9CD90DD90ED90D8
:10559000FD90BDABACABA70196010E9483EA2B0145
:1055A0003C01F101608371838283938320E030E0CA
:1055B00040EA51EC0E94AAEC87FD0AC020E030E0EE
:1055C00040EA51E4C301B2010E9438E618162CF4F7
:1055D000F401849118160CF456C4D101CD90DD90DD
:1055E000ED90FD901D0120E030E040EA51ECC70154
:1055F000B6010E94AAEC87FD0AC020E030E040EA34
:1056000051E4C701B6010E9438E618164CF5EDEDDD
:10561000FDE184918F010F5F1F4F811103C0E5EF02
:10562000F5E004C00E94C689F801F3CF84918F0190
:105630000F5F1F4F882321F00E94C689F801F6CF23
:1056400088E290E099A388A388EC90E09DA78CA7BE
:10565000BE01605E7F4FCE018C960E9460B5C3C3D1
:105660000C5F1F4FBFEF8B1A9B0AE3E1F3E2E017D9
:10567000F10709F083CF4CE3E42E45E0F42E10E06F
:10568000F50181919191A191B1915F01F701819310
:105690009193A193B1937F01812F0E9490AD1F5FE1
:1056A000133071F70E94459583E992E09DA78CA77E
:1056B00004E610E019A308A3BE01645D7F4FCE018C
:1056C00080960E9460B58AEB92E09DA78CA719A3F3
:1056D00008A3BE01645D7F4FCE0180960E9460B535
:1056E00082C383E50E94914C882309F47CC30E9405
:1056F000E14B709303026093020275C38DED90E05D
:105700000E94D0AD81116FC383E50E94914C81113D
:1057100003C0E2EFFDE13AC00091520710E00E94A1
:10572000E14B000F111FF801E85CFD4F71836083AE
:105730008091520790E07C01EE0CFF1CEE0CFF1CE8
:1057400087010F5D1D4F880F991FFC01E85CFD4F1D
:1057500060817181072E000C880B990B0E943EE638
:105760002AE037ED43E25CE30E949DE6F701E15D4C
:10577000FE4E20813181428153810E949DE6D801F5
:105780006D937D938D939C9313972DC384918F017B
:105790000F5F1F4F882321F00E94C689F801F6CFC2
:1057A00085E40E94C68980915207805D0E94C68967
:1057B000E0915207F0E0EE0FFF1FE85CFD4F6081C3
:1057C000718183E196E00E944FC585E20E94C689FF
:1057D0008AE00E94C68907C380E50E94484C88235E
:1057E00009F401C30E94E14B6B017C0183E50E9437
:1057F000914C882321F00E94E14B8B0102C00FEFF6
:105800001FEFC8010196039708F0EDC2D7FCEBC269
:105810008C2DEBE1F6E09491891709F43FC33196A2
:10582000B6E0EB34FB07B9F73CC383E50E94914C2B
:10583000882319F00E94E14B02C064E071E079A373
:1058400068A380E50E94914C882339F00E94E14BC7
:105850006938E3E17E0730F402C068EE73E07A83D2
:10586000698304C088E893E19A838983BE01605EFE
:105870007F4FCE0101960E9460B5B5C285E40E94BB
:10588000914C811110C080E50E94484C882391F012
:105890000E94114C60934007709341078093420728
:1058A0009093430707C00E94F14B882361F3EDED0D
:1058B000FDE171C089E40E94484C882381F00E9478
:1058C000114C2CEA35EC47E25EE30E949DE66093C2
:1058D0003C0770933D0780933E0790933F0784E415
:1058E0000E94484C882381F00E94114C2CEA35EC30
:1058F00047E25EE30E9460EB6093440770934507C4
:105900008093460790934707E2EFFDE184918F0172
:105910000F5F1F4F882321F00E94C689F801F6CF40
:1059200040914007509141076091420770914307B1
:1059300083E596E00E9432C52CEA35EC47E25EE34F
:1059400060913C0770913D0780913E0790913F0721
:105950000E9460EBAB01BC018FE496E00E9432C56F
:105960002CEA35EC47E25EE360914407709145070D
:1059700080914607909147070E949DE6AB01BC01CC
:105980008BE496E00E9432C58AE00E94C6892BC251
:105990000E94C689F80184918F010F5F1F4F81110A
:1059A000F7CFE7E5F6E084918F010F5F1F4F882363
:1059B00009F419C20E94C689F801F5CF83E50E9457
:1059C000484C182F882371F00E94114C0E94C8EB9C
:1059D000709326026093250221E0672B09F020E0F6
:1059E0002093130780E50E94484C882359F02091AA
:1059F000250230912602232B11F00E94024C809345
:105A00001307F1C11111EFC1E2EFFDE184918F01A4
:105A10000F5F1F4F882321F00E94C689F801F6CF3F
:105A200080911307882319F06BE173E002C06EE1E7
:105A300073E08EE796E00E9468C560912502709140
:105A400026028DE696E00E944FC5E9E6F6E08491D5
:105A50008F010F5F1F4F882309F4C5C10E94C689BB
:105A6000F801F5CF0E94028FBEC180E50E94484C2C
:105A7000882351F00E94114C6093380770933907C6
:105A800080933A0790933B0789E40E94484C88230F
:105A900081F00E94114C2CEA35EC47E25EE30E9453
:105AA0009DE6609334077093350780933607909393
:105AB000370784E40E94484C882381F00E94114CEF
:105AC0002CEA35EC47E25EE30E9460EB609330071E
:105AD000709331078093320790933307E2EFFDE133
:105AE00084918F010F5F1F4F882321F00E94C68988
:105AF000F801F6CF409138075091390760913A0785
:105B000070913B0789E996E00E9432C52CEA35EC9A
:105B100047E25EE360913407709135078091360764
:105B2000909137070E9460EBAB01BC0185E996E0DC
:105B30000E9432C52CEA35EC47E25EE36091300703
:105B40007091310780913207909133070E949DE652
:105B5000AB01BC0181E996E00E9432C58AE00E9457
:105B6000C68941C10E94C689F80184918F010F5FE7
:105B70001F4F8111F7CFEDE9F6E084918F010F5FA0
:105B80001F4F882309F42FC10E94C689F801F5CF61
:105B90000E94DF8D28C10E94537025C10E94EBC274
:105BA00022C183E50E94484C882321F00E94024CC8
:105BB00091E089270E947CBE16C181E080931B077B
:105BC0000E94496A10921B07882309F40CC1E2EF76
:105BD000FDE184918F010F5F1F4F811103C0ECEA3B
:105BE000F6E004C00E94C689F801F3CF84918F01CA
:105BF0000F5F1F4F882309F4F6C00E94C689F80181
:105C0000F5CF8091350A882309F4EDC081E08093B7
:105C1000380AE9C08AE50E94914C811103C0EAEB81
:105C2000F6E00BC00E94114C60933B1170933C1145
:105C300080933D1190933E11D6C084918F010F5FE8
:105C40001F4F882321F00E94C689F801F6CF4091AA
:105C50003B1150913C1160913D1170913E1187EBC9
:105C600096E00E9432C58AE00E94C689BCC08BE4DF
:105C70000E94914C811103C0E2EFFDE136C08BE43C
:105C80000E94914C8823C1F00E94114C6B017C0151
:105C900020E030E0A9010E94AAEC87FD0AC020E0C4
:105CA00030E040E251E4C701B6010E9438E6181620
:105CB00034F4E9EDF6E00EC0C12CD12C76010E943F
:105CC000186AC092E706D092E806E092E906F092E0
:105CD000EA0689C084918F010F5F1F4F882309F462
:105CE00082C00E94C689F801F5CF84918F010F5FB1
:105CF0001F4F882321F00E94C689F801F6CF4091FA
:105D0000E7065091E8066091E9067091EA0688EF8F
:105D100096E00E9432C58AE00E94C68964C081E094
:105D20008093270283E50E94914C882339F00E94DA
:105D3000024C811158C00E9448CE55C083E50E9494
:105D4000484CF7CF0E9494B54EC0F09017180E94AF
:105D5000186A1091801080E00E9426ACFF2029F183
:105D6000E2EFFDE184918F010F5F1F4F882321F047
:105D70000E94C689F801F6CF84E50E94C6896F2D7E
:105D800070E080E090E04AE00E94E98C80E20E94AE
:105D9000C689E5E1F7E084918F010F5F1F4F8823EB
:105DA00011F10E94C689F801F6CF10924210812F9E
:105DB0000E9426ACE2EFFDE184918F010F5F1F4F3F
:105DC000882321F00E94C689F801F6CF6091421025
:105DD00070E083E097E00E944FC58AE00E94C68988
:105DE00002C00E9494B5109243100E942BCE96C020
:105DF0000E94A6AA0E9457CAF6CF0E94E14BAB01AF
:105E0000BC014093AF0C5093B00C6093B10C7093F5
:105E1000B20C8EEF9BE00E94EF97E5CF0E94186ACC
:105E200088E50E94484C882331F05F9A80913504C0
:105E30008E7F8093350489E50E94484C882339F091
:105E40008A9A479A809135048D7F809335048AE53C
:105E50000E94484C882361F08091080180958170F0
:105E600080930601479A809135048B7F8093350497
:105E700085E40E94484C882309F4B5CF129AB3CF29
:105E80000E94A4B7B0CFF7FAF094F7F8F094D101DC
:105E9000CD92DD92ED92FC9213979FCB0E946CE124
:105EA000A2CF0E94186ABC2C60E08C2D0E9407B61D
:105EB0000F3FBFEF1B0759F48C2D0E94B1B531E0A5
:105EC00020E0892B09F030E0032F122F05C00130AC
:105ED000110561F401E010E08B2D0E94B1B580172F
:105EE000910709F480CF0E94FCA0F6CF00E010E0FB
:105EF000F3CF61E0812F0E9407B66E2D812F0E94A3
:105F0000D9B5F12CB701812F0E9443B6193009F0A1
:105F10006ACFF0924704E092460465CFC657DF4F40
:105F20000FB6F894DEBF0FBECDBFDF91CF911F91AA
:105F30000F91FF90EF90DF90CF90BF90AF909F9028
:105F40008F907F906F905F904F903F902F9008952B
:105F50002F923F924F925F926F927F928F929F9279
:105F6000AF92BF92CF92DF92EF92FF920F931F9367
:105F7000CF93DF93CDB7DEB76F970FB6F894DEBF40
:105F80000FBECDBFC0905004D0905104E090520499
:105F9000F090530420E030E040EA50E4C701B6013D
:105FA0000E9438E687FD19C120E030E041E953E462
:105FB000C701B6010E94AAEC18160CF40EC110928B
:105FC000520E1092510E809109014091500E042EF4
:105FD000000C550B817021E0822790E0481759078B
:105FE00009F433C080910901817028272093500E55
:105FF00081111BC00E94B580EDE3FDE084918F010B
:10600000882351F0082E000C990B0E94B0800F5F7E
:106010001F4FF8018491F4CF8DE090E00E94B08092
:106020008AE090E00E94B08010C0E1E4FDE084913D
:106030008F01882389F3082E000C990B0E94B080F1
:106040000F5F1F4FF8018491F4CF8091430E83308E
:1060500009F44CC02CF4882351F08130D9F072C07F
:10606000843009F43EC0853009F44DC06BC0809186
:10607000350A882309F466C081E08093430E0E94AC
:10608000F8586093470E7093480E8093490E909392
:106090004A0E58C08091350A811154C08091010C7C
:1060A000882321F082E08093430E4CC01092430E6F
:1060B000E9E3FDE084918F01882351F0082E000C64
:1060C000990B0E94B0800F5F1F4FF8018491F4CFAD
:1060D0008DE090E00E94B0808AE090E00E94B08065
:1060E00031C08091900E8823E9F22CC08091350A4E
:1060F000811128C08091B7099091B809891B8F70D0
:1061000009F496C01FC08091350A81111BC080918F
:10611000B7099091B809891B8F7009F4ABC012C000
:106120008DE090E00E94B0808AE090E00E94B08014
:106130001092430E89E19DE09093A8078093A707F2
:106140000E94F2898091380E9091390E03974CF598
:1061500073E4272E79E0372EE0E68E2EEAEE9E2EAF
:10616000A12CB12C8EE99FE00E94634B18161906F2
:10617000C4F48091380E9091390E049794F48EE90E
:106180009FE00E94274B80933E0EE0913F0EF091DE
:10619000400E8A3019F08D3009F07DC0309709F03B
:1061A00083C08091380E9091390E009711F40C94B1
:1061B000293F01979093390E8093380E80913A0EC3
:1061C00090913B0E019664E070E00E946DED90931B
:1061D0003B0E80933A0E0C94293F8091510E909182
:1061E000520E8136FAEE9F07E8F01092520E10928E
:1061F000510EE5E4FDE084918F01882351F0082ED3
:10620000000C990B0E94B0800F5F1F4FF801849122
:10621000F4CF8DE090E00E94B0808AE090E00E9490
:10622000B080D1CE01969093520E8093510ECBCE7A
:1062300085E29DE09093A8078093A7070E94F289CA
:106240008091900E882311F082E001C084E0809359
:10625000430EE1E2FDE084918F01882309F438CFF9
:10626000082E000C990B0E94B0800F5F1F4FF801A1
:106270008491F3CFEDE1FDE084918F01882309F44F
:106280004FCF082E000C990B0E94B0800F5F1F4F5C
:10629000F8018491F3CF8A3309F480CFEF35F1050B
:1062A00014F40C94BD3C7ACF80913C0E90913D0E3D
:1062B00020E6289F7001299FF00C112487010854C3
:1062C000134FE00FF11F108261E470E0C8010E94DB
:1062D000D4ED009711F40C94A13C9093420E80935E
:1062E000410E801B910B8E0D9F1D60E070E0875466
:1062F000934F0E9439E20E94C8EBCB01770FAA0BA3
:10630000BB0B8232910510F00C94A13CFC01882754
:10631000EE58FF4F8F4F0C9480EDE4E1FDE0849147
:106320008F01882351F0082E000C990B0E94B08039
:106330000F5F1F4FF8018491F4CF20E030E040E080
:106340005FE36091500470915104809152049091E8
:1063500053041EC0EFE0FDE084918F01882351F0CB
:10636000082E000C990B0E94B0800F5F1F4FF801A0
:106370008491F4CF60914E0470914F04072E000C6D
:10638000880B990B0E943EE620E030E040E05FE39E
:106390000E9484EA0E94C8EBCB010E94EA4D0E9451
:1063A000BCD78DE090E00E94B0808AE090E00E942F
:1063B000B0800C94A13CEAE0FDE084918F01882339
:1063C00051F0082E000C990B0E94B0800F5F1F4FF8
:1063D000F8018491F4CF20E030E040E05FE3609189
:1063E0004A0470914B0480914C0490914D04D0CF9D
:1063F000E5E0FDE084918F01882351F0082E000C28
:10640000990B0E94B0800F5F1F4FF8018491F4CF69
:106410006091480470914904B1CF209146043091B5
:10642000470444E6429FC001439F900D11246FEF43
:1064300070E00E946DED8B016536710510F004E689
:1064400010E0E0E0FDE084917F01882359F0082E00
:10645000000C990B0E94B080FFEFEF1AFF0AF701C2
:106460008491F3CFB80180E090E036C7ECEFFCE018
:1064700084918F01882351F0082E000C990B0E9403
:10648000B0800F5F1F4FF8018491F4CF80E290E05D
:106490000E94B080E8EFFCE084918F01882351F0E6
:1064A000082E000C990B0E94B0800F5F1F4FF8015F
:1064B0008491F4CF60913604709137048091380450
:1064C000909139040E94BDD780E290E00E94B08094
:1064D000E4EFFCE084918F01882351F0082E000C3A
:1064E000990B0E94B0800F5F1F4FF8018491F4CF89
:1064F00060913A0470913B0480913C0490913D047A
:106500000E94BDD780E290E00E94B080E0EFFCE006
:1065100084918F01882351F0082E000C990B0E9462
:10652000B0800F5F1F4FF8018491F4CF60913E045B
:1065300070913F0480914004909141040E94BDD726
:1065400080E290E0A0C58091350A882309F450C00C
:10655000EBEEFCE084918F01882351F0082E000CB3
:10656000990B0E94B0800F5F1F4FF8018491F4CF08
:106570008091360A882359F18091010C882329F1F2
:106580008091AB0C9091AC0CA091AD0CB091AE0C85
:106590000097A105B105C1F0BC01CD016D597F4F38
:1065A0008F4F9F4F24E630E040E050E00E9426EA03
:1065B0006091AF0C7091B00C8091B10C9091B20CC5
:1065C0000E9426EA822F01C080E090E0E6CEE7EE4E
:1065D000FCE084918F01882309F4E3CE082E000C9F
:1065E000990B0E94B0800F5F1F4FF8018491F3CF89
:1065F000EFEDFCE084918F01882309F4D2CE082EC0
:10660000000C990B0E94B0800F5F1F4FF80184911E
:10661000F3CFEAEDFCE084918F01882351F0082E3E
:10662000000C990B0E94B0800F5F1F4FF8018491FE
:10663000F4CF8091470E9091480EA091490EB091F1
:106640004A0E892B8A2B8B2B09F477C00E94F858AD
:10665000A50194010E9426EA69017A016091470E22
:106660007091480E8091490E90914A0EA5019401B7
:106670000E9426EA8601021B130BC8016CE370E03E
:106680000E9459EDCB019927EAE0F0E0BF010E949A
:106690006DED282FCB01BF010E946DED805D8093D1
:1066A0002D04205D20932E0410922F048DE294E09F
:1066B0000E94BCD780E290E00E94B080E8EDFCE050
:1066C00084917F01882359F0082E000C990B0E94B9
:1066D000B080FFEFEF1AFF0AF7018491F3CF80E259
:1066E00090E00E94B080C8016CE370E00E9459ED18
:1066F0006AE070E00E946DED605D60932D04805D46
:1067000080932E0410922F048DE294E00E94BCD757
:1067100080E290E00E94B080E6EDFCE084918F0181
:10672000882309F43ECE082E000C990B0E94B080FD
:106730000F5F1F4FF8018491F3CF80E290E00E9439
:10674000B080EEECFCE084918F01882309F429CE1F
:10675000082E000C990B0E94B0800F5F1F4FF801AC
:106760008491F3CF1092710E8091090180FF11C0C6
:10677000EAECFCE084918F01882309F412CE082E04
:10678000000C990B0E94B0800F5F1F4FF80184919D
:10679000F3CF83E50E9458D7882341F00E9473D736
:1067A0000E94CDEB7093460E6093450EE6ECFCE044
:1067B00084918F01882351F0082E000C990B0E94C0
:1067C000B0800F5F1F4FF8018491F4CF8DE090E00F
:1067D0000E94B0808AE090E00E94B08080918F0E8D
:1067E000882309F442C28091450E9091460E843070
:1067F000910509F4C8C08830910509F47DC1892B41
:1068000009F0E7C3EAEEFAE084918F01882351F0A2
:10681000082E000C990B0E94B0800F5F1F4FF801EB
:106820008491F4CF8DE090E00E94B0808AE090E007
:106830000E94B080EFEDFAE084918F01882351F03F
:10684000082E000C990B0E94B0800F5F1F4FF801BB
:106850008491F4CF8DE090E00E94B0808AE090E0D7
:106860000E94B080E3EDFAE084918F01882351F01B
:10687000082E000C990B0E94B0800F5F1F4FF8018B
:106880008491F4CF8DE090E00E94B0808AE090E0A7
:106890000E94B080E7ECFAE084918F01882351F0E8
:1068A000082E000C990B0E94B0800F5F1F4FF8015B
:1068B0008491F4CF8DE090E00E94B0808AE090E077
:1068C0000E94B080E9EBFAE084918F01882351F0B7
:1068D000082E000C990B0E94B0800F5F1F4FF8012B
:1068E0008491F4CF8DE090E00E94B0808AE090E047
:1068F0000E94B080EBEAFAE084918F01882351F086
:10690000082E000C990B0E94B0800F5F1F4FF801FA
:106910008491F4CF8DE090E00E94B0808AE090E016
:106920000E94B080EEE9FAE084918F01882351F053
:10693000082E000C990B0E94B0800F5F1F4FF801CA
:106940008491F4CF8DE090E00E94B0808AE090E0E6
:106950000E94B080E1E9FAE084918F01882351F030
:10696000082E000C990B0E94B0800F5F1F4FF8019A
:106970008491F4CF8DE090E00E94B0808AE090E0B6
:106980000E94B08026C3E3E8FAE084918F01882357
:1069900051F0082E000C990B0E94B0800F5F1F4F22
:1069A000F8018491F4CF8DE090E00E94B0808AE0FD
:1069B00090E00E94B080E5E7FAE084918F0188239F
:1069C00051F0082E000C990B0E94B0800F5F1F4FF2
:1069D000F8018491F4CF8DE090E00E94B0808AE0CD
:1069E00090E00E94B080EFE5FAE084918F01882367
:1069F00051F0082E000C990B0E94B0800F5F1F4FC2
:106A0000F8018491F4CF8DE090E00E94B0808AE09C
:106A100090E00E94B080E9E4FAE084918F0188233D
:106A200051F0082E000C990B0E94B0800F5F1F4F91
:106A3000F8018491F4CF8DE090E00E94B0808AE06C
:106A400090E00E94B080E7E3FAE084918F01882310
:106A500051F0082E000C990B0E94B0800F5F1F4F61
:106A6000F8018491F4CF8DE090E00E94B0808AE03C
:106A700090E00E94B080E5E2FAE084918F018823E3
:106A800051F0082E000C990B0E94B0800F5F1F4F31
:106A9000F8018491F4CF8DE090E00E94B0808AE00C
:106AA00090E00E94B080E7E1FAE084918F018823B2
:106AB00051F0082E000C990B0E94B0800F5F1F4F01
:106AC000F8018491F4CF8DE090E00E94B0808AE0DC
:106AD00090E00E94B080E9E0FAE084918F01882381
:106AE00009F448CF082E000C990B0E94B0800F5F6C
:106AF0001F4FF8018491F3CFE2E0FAE084918F0117
:106B0000882351F0082E000C990B0E94B0800F5F73
:106B10001F4FF8018491F4CF8DE090E00E94B08087
:106B20008AE090E00E94B080EBEFF9E084918F0161
:106B3000882351F0082E000C990B0E94B0800F5F43
:106B40001F4FF8018491F4CF8DE090E00E94B08057
:106B50008AE090E00E94B080E4EEF9E084918F0139
:106B6000882351F0082E000C990B0E94B0800F5F13
:106B70001F4FF8018491F4CF8DE090E00E94B08027
:106B80008AE090E00E94B080EDECF9E084918F0102
:106B9000882351F0082E000C990B0E94B0800F5FE3
:106BA0001F4FF8018491F4CF8DE090E00E94B080F7
:106BB0008AE090E00E94B080E6EBF9E084918F01DA
:106BC000882351F0082E000C990B0E94B0800F5FB3
:106BD0001F4FF8018491F4CF8DE090E00E94B080C7
:106BE0008AE090E00E94B080EFE9F9E084918F01A3
:106BF000882351F0082E000C990B0E94B0800F5F83
:106C00001F4FF8018491F4CF8DE090E00E94B08096
:106C10008AE090E00E94B080ECE8F9E084918F0176
:106C2000882351F0082E000C990B0E94B0800F5F52
:106C30001F4FF8018491F4CF8DE090E00E94B08066
:106C40008AE090E00E94B080E9E7F9E084918F014A
:106C5000882309F48FCE082E000C990B0E94B08077
:106C60000F5F1F4FF8018491F3CF8091360A88237C
:106C700009F486C181E08093B30C1092B50C109298
:106C8000B40C85E89AE00E94369A8BE1E5E8FAE0D8
:106C9000DE01159601900D928A95E1F78091830AA5
:106CA0009091840A9C838B838DEE92E09A838983F2
:106CB00040E050E0BE016F5F7F4F80E090E00E94B7
:106CC000E382CE0101960E9492A0C090B40CD090B5
:106CD000B50C0091450E1091460EC601801B910B1C
:106CE000049720F06801F3E0CF0ED11C5AE6452E40
:106CF00059E0552E6BE5662E69E0762EC016D1065A
:106D000008F467C10115110509F0A1C069E37AE033
:106D100085E89AE00E94FE9862E273E089E39AE0D7
:106D20000E94DFED892B09F04AC0F20184914AE606
:106D3000E42E49E0F42E882359F0082E000C990B1C
:106D40000E94B080FFEFEF1AFF0AF7018491F3CFA2
:106D50008DE090E00E94B0808AE090E00E94B080D8
:106D6000F30184913BE5E32E39E0F32E882359F0BB
:106D7000082E000C990B0E94B080FFEFEF1AFF0A5B
:106D8000F7018491F3CF8DE090E00E94B0808AE01B
:106D900090E00E94B0804AE060E070E0CB010E9489
:106DA000E98CEBE4F9E084917F012FEFE21AF20A1B
:106DB000882309F4E2C00E94C689F701F4CFE7E412
:106DC000F9E084917F01882359F0082E000C990B7B
:106DD0000E94B080FFEFEF1AFF0AF7018491F3CF12
:106DE0008DE090E00E94B0808AE090E00E94B08048
:106DF000F101849123E4E22E29E0F22E882359F058
:106E0000082E000C990B0E94B080FFEFEF1AFF0ACA
:106E1000F7018491F3CF8DE090E00E94B0808AE08A
:106E200090E00E94B0804AE060E070E0CB010E94F8
:106E3000E98CEEE3F9E084917F012FEFE21AF20A88
:106E4000882309F49AC00E94C689F701F4CF60E054
:106E500070E0C80101970E94A1848091370A8823BD
:106E600009F45FC0ECE3F9E084917F01882359F0D5
:106E7000082E000C990B0E94B080FFEFEF1AFF0A5A
:106E8000F7018491F3CF89E39AE00E94BCD78DE0AB
:106E900090E00E94B0808AE090E00E94B080EAE337
:106EA000F9E084917F01882359F0082E000C990B9A
:106EB0000E94B080FFEFEF1AFF0AF7018491F3CF31
:106EC00086E49AE00E94BCD78DE090E00E94B080FA
:106ED0008AE090E00E94B080C801A0E0B0E04AE003
:106EE000BC01CD010E94E98CE8E3F9E084917F01C7
:106EF0002FEFE21AF20A882321F00E94C689F701D7
:106F0000F5CF96E4E92E9AE0F92EF70181917F0101
:106F1000882319F00E94C689F8CF8AE00E94C689AA
:106F20002CC089E39AE00E94BCD78DE090E00E94DB
:106F3000B0808AE090E00E94B08086E49AE00E94EF
:106F4000BCD78DE090E00E94B0808AE090E00E9483
:106F5000B080C801A0E0B0E04AE0BC01CD010E94D1
:106F6000E98C86E4E82E8AE0F82EF70181917F0112
:106F7000882399F20E94C689F8CF0F5F1F4FBECEBB
:106F8000E9E2F9E084918F01882351F0082E000C8A
:106F9000990B0E94B0800F5F1F4FF8018491F4CFCE
:106FA0008DE090E00E94B0808AE090E00E94B08086
:106FB000EAE1F9E084918F01882309F4DBCC082E03
:106FC000000C990B0E94B0800F5F1F4FF801849155
:106FD000F3CFE2ECFCE084918F01882309F4E1C94E
:106FE000082E000C990B0E94B0800F5F1F4FF80114
:106FF0008491F3CF8091350A882339F00E9415825D
:10700000A0C48091350A8823E9F00E940BB199C48D
:107010008091430E823019F0833609F092C40E94A9
:10702000F581EEEBFCE084918F01882309F4B9C966
:10703000082E000C990B0E94B0800F5F1F4FF801C3
:107040008491F3CF8091430E833609F07AC4DDCF6B
:1070500085EB9CE00E94B5A08091B7099091B8099A
:10706000891B8F7009F06DC48091430E823009F442
:1070700068C4833609F099C464C48DE090E00E942E
:10708000B0808AE090E00E94B0808BC98091B709FF
:107090009091B809891B8F7009F053C48091430EF9
:1070A000823009F44EC4833609F44BC48091010C3C
:1070B0008111CFC446C483E50E9458D7811126C0F0
:1070C00083E40E9458D7882309F43BC48091B70910
:1070D0009091B809891B8F7009F033C420E030E02B
:1070E00040E251E460913E0470913F04809140047D
:1070F000909141040E9438E687FF08C082EA9CE034
:107100009093A8078093A7070E94F2890E9473D7E3
:1071100020E030E0A9010E9438E687FD10C00E94FF
:1071200073D720E030E849E853E40E94AAEC18162F
:107130004CF00E9473D70E94CDEBCB0105C080E0DC
:1071400090E002C083E191E00E94ED59FAC383E52B
:107150000E9458D7882309F4F4C30E9473D720E013
:1071600030E0A9010E9438E687FD10C00E9473D765
:1071700020E030E046E153E40E94AAEC18164CF0FF
:107180000E9473D70E94CDEBCB0105C080E090E058
:1071900002C086E990E00E94204ED3C383E50E949E
:1071A00058D78823D9F00E9473D720E030E04FE70A
:1071B00053E40E949DE620E030E048EC52E40E9457
:1071C00060EB0E94CDEB6F3F710519F010F06FEF8F
:1071D00070E07093470460934604E3C88FEF90E03B
:1071E0009093470480934604DCC88091B70990913E
:1071F000B809891B8F7009F0D4C88091350A8111B4
:10720000D0C80E94C68E5F9A809135048E7F80938D
:1072100035048A9A479A809135048D7F809335048E
:10722000809108018095817080930601479A809132
:1072300035048B7F80933504129AB3C883E50E948E
:1072400058D7882319F10E9473D720E030E040E23C
:1072500052E40E9438E687FD0FC00E9473D720E0F9
:1072600030EC49E754E40E94AAEC181644F00E945E
:1072700073D70E94C8EB05C068E270E002C067EEF9
:1072800073E070930302609302025BC3ECE9FCE0DD
:1072900084918F01882351F0082E000C990B0E94D5
:1072A000B0800F5F1F4FF8018491F4CFC0900202AD
:1072B000D09003020D2C000CEE08FF08F7FE0EC064
:1072C0006DE28EE99FE00E94DA4A66277727CB01BC
:1072D0006C197D098E099F094AE003C04AE0C70185
:1072E000B6010E947CD75DC88091B7099091B8091A
:1072F000891B8F7009F025C38091430E823009F4F9
:1073000020C3833609F0EBC21CC38091B70990916A
:10731000B809891B8F7009F044C88091430E8230F0
:1073200009F43FC8833609F0B6C33BC88091B7095A
:107330009091B809891B8F7009F003C38091430EA7
:10734000823009F4FEC2833609F0FBC4FAC2809190
:10735000B7099091B809891B8F7009F0F2C280912A
:10736000430E823009F4EDC2833609F020C5E9C22C
:107370008091B7099091B809891B8F7009F0E1C21B
:107380008091430E823009F4DCC2833609F045C592
:10739000D8C28091710E811103C00E94B580C4C112
:1073A0008E3271F58091720E8E3209F046C1809155
:1073B000D60B882309F4B8C181508093D60B88235B
:1073C00061F090E001974FE1489F9001499F300D97
:1073D0001124C9018056954F02C082E69AE02BE144
:1073E000FC013496A5E8BAE001900D922A95E1F7E8
:1073F000FC01828193819093840A8093830A94C1D3
:107400008C3309F01AC164E273E081E79EE00E94C8
:10741000DFED892B21F481E080938F0E85C163E33A
:1074200073E081E79EE00E94DFED892B79F4E6EFBF
:10743000F8E084918F010F5F1F4F882321F00E9495
:10744000C689F801F6CF89ED98E0E4C06AE473E0FC
:1074500081E79EE00E94DFED892B79F4E5EBF8E00F
:1074600084918F010F5F1F4F882321F00E94C689EE
:10747000F801F6CF82EA98E0CDC061E673E081E7DB
:107480009EE00E94DFED892B79F4E7E8F8E0849133
:107490008F010F5F1F4F882321F00E94C689F801DA
:1074A000F6CF82E898E0B6C06FE673E081E79EE031
:1074B0000E94DFED892B79F4E2E6F8E084918F01F8
:1074C0000F5F1F4F882321F00E94C689F801F6CF75
:1074D0008DE598E09FC062E873E081E79EE00E943E
:1074E000DFED892B79F4E2E4F8E084918F010F5FFE
:1074F0001F4F882321F00E94C689F801F6CF89E347
:1075000098E088C060E973E081E79EE00E94DFEDCB
:10751000892B71F406E118E0F8018491882329F0A1
:107520000F5F1F4F0E94C689F7CF8FE098E072C0AF
:1075300066EA73E081E79EE00E94DFED892B79F433
:10754000E0EFF7E084918F010F5F1F4F882321F058
:107550000E94C689F801F6CF89EE97E05BC068EB20
:1075600073E081E79EE00E94DFED892B79F4E1ED85
:10757000F7E084918F010F5F1F4F882321F00E9455
:10758000C689F801F6CF80EC97E044C063EC73E065
:1075900081E79EE00E94DFED892B79F4E7EAF7E0CE
:1075A00084918F010F5F1F4F882321F00E94C689AD
:1075B000F801F6CF85E997E02DC06FEC73E081E725
:1075C0009EE00E94DFED892B79F4EAE7F7E08491F1
:1075D0008F010F5F1F4F882321F00E94C689F80199
:1075E000F6CF88E697E016C06DED73E081E79EE088
:1075F0000E94DFED892BA9F4EEE4F7E084918F017E
:107600000F5F1F4F882321F00E94C689F801F6CF33
:107610008DE397E09093A8078093A7070E94F289D3
:1076200083C06AEE73E081E79EE00E94DFED892B64
:1076300009F07AC010928F0E77C01D8218861C82C6
:107640001B828DEE92E09A8389838091880A811152
:1076500003C062E67AE002C061E87AE06115710574
:1076600019F06C5F7F4F02C060E070E021E041E7FD
:107670005EE0CE0105960E94659E882361F18BE154
:10768000FE013596A5E8BAE001900D928A95E1F7E2
:107690002B813C813093840A2093830A8091D60BFE
:1076A0008A3008F03DC091E0980F9093D60BFFE12F
:1076B0008F9FC0011124DC01AC55B54F4BE1E5E8CB
:1076C000FAE001900D924A95E1F7FC01E056F54F82
:1076D0003383228325C0E2EFFDE184918F010F5FA8
:1076E0001F4F882321F00E94C689F801F6CFE7E2F8
:1076F000F7E084918F010F5F1F4F882321F00E94D4
:10770000C689F801F6CF01E71EE0F80181918F01EB
:10771000882319F00E94C689F8CF8AE00E94C689A2
:10772000CE0101960E9492A01092710E80910901E3
:1077300080FF07C1E0EEFBE084918F01882311F404
:107740000C94D131082E000C990B0E94B0800F5F71
:107750001F4FF8018491F2CF8FE40E9458D7811116
:107760000C94D13183E40E9458D70C94D13183E535
:107770000E9458D7811159C08FE40E9458D788239E
:1077800019F088EA9BE007C084E50E9458D7882357
:1077900049F080E89BE09093A8078093A7070E9498
:1077A000F28943C083E40E9458D7882319F087E503
:1077B0009BE0F1CF81E50E9458D7882319F08FE232
:1077C0009BE0E9CF88E40E9458D78823C9F0EBE218
:1077D000FBE084918F01882351F0082E000C990B57
:1077E0000E94B0800F5F1F4FF8018491F4CF8DE0AD
:1077F00090E00E94B0808AE090E00E94B08015C0C6
:107800008CE40E9458D7882381F0E7E2FBE0849162
:107810008F01882361F3082E000C990B0E94B08021
:107820000F5F1F4FF8018491F4CFEFEEFBE08491DE
:107830008F01882311F40C94D131082E000C990B80
:107840000E94B0800F5F1F4FF8018491F2CF8091AA
:10785000B7098091B8090C94D13183E50E9458D7BB
:10786000882309F46EC08FEF9AE09093A807809365
:10787000A7070E94F289EFEEFBE084918F01882335
:1078800011F40C94D131082E000C990B0E94B08099
:107890000F5F1F4FF8018491F2CFEAEFFAE0849175
:1078A0008F01882351F0082E000C990B0E94B080A4
:1078B0000F5F1F4FF8018491F4CFE5EFFAE0849158
:1078C0008F01882311F40C94D131082E000C990BF0
:1078D0000E94B0800F5F1F4FF8018491F2CF88E5BE
:1078E0000E9458D7811106C089E50E9458D7882385
:1078F00009F4C3C088E50E9458D7882341F086E97F
:107900009CE09093A8078093A7070E94F28989E5DD
:107910000E9458D7882341F080E99CE09093A80703
:107920008093A7070E94F2898AE50E9458D788238E
:1079300041F08AE89CE09093A8078093A7070E94F3
:10794000F28980913C0E90913D0E019664E070E0CA
:107950000E946DED90933D0E80933C0E8091380E09
:107960009091390E01969093390E8093380E1092B3
:10797000400E10923F0E0C94B23040913C0E50914C
:107980003D0E9F012F5F3F4F3093400E20933F0EDF
:1079900090E6949F9001959F300D11242854334F09
:1079A000E20FF31F80830C94B2300091410E1091CE
:1079B000420E780124E0E20EF11C6AE270E0C70199
:1079C0000E94D4EDF80124812F3221F4B8016B5FBD
:1079D0007F4F03C02C3339F4B70181E79EE00E944A
:1079E000E8ED0C94D1311092710E009719F0FC0162
:1079F000319710828091410E9091420E40E061E0FB
:107A000004960E9486D58091010C882389F0E1EBD1
:107A1000FCE084918F01882309F42FCB082E000C01
:107A2000990B0E94B0800F5F1F4FF8018491F3CF34
:107A3000EDEAFCE084918F01882309F41ECB082E27
:107A4000000C990B0E94B0800F5F1F4FF8018491CA
:107A5000F3CF0E94F581E9EAFCE084918F0188234D
:107A600011F40C94D131082E000C990B0E94B080B7
:107A70000F5F1F4FF8018491F2CF8AE50E9458D71B
:107A8000811138CF83E40E9458D7882309F459CF55
:107A900086E89CE050CF86E40E9458D7882309F4FA
:107AA0004DC10E9473D70E94CDEB8B0182E89CE010
:107AB0009093A8078093A7070E94F28988E50E9407
:107AC00058D7882309F451C00E9473D72B013C0179
:107AD0002DEC3CEC4CE45EE30E9438E69E012F5F07
:107AE0003F4F7901181674F020E030E0A901C3017E
:107AF000B2010E94AAEC18162CF41F930F9387E78B
:107B00009CE005C12DEC3CEC4CEC5DEBC301B201FB
:107B10000E9438E618167CF020E030E040E85FEB89
:107B2000C301B2010E94AAEC18162CF41F930F9304
:107B30008BE69CE0ECC01F930F93C301B2010E943F
:107B4000C8EB7F936F9381E69CE09F938F93FF92A6
:107B5000EF920E940AE60FB6F894DEBF0FBECDBFCB
:107B6000CE0101960E94CD89DFC089E50E9458D7D9
:107B7000882309F441C00E9473D72B013C012DECEE
:107B80003CEC4CE45EE30E9438E6FE0131967F0156
:107B9000181674F020E030E0A901C301B2010E9480
:107BA000AAEC18162CF41F930F9386E59CE0AFC047
:107BB0002DEC3CEC4CEC5DEBC301B2010E9438E6CD
:107BC00018167CF020E030E040E85FEBC301B20122
:107BD0000E94AAEC18162CF41F930F938AE49CE0E1
:107BE00096C01F930F93C301B2010E94C8EB7F930D
:107BF0006F9380E49CE0A9CF8AE50E9458D7882340
:107C000009F441C00E9473D72B013C012DEC3CECE0
:107C10004CE45EE30E9438E6FE0131967F011816BF
:107C200074F020E030E0A901C301B2010E94AAEC87
:107C300018162CF41F930F9385E39CE068C02DEC7D
:107C40003CEC4CEC5DEBC301B2010E9438E6181627
:107C50007CF020E030E040E85FEBC301B2010E941D
:107C6000AAEC18162CF41F930F9389E29CE04FC0E6
:107C70001F930F93C301B2010E94C8EB7F936F93D0
:107C80008FE19CE062CF85E40E9458D7882309F4F5
:107C90004BC00E9473D72B013C012DEC3CEC4CE413
:107CA0005EE30E9438E6FE0131967F01181674F0FB
:107CB00020E030E0A901C301B2010E94AAEC18162D
:107CC0002CF41F930F9384E19CE021C02DEC3CEC3D
:107CD0004CEC5DEBC301B2010E9438E618167CF053
:107CE00020E030E040E85FEBC301B2010E94AAEC63
:107CF00018162CF41F930F9388E09CE008C0C30172
:107D0000B2010E94C8EB7F936F938DEF9BE09F932E
:107D10008F93FF92EF920E940AE60F900F900F90C0
:107D20000F900F900F901CCF89EF9BE09093A807C6
:107D30008093A7070E94F2890C94D13100E010E0F3
:107D4000B5CE20E030E040E251E460913E04709115
:107D50003F0480914004909141040E9438E687FFDF
:107D600008C082EF9BE09093A8078093A7070E942A
:107D7000F28982E390E090934904809348040E9442
:107D8000B07688EC90E00E94ED59EFEEFBE0849134
:107D90008F01882311F40C94D131082E000C990B1B
:107DA0000E94B0800F5F1F4FF8018491F2CF20E056
:107DB00030E040E251E460913E0470913F048091D4
:107DC0004004909141040E9438E687FF08C088EE85
:107DD0009BE09093A8078093A7070E94F28980E513
:107DE00090E090934904809348040E94B07680EF1D
:107DF00090E00E94ED59EFEEFBE084918F01882323
:107E000011F40C94D131082E000C990B0E94B08013
:107E10000F5F1F4FF8018491F2CF80E090E00E9445
:107E2000ED5910924904109248040E94B076E4EE95
:107E3000FBE084918F01882311F40C94D131082E3A
:107E4000000C990B0E94B0800F5F1F4FF8018491C6
:107E5000F2CF6F960FB6F894DEBF0FBECDBFDF91A5
:107E6000CF911F910F91FF90EF90DF90CF90BF9037
:107E7000AF909F908F907F906F905F904F903F90CA
:107E80002F9008952F923F924F925F926F927F9220
:107E90008F929F92AF92BF92CF92DF92EF92FF921A
:107EA0000F931F93CF93DF93CDB7DEB762970FB6D3
:107EB000F894DEBF0FBECDBFF8948FEF9FEF909385
:107EC0008900809388002AE02A8B212C312C789419
:107ED0008091A6049091A704A091A804B091A90450
:107EE000892B8A2B8B2B09F00FC280911E078823C8
:107EF000E1F010921E0780911C0790911D07892BBD
:107F000009F402C210925E0410921D0710921C0721
:107F10009091B7098091B809981709F4F5C180913B
:107F2000B8098F5F8F708093B80980911C0790917A
:107F30001D07892B09F4E8C14091A2045091A304C4
:107F40006091A4047091A50480919E0490919F0477
:107F5000A091A004B091A1040091950410E020E04C
:107F600030E0841B950BA60BB70B081719072A07DF
:107F70003B0710F4D901C801E82F840F951FA61FF5
:107F8000B71F8093A2049093A304A093A404B0937A
:107F9000A5042091840030918500245E3F4F4091DC
:107FA0007A0450917B0460917C0470917D048091EF
:107FB0006A0490916B04A0916C04B0916D04840FDD
:107FC000951FA61FB71F80937A0490937B04A093FC
:107FD0007C04B0937D04B7FD1CC0889A8091861004
:107FE00090918710A0918810B0918910409104025F
:107FF000042E000C550B660B770B840F951FA61FE4
:10800000B71F8093861090938710A0938810B09329
:10801000891040917E0450917F046091800470919A
:10802000810480916E0490916F04A0917004B091CE
:108030007104840F951FA61FB71F80937E04909331
:108040007F04A0938004B0938104B7FD1CC08E9A76
:1080500080918A1090918B10A0918C10B0918D100E
:1080600040910502042E000C550B660B770B840F14
:10807000951FA61FB71F80938A1090938B10A09313
:108080008C10B0938D1040918204509183046091C4
:108090008404709185048091720490917304A0917E
:1080A0007404B0917504840F951FA61FB71F8093A9
:1080B000820490938304A0938404B0938504B7FD55
:1080C0003FC080915804F09106028823C9F0809146
:1080D000560482FF02C0F7FD06C080915504882334
:1080E00011F40C94EC48809156049091570493FF3E
:1080F00002C0F7FD0CC080915404811108C006C075
:1081000080910B018095887080930901419A40917C
:108110008E1050918F1060919010709191108F2F50
:10812000FF0F990BAA0BBB0B840F951FA61FB71F40
:1081300080938E1090938F10A0939010B093911015
:10814000409186045091870460918804709189045D
:108150008091760490917704A0917804B09179048D
:10816000840F951FA61FB71F8093860490938704E2
:10817000A0938804B0938904B7FD3AC0409192104F
:10818000509193106091941070919510C0900702D7
:108190000C2C000CDD08EE08FF084C0D5D1D6E1D5B
:1081A0007F1D40939210509393106093941070939E
:1081B0009510409166045091670460916804709135
:1081C0006904841B950BA60BB70B809386049093D0
:1081D0008704A0938804B0938904909159048091F6
:1081E000930493FF02C0815001C08F5F809393047A
:1081F00080917A0490917B04A0917C04B0917D04DD
:10820000B7FD15C040916604509167046091680401
:1082100070916904841B950BA60BB70B80937A04AD
:1082200090937B04A0937C04B0937D048898809104
:108230007E0490917F04A0918004B0918104B7FDE9
:1082400015C0409166045091670460916804709174
:108250006904841B950BA60BB70B80937E04909347
:108260007F04A0938004B09381048E98809182044F
:1082700090918304A0918404B0918504B7FD3AC025
:10828000409166045091670460916804709169049C
:10829000841B950BA60BB70B8093820490938304E9
:1082A000A0938404B0938504809158048823E1F05E
:1082B0008091560482FF04C08091060287FD05C0AC
:1082C00080915504882309F48FC7809156049091BA
:1082D000570493FF04C08091060287FD0BC0809174
:1082E0005404811107C005C080910B0188708093F0
:1082F00009014198E15041F08091840090918500FE
:1083000082179307C8F34BCE80911102909112020D
:10831000A0911302B0911402892B8A2B8B2B09F0A8
:108320008AC080919404882309F453C08090A204E9
:108330009090A304A090A404B090A504C0908F04D2
:10834000D0909004E0909104F090920440919304B6
:10835000C814D904EA04FB0480F480915F0490916E
:10836000600420916304309164042817390728F4CD
:10837000415040939304019714C08C149D04AE04A3
:10838000BF04E0F480915F04909160042091610447
:10839000309162048217930788F44F5F40939304EF
:1083A00001969093600480935F0440910D02509178
:1083B0000E0260910F02709110020EC08FEF9FEFBE
:1083C000DC0180930D0290930E02A0930F02B093F4
:1083D00010024FEF5FEFBA018091930487FD02C056
:1083E000169801C0169A80918400909185004C9651
:1083F000209193042223B9F0149A2091930427FF2B
:1084000002C02F5F01C02150209393041498209143
:108410009304222369F3209184003091850028176A
:108420003907C8F3E5CF40931102509312026093CD
:108430001302709314028091A6049091A704A09156
:10844000A804B091A904892B8A2B8B2B09F049C66B
:10845000A0911C07B0911D07109711F40C94964A37
:108460008090A2049090A304A090A404B090A504CE
:1084700040919E0450919F046091A0047091A104CA
:1084800084169506A606B706D8F010925E041092E0
:108490001D0710921C079091B7098091B809981791
:1084A00011F40C94964A8091B8098F5F8F70809375
:1084B000B80940EDC42E47E0D42EE12CF12C1AC4AB
:1084C00040919A0450919B0460919C0470919D048A
:1084D000481559056A057B0508F4AAC14091960420
:1084E000509197046091980470919904D6960D91DB
:1084F0001D912D913C91D997401751076207730741
:1085000008F077C1411551056105710549F4809066
:108510005A0490905B04A0905C04B0905D0464C128
:10852000E12CF980842E952F862F0A811B81FD81F5
:10853000EE813F8128859C80E091F317E89D912C86
:10854000FF273091F417389D900CF11D1090F5170E
:10855000189CF00DE99F900CF11D399FF00DE89FDC
:10856000F00D092D1F2F099DE12D332722270F9F85
:10857000E00D311D2E1D199DE00D311D2E1D1F9F7B
:10858000300D211D032F122F099DF12C3327222797
:108590000F9FF00C311D2E1D199DF00C311D2E1D4D
:1085A0001F9F300D211D032F122FEE2780905A049C
:1085B00090915B0480915C040090B6040E2809F44D
:1085C00083C03091B204309FE1198E089E098E0954
:1085D0002091B304209FE01981089E098E09F09034
:1085E000B404F09E801891098E09319FE01981082A
:1085F0009E098E09219F801891098E09F19E90197C
:108600008109099DF12C332722270F9FF00C311D82
:108610002E1D199DF00C311D2E1D1F9F300D211D8B
:10862000032F122F3091AE04309FE10D8E1C9E1D42
:108630008E1D2091AF04209FE00D811C9E1D8E1D7C
:10864000F090B004F09E800C911D8E1D319FE00DC6
:10865000811C9E1D8E1D219F800C911D8E1DF19EE3
:10866000900D811D099DF12C332722270F9FF00CBF
:10867000311D2E1D199DF00C311D2E1D1F9F300D1B
:10868000211D032F122F3091AA04309FE1198E086B
:108690009E098E092091AB04209FE01981089E0954
:1086A0008E09F090AC04F09E801891098E09319FDC
:1086B000E01981089E098E09219F801891098E0971
:1086C000F19E9019810982C03091B204309FE10D72
:1086D0008E1C9E1D8E1D2091B304209FE00D811CD9
:1086E0009E1D8E1DF090B404F09E800C911D8E1D79
:1086F000319FE00D811C9E1D8E1D219F800C911DC0
:108700008E1DF19E900D811D099DF12C332722278E
:108710000F9FF00C311D2E1D199DF00C311D2E1DCB
:108720001F9F300D211D032F122F3091AE04309F5B
:10873000E1198E089E098E092091AF04209FE0194F
:1087400081089E098E09F090B004F09E801891096E
:108750008E09319FE01981089E098E09219F80189A
:1087600091098E09F19E90198109099DF12C3327F9
:1087700022270F9FF00C311D2E1D199DF00C311D6D
:108780002E1D1F9F300D211D032F122F3091AA0483
:10879000309FE10D8E1C9E1D8E1D2091AB04209FED
:1087A000E00D811C9E1D8E1DF090AC04F09E800C8F
:1087B000911D8E1D319FE00D811C9E1D8E1D219FE0
:1087C000800C911D8E1DF19E900D811D11249C82A7
:1087D000F9820A831B83FD83EE833F832887912CD4
:1087E000992AA12CB12CA82A89E495E121E0298BB2
:1087F00014C0D2968D909D90AD90BC90D597F4CF3B
:10880000B694A79497948794D988DD0CD98A049656
:1088100025E18536920709F4EDC4FC010591159117
:1088200025913491081519052A053B0548F3E2C442
:1088300040908F0450909004609091047090920446
:10884000481459046A047B0408F0C3C180918E0463
:10885000811121C0FD01EE5BFF4FE080F1800281BC
:10886000138178962081318142815381D2966D9116
:108870007D918D919C91D5970E9461C4DD24D39404
:10888000D0928E04E0911C07F0911D0782A993A954
:10889000A4A9B5A98EC140918A0450918B0460911E
:1088A0008C0470918D04DA960D911D912D913C915F
:1088B000DD97401751076207730708F073C1411530
:1088C00051056105710549F480915A0490915B044A
:1088D000A0915C04B0915D046CC1F0E0E985842F47
:1088E000352F262FAA857B856C855D85BE854F85B6
:1088F0009889B091F317B89F612D55274091F417CF
:10890000489F600D511D1090F517189E500DB39F94
:10891000600D511D439F500DB29F500DA62F752F16
:10892000A69FB12D44279927A59FB00D411D9F1FDC
:10893000769FB00D411D9F1F759F400D911DA42F67
:10894000792FA69FE12D44279927A59FE00D411D72
:108950009F1F769FE00D411D9F1F759F400D911D2C
:10896000A42F792FBB2780915A0430915B0420916A
:108970005C040090B6040F2A09F483C04091B2044D
:108980004A9FB1198F0B3F0B2F0B9091B3049A9F05
:10899000B01981093F0B2F0BE091B404EA9F8019B5
:1089A00031092F0B479FB01981093F0B2F0B979F60
:1089B000801931092F0BE79F30192109A69FE12D5E
:1089C00044279927A59FE00D411D9F1F769FE00D2D
:1089D000411D9F1F759F400D911DA42F792F409120
:1089E000AE044A9FB10D8F1F3F1F2F1F9091AF0400
:1089F0009A9FB00D811D3F1F2F1FE091B004EA9F89
:108A0000800D311D2F1F479FB00D811D3F1F2F1F50
:108A1000979F800D311D2F1FE79F300D211DA69FB1
:108A2000E12D44279927A59FE00D411D9F1F769FAB
:108A3000E00D411D9F1F759F400D911DA42F792FA3
:108A40004091AA044A9FB1198F0B3F0B2F0B9091B5
:108A5000AB049A9FB01981093F0B2F0BE091AC0436
:108A6000EA9F801931092F0B479FB01981093F0BED
:108A70002F0B979F801931092F0BE79F3019210980
:108A800082C04091B2044A9FB10D8F1F3F1F2F1F1C
:108A90009091B3049A9FB00D811D3F1F2F1FE0914D
:108AA000B404EA9F800D311D2F1F479FB00D811D1B
:108AB0003F1F2F1F979F800D311D2F1FE79F300DE8
:108AC000211DA69FE12D44279927A59FE00D411D5B
:108AD0009F1F769FE00D411D9F1F759F400D911DAB
:108AE000A42F792F4091AE044A9FB1198F0B3F0BF1
:108AF0002F0B9091AF049A9FB01981093F0B2F0B58
:108B0000E091B004EA9F801931092F0B479FB019FB
:108B100081093F0B2F0B979F801931092F0BE79F7E
:108B200030192109A69FE12D44279927A59FE00D23
:108B3000411D9F1F769FE00D411D9F1F759F400D9A
:108B4000911DA42F792F4091AA044A9FB10D8F1F28
:108B50003F1F2F1F9091AB049A9FB00D811D3F1FA7
:108B60002F1FE091AC04EA9F800D311D2F1F479FFE
:108B7000B00D811D3F1F2F1F979F800D311D2F1F8F
:108B8000E79F300D211D1124E987AA877B876C8719
:108B90005D87BE874F87988B90E0932BA0E0B0E075
:108BA000A22B07C0A65ABF4F8D919D910D90BC91ED
:108BB000A02D29E435E141E0498BF901459155911A
:108BC00065917491481759076A077B0708F49CC39D
:108BD000AAC3809193048823E1F0FD01E85BFF4F75
:108BE0004081518160E070E000910D0210910E0211
:108BF00020910F023091100240175107620773074E
:108C000041F010921102109212021092130210926F
:108C100014024091090250910A0260910B02709176
:108C20000C0277FF5FC0AE5ABF4FCD90DD90ED9044
:108C3000FC9089E495E121E0FC0145915591659115
:108C400074914C155D056E057F0550F4F694E7941C
:108C5000D794C794220F049675E18536970761F77C
:108C60002093950480E2C816D104E104F10428F4AD
:108C700070E2C72ED12CE12CF12C90E2C91AD10858
:108C8000E108F108C114A8E0DA06E104F10408F4EF
:108C900006C4B4E0DB9EC0011124875B9E4EFC013C
:108CA000329625913491EC2D6627E39FA001E29F37
:108CB000410D561F0694461F561F112460E070E0B8
:108CC000FC0125913491C901A0E0B0E0841B950B13
:108CD000A60BB70B8093090290930A02A0930B0294
:108CE000B0930C02C0900902D0900A02E0900B02EF
:108CF000F0900C0280911C0790911D07892B09F0C0
:108D0000E8C10E94E0C490931D0780931C07892B43
:108D100009F4DFC1E0911C07F0911D07808183FFFA
:108D20003EC085899689A789B08D809386109093DF
:108D30008710A0938810B0938910818D928DA38D98
:108D4000B48D80938A1090938B10A0938C10B09365
:108D50008D10858D968DA78DB0A180938E109093E8
:108D60008F10A0939010B093911081A192A1A3A114
:108D7000B4A18093921090939310A0939410B09309
:108D800095109091B7098091B809981709F4B9CF57
:108D90008091B8098F5F8F708093B809B2CFC58872
:108DA000D688E788F08C81E0C114D104E104F10495
:108DB00009F480E0018D128D238D348D011511058C
:108DC0002105310509F08260458D568D678D70A1B2
:108DD000411551056105710509F0846080935E04B9
:108DE00010928A0410928B0410928C0410928D04BD
:108DF000109296041092970410929804109299047D
:108E000085A196A1A7A1B0A580939E0490939F04ED
:108E1000A093A004B093A104882499245401881A33
:108E2000990AAA0ABB0A8092860490928704A092AB
:108E30008804B09289048092820490928304A09264
:108E40008404B092850480927E0490927F04A09264
:108E50008004B092810480927A0490927B04A09264
:108E60007C04B0927D04CC0CDD1CEE1CFF1CC09277
:108E70006A04D0926B04E0926C04F0926D04000FCF
:108E8000111F221F331F00936E0410936F04209351
:108E9000700430937104440F551F661F771F409371
:108EA000720450937304609374047093750441A129
:108EB00052A163A174A1440F551F661F771F4093F1
:108EC0007604509377046093780470937904880F44
:108ED000991FAA1FBB1F8093660490936704A093F9
:108EE0006804B09369041092A2041092A304109233
:108EF000A4041092A50482A593A5A4A5B5A580936A
:108F00009A0490939B04A0939C04B0939D0486A51F
:108F100097A5A0A9B1A980938F0490939004A093E2
:108F20009104B093920481A580936504DF01A95B4D
:108F3000BF4F9C9190939404992339F115962D91EC
:108F40003C911197309364042093630412972D9100
:108F50003C911197309362042093610410921102A6
:108F600010921202109213021092140212972D9175
:108F70003C91A90160E070E040930D0250930E0215
:108F800060930F02709310020CC088248A94982C6E
:108F9000540180920D0290920E02A0920F02B092A4
:108FA0001002EA5BFF4F90812091590492130AC08E
:108FB0002091080230E0482F082E000C550B421774
:108FC000530731F090935904809308020E94B3C470
:108FD00080913B0581110E94BFBD2FEF3FEFA9019A
:108FE0002093090230930A0240930B0250930C0223
:108FF000E0911C07F0911D07DF01DE96ED90FD90DA
:109000000D911C9122A933A944A955A9EA5AFF4FF1
:1090100060817181828193810E9461C410928E046B
:10902000E0911C07F0911D07EA5AFF4F8080918064
:10903000A280B38089E495E121E0FC01459155913E
:1090400065917491481559056A057B0558F4B694E5
:10905000A79497948794220F0496A5E6B5E1A817E4
:10906000B90759F720939504B0E28B169104A10437
:10907000B10428F4B0E28B2E912CA12CB12C30E25B
:10908000831A9108A108B108811448E09406A1044C
:10909000B10408F428C254E0959EC0011124875BF6
:1090A0009E4EFC01329625913491782D6627739F50
:1090B000A001729F410D561F0694461F561F112492
:1090C000FC01C590D490E12CF12CC41AD50AE1081A
:1090D000F108C092A604D092A704E092A804F092EE
:1090E000A9040091A6041091A7042091A80430912E
:1090F000A9044091110250911202609113027091E3
:109100001402F02E198BF22FE32F4017510762073C
:10911000730720F4F42E598BF62FE72F8F2D9989A2
:10912000AF2FBE2F0097E1E0AE07B10520F08FEF23
:109130009FEFA0E0B0E0081B190B2A0B3B0B00933C
:10914000A6041093A7042093A8043093A9044F3FCA
:10915000FFEF5F076F077F0761F0481B590B6A0B32
:109160007B0B409311025093120260931302709391
:109170001402F8942091840030918500205F3F4FC5
:109180004A8941504A8B442341F0280E391E221649
:10919000330610F40C94673F01C019013092890026
:1091A00020928800789462960FB6F894DEBF0FBEC6
:1091B000CDBFDF91CF911F910F91FF90EF90DF9086
:1091C000CF90BF90AF909F908F907F906F905F9067
:1091D0004F903F902F90089580910B01809588705B
:1091E000809309010C94734080910B0188708093E7
:1091F00009016BC839893093950480E2881691047F
:10920000A104B10428F430E2832E912CA12CB12CBE
:1092100030E2831A9108A108B108811488E0980609
:10922000A104B10420F1E4E09E9EC0011124875BFB
:109230009E4EFC01329625913491F82DEE27F39F36
:109240007001F29FE10CFE1E0694EE1EFE1E11241C
:10925000FC01C590D490860120E030E0480159011E
:109260008E189F08A108B1087501640122C09501FC
:1092700084013695279517950795F801EC7FCF0166
:10928000875B924FFC01C590D490FC0132962591EA
:109290003491E82DE770E29FC001E39F900D112407
:1092A00023E0969587952A95E1F7C81AD90AE12C0B
:1092B000F12C4C0D5D1D6E1D7F1D40939604509347
:1092C000970460939804709399049091940480910A
:1092D0009304992309F474C0882309F40BCDA85B87
:1092E000BF4F8D919C91A0E0B0E040910D02509154
:1092F0000E0260910F027091100284179507A60765
:10930000B70709F060C0F6CCB695A79597958795F5
:10931000D988DD0CD98A2C5F3F4F45E655E14217CD
:10932000530709F04ACC598950939504803291052E
:10933000A105B10520F480E290E0A0E0B0E08097C4
:10934000A109B109811558E09507A105B10508F4F7
:1093500043C074E0979F90011124275B3E4EF901B2
:10936000329645915491EE27859FB001849F610DFF
:109370007E1F06946E1F7E1F1124F901C590D490A4
:10938000E12CF12CC61AD70AE108F10880918A0471
:1093900090918B04A0918C04B0918D048C0D9D1D37
:1093A000AE1DBF1D80938A0490938B04A0938C0400
:1093B000B0938D0480919404811130C08091930406
:1093C000882309F497CC1092110210921202109285
:1093D0001302109214028ECCAC01BD0176956795F4
:1093E00057954795FA01EC7F9F01275B324FF901B2
:1093F000C590D490F9013296459154918770849F1D
:109400009001859F300D1124F3E036952795FA954C
:10941000E1F7C21AD30AE12CF12CB8CF8989480EA2
:10942000511C611C711C80911C0790911D074814F0
:1094300059046A047B04D8F420919304222309F48C
:1094400059CCFC01E85BFF4F20813181A90160E02C
:1094500070E000910D0210910E0220910F023091E8
:109460001002401751076207730709F443CC1092AA
:109470001102109212021092130210921402FC01B7
:10948000E85BFF4F80819181A0E0B0E080930D0206
:1094900090930E02A0930F02B09310022BCCD70131
:1094A000C601B695A79597958795FC01EC7FCF01EE
:1094B000875B924FFC0125913491FC0132964591D6
:1094C00054916C2D6770649FC001659F900D1124AD
:1094D00063E0969587956A95E1F7281B390BC901DA
:1094E000A0E0B0E0F7CBD501C401B695A79597955C
:1094F0008795FC01EC7FCF01875B924FFC01C59003
:10950000D490FC01329625913491482D4770429FAA
:10951000C001439F900D1124A3E096958795AA95CD
:10952000E1F7C81AD90AE12CF12CD3CD80EDC82E71
:1095300087E0D82EE12CF12CE4CBCF92DF92EF9292
:10954000FF92CF93DF936B017C01EA0121E338E0C6
:1095500040EA50EC0E94AAEC87FD23C022E430E0F0
:109560004CE553E4C701B6010E9438E61816CCF06A
:10957000C880D980EA80FB802FE632E143E85AEBCD
:10958000C701B6010E94AAEC87FD0BC0C1E022E42E
:1095900030E04CE553E4C701B6010E9438E61816E6
:1095A0000CF4C0E08C2FDF91CF91FF90EF90DF9013
:1095B000CF9008950F931F93CF93DF93FC01A6855F
:1095C000B7858D0100581F4FE80188819981019668
:1095D0008F779927AD014E575F4FEA012881398176
:1095E00028173907D1F3E80128813981A20FB31F69
:1095F0006C93A685B785A058BF4F11969C938E9308
:10960000A689B7892C9181E090E0078C02C0880F71
:10961000991F0A94E2F7822B8C9381E081A304883E
:10962000F589E02D80818064808381E090E0DF9186
:10963000CF911F910F910895FC0181A1882329F0FA
:10964000A489B5898C9186FFFBCF11A20895FC01F6
:10965000A485B585FD01E058FF4F20813181329608
:10966000808191812817390779F080819181A80F35
:10967000B91F8C91208131812F5F3F4F2F77332786
:109680003183208390E008958FEF9FEF0895DC01F0
:109690001C96ED91FC911D97DF01A058BF4F2D91B5
:1096A0003C91119712968D919C911197281739072B
:1096B00039F08D919C91E80FF91F808190E0089519
:1096C0008FEF9FEF0895FC0124853585F901E0585F
:1096D000FF4F8081918132962081318180589F4F48
:1096E000821B930B60E870E00C946DED0895089573
:1096F00080E090E00895CF92DF92EF92FF92C090C9
:109700003002D0903102E0903202F0903302FC013E
:1097100080819181A281B381809330029093310244
:10972000A0933202B09333020E9457CAC092300213
:10973000D0923102E0923202F0923302FF90EF9029
:10974000DF90CF90089580919A1890919B18981768
:1097500059F0E92FF0E0E65EF74E80819F5F9F773A
:1097600090939B1890E008958FEF9FEF08951F92BC
:109770000F920FB60F9211240BB60F922F938F9367
:109780009F93EF93FF9320919B18E0919A1881E0AB
:109790008E0F8F779091C600281729F0F0E0E65ED3
:1097A000F74E9083E82FE0939A18FF91EF919F91E5
:1097B0008F912F910F900BBE0F900FBE0F901F90A7
:1097C00018958091250490912604009731F04AE085
:1097D00050E060E070E00C948CE360E070E0CB015E
:1097E0000895EFDF97FD0AC0ECDF6F3F710581053B
:1097F000910509F02CF4E5DF862F089580E00895A7
:109800008FEF08958091250490912604892B31F0E3
:10981000E8DF91E0811103C090E001C091E0892F61
:1098200008950F931F93CF93809125049091260460
:10983000009711F1FC018F01C1912C2F2F7DA9F010
:10984000C53411F0C536B9F7F801108260E070E058
:1098500080912504909126040E9439E2F801C0838A
:10986000562F472F382F292F0BC060E070E0CF9183
:109870001F910F910C9439E250E040E030E020E07D
:10988000652F742F832F922FCF911F910F910895E1
:1098900081548A3108F042C0E82FF0E0409111185D
:1098A00050911218609113187091141804C0769595
:1098B0006795579547958A95D2F7842F817040FF19
:1098C0002FC0E950F84E9081992309F1E09176106C
:1098D000F0917710E90FF11D908120ED290F2A30CA
:1098E00098F09E3211F491810CC09D3211F09B32A0
:1098F00071F4918120ED290F2A3030F09E3239F435
:10990000928190539A3018F42E2F9F2F02C020E09E
:1099100090E02093250490932604089580E0089514
:109920000895B6DF882341F081E02091250430912D
:109930002604232B09F480E0089580E1E6E3F4E0B7
:10994000A2EBB0E101900D928A95E1F708952F9274
:109950003F924F925F926F927F928F929F92AF92BF
:10996000BF92CF92DF92EF92FF920F931F93CF930C
:10997000DF9300D01F921F92CDB7DEB77C018B0121
:109980006A0119018090360490903704A090380441
:10999000B0903904A5019401FC016081718182813C
:1099A00093810E9438E6F1E0FD83811112C020917D
:1099B0003A0430913B0440913C0450913D04F8013D
:1099C00060817181828193810E9438E6811101C09A
:1099D0001D82F601408051806280738020911502C3
:1099E000309116024091170250911802C301B20142
:1099F0000E9438E6882309F453C040921502509221
:109A00001602609217027092180220E030E040E4E3
:109A100050E46091FF0670910007809101079091DA
:109A200002070E9460EB69837A838B839C83809218
:109A3000B2109092B310A092B410B092B510809171
:109A40003A0490913B04A0913C04B0913D04809372
:109A5000B6109093B710A093B810B093B910F60158
:109A600080819181A281B3818093BA109093BB10C1
:109A7000A093BC10B093BD10809142049091430418
:109A8000A0914404B09145048093BE109093BF1000
:109A9000A093C010B093C110CE0101962CDE4DDF13
:109AA000FD81FF2309F16090FB067090FC06809019
:109AB000FD069090FE06A090F706B090F806C090C4
:109AC000F906D090FA069501A601B301C4010E94DF
:109AD000AAEC181614F05301640120E030E040E2D3
:109AE00051E4B501C6010CC020E030E040EC5FE37A
:109AF0006091030770910407809105079091060714
:109B00000E9460EB69837A838B839C832091240479
:109B1000222349F0AB01BC0189E695E10E9432C5E0
:109B20008AE00E94C689F70180819181A281B38178
:109B30008093B2109093B310A093B410B093B5106B
:109B4000F80180819181A281B3818093B6109093B6
:109B5000B710A093B810B093B910F10120813181F2
:109B6000428153816091BE107091BF108091C010EE
:109B70009091C1100E9484EA6093BE107093BF1050
:109B80008093C0109093C110CE010196B4DDD5DE54
:109B90000F900F900F900F900F90DF91CF911F912A
:109BA0000F91FF90EF90DF90CF90BF90AF909F907C
:109BB0008F907F906F905F904F903F902F9008957F
:109BC00080E1E2EBF0E1A6E3B4E001900D928A952A
:109BD000E1F708959C0197FD0EC08436910584F04D
:109BE00064E670E00E946DEDCB016AE070E00E94D7
:109BF0006DED805D06C03195219531098DE201C082
:109C000080E2809331042A30310564F0EAE0F0E02C
:109C1000C901BF010E946DEDCB01BF010E946DED36
:109C2000805D01C080E280933204C9016AE070E087
:109C30000E946DED805D8093330481E394E008958C
:109C40008E3691051CF02EE680E002C0282F892F69
:109C500020934804809349040C94B0762F923F924D
:109C60004F925F926F927F928F929F92AF92BF922C
:109C7000CF92DF92EF92FF920F931F93CF93DF93D8
:109C8000CDB7DEB7C455D1090FB6F894DEBF0FBE0D
:109C9000CDBFE8E2F8E184918F010F5F1F4F882369
:109CA00021F00E94C689F801F6CF0E9463B48111A9
:109CB0000C94105880E090E0A0E8BFE38093AA10D5
:109CC0009093AB10A093AC10B093AD1080E090E0F7
:109CD000A0ECB0E48093AE109093AF10A093B010BE
:109CE000B093B1108DEC9CECACE4BEE38093A61075
:109CF0009093A710A093A810B093A91080E090E0D3
:109D0000A8ECB1E48093280590932905A0932A0537
:109D1000B0932B058CE390E0909327058093260564
:109D200088EC90E0909325058093240510922305FC
:109D30008FE4F7DD882311F074DD04C060E070E08B
:109D400080E190E46BAF7CAF8DAF9EAF83E4E9DD43
:109D5000882311F057DD02C083E49ADD61968FAF4E
:109D600061978BE4DEDD882311F04CDD02C08BE4CB
:109D70008FDD60968FAF609782E4D3DD8823E9F0B2
:109D800050DD0E94C8EB709327056093260561158E
:109D9000710599F0685271096536710570F0E3EF4D
:109DA000F7E184918F010F5F1F4F882311F40C940A
:109DB00010580E94C689F801F4CF8CE4B2DD8823E4
:109DC00051F12FDD6B017C016093A6107093A710F9
:109DD0008093A8109093A91020E030E0A9010E9480
:109DE000AAEC87FD0AC020E030E040E050E4C70163
:109DF000B6010E9438E6181674F4EBECF7E1849192
:109E00008F010F5F1F4F882311F40C9410580E948C
:109E1000C689F801F4CF81E53BDD882309F440C011
:109E20008091250490912604892B19F4E0EAF7E14A
:109E30002BC0F7DC6B017C016093AE107093AF1008
:109E40008093B0109093B1102DEC3CEC4CE45DE3AA
:109E50000E94AAEC87FD0AC020E030E040E751E410
:109E6000C701B6010E9438E61816D4F4EFE6F7E110
:109E700084918F010F5F1F4F882311F40C941058A9
:109E80000E94C689F801F4CF84918F010F5F1F4FA4
:109E9000882311F40C9410580E94C689F801F4CF5D
:109EA00083E53FDD882319F1BCDC4B015C012DEC1F
:109EB0003CEC4CEC5DE30E94AAEC87FD0AC020E07C
:109EC00030E040E85FE3C501B4010E9438E61816AF
:109ED000ACF4E8E4F7E184918F010F5F1F4F882312
:109EE00011F40C9410580E94C689F801F4CF5DEC6F
:109EF000852E5CEC952EA92C5EE3B52E80E5C8DCA2
:109F0000882309F443C08091250490912604892B6D
:109F100071F4E0E1F7E184918F010F5F1F4F882317
:109F200011F40C9410580E94C689F801F4CF809166
:109F300023058F5F8093230574DC6B017C016093A4
:109F400028057093290580932A0590932B0520E01E
:109F500030E0A9010E94AAEC87FD0AC020E030E0B1
:109F600048EC51E4C701B6010E9438E6181674F4B3
:109F7000E8EEF6E184918F010F5F1F4F882311F403
:109F80000C9410580E94C689F801F4CF86E4C9DC0D
:109F9000882319F146DC6B017C0120E030E040E8C9
:109FA0005FE30E94AAEC87FD0AC020E030E040E8B1
:109FB00050E4C701B6010E9438E61816A4F4EFEB8E
:109FC000F6E184918F010F5F1F4F882311F40C94E9
:109FD00010580E94C689F801F4CFC12CD12C40EE54
:109FE000E42E4FE3F42EA7019601C701B6010E94AB
:109FF0009DE69B01AC0160E070E084E490E40E9487
:10A0000060EB2091AA103091AB104091AC105091B0
:10A01000AD100E949DE62B013C01A5019401C501F4
:10A02000B4010E949DE6A70196010E949DE62CEED8
:10A0300031E548EB5DE30E9460EB9B01AC01C3019D
:10A04000B2010E949DE66093AA107093AB108093BA
:10A05000AC109093AD1088E464DC8823C9F0E1DB98
:10A060000E94C8EB7093250560932405655A710919
:10A070006437710568F0E1E9F6E184918F010F5FC3
:10A080001F4F882309F4CCC70E94C689F801F5CF79
:10A0900085E5FEDB8823E9F00E94F858611571051B
:10A0A0008105910511F00E9430E280912504909184
:10A0B0002604892B11F0B5DB04C060E070E088E471
:10A0C00092E460931F05709320058093210590937F
:10A0D000220582E5DDDB81110DC0EDE5F6E184911D
:10A0E0008F010F5F1F4F882309F49AC70E94C6890A
:10A0F000F801F5CF8091250490912604892BA9F0D1
:10A1000060DB2F967FAF6EAF2F97161617069CF069
:10A11000E9E2F6E184918F010F5F1F4F882309F474
:10A120007FC70E94C689F801F5CF8AE190E02F969B
:10A130009FAF8EAF2F9788E5F4DB882361F071DB4A
:10A14000209118043091190440911A0450911B0475
:10A150000E9483EA08C060913604709137048091B0
:10A1600038049091390460931B0570931C0580930B
:10A170001D0590931E0589E5D4DB882361F051DB32
:10A1800020911C0430911D0440911E0450911F0425
:10A190000E9483EA08C060913A0470913B04809168
:10A1A0003C0490913D0460931705709318058093CB
:10A1B000190590931A0560911B0570911C058091FB
:10A1C0001D0590911E0547E155E0B7D981110DC0DD
:10A1D000EFEFF5E184918F010F5F1F4F882309F4A2
:10A1E0001FC70E94C689F801F5CF84E451DB91E0D6
:10A1F00089270E9426AC20E030E040EA50E46091DC
:10A200003E0470913F0480914004909141040E946B
:10A2100038E687FF14C0198A1A8A1B8A1C8A80E0D4
:10A2200090E0A0EAB0E489839A83AB83BC83BE014B
:10A230006F5E7F4FCE0101960E9445B4C1DCD8D736
:10A240006B017C01A8E8CA0EA3E1DA1EE11CF11C37
:10A250008091260590912705F3DC60912605709189
:10A260002705072E000C880B990B0E943EE69B01E8
:10A27000AC0160914A0470914B0480914C04909120
:10A280004D040E9483EA4B015C0120E030E0A9010B
:10A290000E94AAEC87FF04C0B7FAB094B7F8B09454
:10A2A00020E030E040E450E4C501B4010E94AAEC93
:10A2B0001816F4F49DD7DC01CB018C199D09AE0969
:10A2C000BF09B7FD0EC094D76B017C01B8E8CB0E77
:10A2D000B3E1DB1EE11CF11C0E94F6758AE00E94CE
:10A2E000C6890E94FCA080919A1880939B18B5CFD4
:10A2F00080912405909125050E94ED5960912405D7
:10A3000070912505072E000C880B990B0E943EE6E4
:10A310009B01AC01609150047091510480915204F2
:10A32000909153040E9483EA4B015C0120E030E0ED
:10A33000A9010E94AAEC87FF04C0B7FAB094B7F84D
:10A34000B09420E030E040E450E4C501B4010E9444
:10A35000AAEC1816F4F44CD7DC01CB018C199D093A
:10A36000AE09BF09B7FD0EC043D76B017C01E8E819
:10A37000CE0EE3E1DE1EE11CF11C0E94F6758AE0C0
:10A380000E94C6890E94FCA080919A1880939B1815
:10A39000B5CF1092420410924304109244041092DC
:10A3A00045040E9414B380912305882399F1C5DAEE
:10A3B000209128053091290540912A0550912B05BF
:10A3C0006091BE107091BF108091C0109091C1102B
:10A3D0000E9484EA6093BE107093BF108093C010F7
:10A3E0009093C11020E030E040E751E46091030712
:10A3F0007091040780910507909106070E9460EB19
:10A4000069837A838B839C83CE01019674D995DA14
:10A410000E9421B180E2E7EFF4E0DF01282F1D92D6
:10A420002A95E9F7E7EDF4E0DF01282F1D922A9540
:10A43000E9F7E7EBF4E0DF011D928A95E9F77DDAB1
:10A440008091A6109091A710A091A810B091A9108A
:10A450008093BA109093BB10A093BC10B093BD1022
:10A4600019821A821B821C829E012F5F3F4F4AEB8A
:10A4700050E166EB70E182EB90E169DA9E01255CC8
:10A480003F4F4AEB50E166EB70E182EB90E15FDA1F
:10A490006196BFAD6197BB2329F06AE374E086E360
:10A4A00094E004C067E175E08BE195E00E9488D8F4
:10A4B000298F3A8F4B8F5C8F6D8F7E8F3FAF2D969C
:10A4C0002FAF2D972D96EFAD2D97E7FD81C4FFADF2
:10A4D000F7FD7EC424E0E202F0011124EF5FF54FA6
:10A4E00040805180628073803FAD84E03802F0018B
:10A4F0001124E351F64FD080C180328023808D2D0E
:10A500009C2DA32DB22D8FAB98AFA9AFBAAFAE01E2
:10A51000495C5F4FB201C30110D8882309F45CC4C1
:10A5200020E030E040EA50E4B201C3010E9484EA36
:10A53000F62E072F182FE92E862F902FA12FBE2D34
:10A540008BAB9CABADABBEAB8D2D9C2DA32DB22D9B
:10A550008FA798ABA9ABBAAB2D969FAD2D97911154
:10A5600052C0AFADA11105C05F2D402F312F2E2D50
:10A5700004C0542D452D362D272D852F942FA32F24
:10A58000B22F8BAB9CABADABBEABBFADB43034F434
:10A59000F42C052D162DE72CBB2369F020E030E0CC
:10A5A00040EA50E46D2D7C2D832D922D0E9483EA8C
:10A5B000362F272F03C09601832D922D432F522F24
:10A5C000BC014FA758AB69AB7AABEFADE4300CF0F0
:10A5D000A7C020E030E040EA50E46D2D7C2D832DB3
:10A5E000922D0E9484EA21966FAF219723967FAF28
:10A5F000239725968FAF259727969FAF2797FFAD77
:10A60000F11185C099C02D962FAD2D9724300CF4F3
:10A6100053C03FAD34305CF020E030E040EA50E41D
:10A62000B201C3010E9483EA362F272F03C0342DC5
:10A63000252DC301432F522FBC014BAB5CAB6DAB3F
:10A640007EAB8FAD8111E3C420E030E040EA50E4FE
:10A65000B201C3010E9483EAF62E072F182FE92EBC
:10A6600020E030E040EA50E46D2D7C2D832D922DCA
:10A670000E9484EA6FA778AB89AB9AAB9FAD992310
:10A6800009F44EC020E030E040EA50E46D2D7C2D0E
:10A69000832D922D0E9483EA21966FAF21972396F6
:10A6A0007FAF239725968FAF259727969FAF279744
:10A6B000AFADA43064F140C0BFADB1110DC020E01A
:10A6C00030E040EA50E4B201C3010E9483EAF62E72
:10A6D000072F182FE92E0FC0EFADE430B4F120E0C2
:10A6E00030E040EA50E4B201C3010E9483EA6BAB60
:10A6F0007CAB8DAB9EAB2196DFAE21972396CFAE80
:10A70000239725963FAE259727962FAE279732EDB4
:10A71000832E33E5932E3BE7A32E31E4B32E29C0DD
:10A720002196DFAE21972396CFAE239725963FAE95
:10A73000259727962FAE279722ED822E23E5922E7E
:10A740002BEFA22E20E4B22E14C02196DFAE21976B
:10A750002396CFAE239725963FAE259727962FAE0B
:10A76000279792ED892E93E5992E9BEFA92E91E4E0
:10A77000B92E8BA99CA9ADA9BEA92C968CAF9DAF73
:10A78000AEAFBFAF2C979C01AD01B201C3010E94D7
:10A7900083EA698B7A8B8B8B9C8B4FA458A869A812
:10A7A0007AA8A30192016D2D7C2D832D922D0E94FC
:10A7B00083EA6D8B7E8B8F8B988F2C962CAD3DAD65
:10A7C0004EAD5FAD2C976091360470913704809147
:10A7D0003804909139040E9483EA2C966CAF7DAFC7
:10A7E0008EAF9FAF2C97A301920160913A047091B4
:10A7F0003B0480913C0490913D040E9483EA2B012C
:10A800003C018F2D902FA12FBE2D89839A83AB837E
:10A81000BC8321968FAD219723969FAD23972596D4
:10A82000AFAD25972796BFAD27978D839E83AF83C6
:10A83000B8878091A6109091A710A091A810B09110
:10A84000A91089879A87AB87BC872DEC3CEC4CEC30
:10A850005CE3C501B4010E949DE62091AA103091ED
:10A86000AB104091AC105091AD100E949DE620912C
:10A8700042043091430440914404509145040E94A5
:10A8800084EA6D877E878F87988B2C962CAD3DADA3
:10A890004EAD5FAD2C97CA01B9010E949DE66B01D8
:10A8A0007C01A3019201C301B2010E949DE69B01BC
:10A8B000AC01C701B6010E9484EA20E030E040E02C
:10A8C00050E40E94AAEC18160CF046C00E9421B178
:10A8D0001BA21CA21DA21EA220E030E040E05FE30C
:10A8E00060913E0470913F04809140049091410436
:10A8F0000E9484EA6F8F78A389A39AA39E012D5D9D
:10A900003F4FAE01415E5F4F6AE374E086E394E03F
:10A910001ED81BA21CA21DA21EA220E030E040E017
:10A920005FE36091A6107091A7108091A81090919C
:10A93000A9100E9484EA6F8F78A389A39AA39E012D
:10A940002D5D3F4FAE01415E5F4FBE01615D7F4FA8
:10A95000CE01C3960E94A74C1F8E18A219A21AA25C
:10A960009E01215E3F4F46EA50E1BE01615D7F4F8F
:10A97000CE01C3960E94A74C0E944DB14090300278
:10A98000509031026090320270903302E090FB06EA
:10A99000F090FC060091FD061091FE06A090F706CF
:10A9A000B090F806C090F906D090FA069501A6017D
:10A9B000B701C8010E94AAEC181614F475018601AB
:10A9C00020E030E040E251E4B701C8010E9460EBB2
:10A9D000609330027093310280933202909333027D
:10A9E00040E0BE016F5E7F4FCE0101960E94C8A479
:10A9F00040923002509231026092320270923302E1
:10AA00000E949D4CA1E0BAE02496BFAFAEAF249760
:10AA100022961FAE1EAE229701E010E021960FACE9
:10AA2000219702C0000F111F0A94E2F72296EEADA3
:10AA3000FFAD229731962296FFAFEEAF229721E02D
:10AA400030E021960FAC219702C0220F331F0A94E9
:10AA5000E2F763963FAF2EAF639787EB282E84E033
:10AA6000382E87EF94E02A969FAF8EAF2A97A7EDF6
:10AA7000B4E02896BFAFAEAF2897EDEEF9E026968A
:10AA8000FFAFEEAF26972A962EAD3FAD2A9765967B
:10AA90003FAF2EAF6597D9018D919C919C012023EA
:10AAA0003123232B09F4ADC06396EEADFFAD639760
:10AAB0008E239F23892B09F4A4C02896AEADBFAD89
:10AAC00028978D919C9180239123892B09F099C01F
:10AAD00020E030E040E050E42496AEADBFAD2497D6
:10AAE0006D917D918D919C910E9484EA6B017C0116
:10AAF00020E030E040E050E42496EEADFFAD249736
:10AB000064817581868197810E9483EA4B015C0193
:10AB100020E030E040E850ECC701B6010E9438E682
:10AB200087FD70C120E030E04BE553E4C701B6017A
:10AB30000E94AAEC181634F4C12CD12CBBE5EB2EE4
:10AB4000B3E4FB2ECBA6DCA6EDA6FEA62696AEAD04
:10AB5000BFAD26974D905D906D907C9020E030E0E9
:10AB600040E85FE3C301B2010E9438E687FD51C1AE
:10AB700020E030E04BE553E4C301B2010E94AAECAF
:10AB8000181634F4412C512CFBE56F2EF3E47F2E84
:10AB90004F8E58A269A27AA24FA258A669A67AA699
:10ABA00020E030E040E850ECC501B4010E9438E6F6
:10ABB00087FD36C120E030E04BE553E4C501B40128
:10ABC0000E94AAEC181634F4812C912C7BE5A72E58
:10ABD00073E4B72E8BA29CA2ADA2BEA2AE01495DCA
:10ABE0005F4FC701B6010E949D4A811120C128967E
:10ABF000EEADFFAD289780819181802B912B9183C1
:10AC000080832A962EAD3FAD2A972E5F3F4F2A961E
:10AC10003FAF2EAF2A976596AEADBFAD65978D91CC
:10AC20009C9180239123892B09F4A6C0F90180818E
:10AC3000918180239123892B09F49EC0F1018081A9
:10AC4000918180239123892B09F096C020E030E088
:10AC500040E050E42696AEADBFAD26976D917D9154
:10AC60008D919C910E9484EA2B013C0120E030E010
:10AC700040E050E42696EEADFFAD269764817581E5
:10AC8000868197810E9483EA4B015C012496AEADD8
:10AC9000BFAD2497CD90DD90ED90FC9020E030E0AA
:10ACA00040E850ECC701B6010E9438E687FDFFC0BE
:10ACB00020E030E04BE553E4C701B6010E94AAEC66
:10ACC000181634F4C12CD12C5BE5E52E53E4F52E97
:10ACD000CBA2DCA2EDA2FEA2CBA6DCA6EDA6FEA630
:10ACE00020E030E040E85FE3C301B2010E9438E6B3
:10ACF00087FDE4C020E030E04BE553E4C301B2013E
:10AD00000E94AAEC181634F4412C512C3BE5632E1A
:10AD100033E4732E4FA258A669A67AA620E030E04D
:10AD200040E85FE3C501B4010E9438E687FDCDC06D
:10AD300020E030E04BE553E4C501B4010E94AAECE9
:10AD4000181634F4812C912C9BE5A92E93E4B92E8E
:10AD50008F8E98A2A9A2BAA2AE01495D5F4FC7012A
:10AD6000B6010E949D4A8111B7C0F1018081918195
:10AD7000802B912B91838083F2E02F0E311C28963B
:10AD80002EAD3FAD28972E5F3F4F28963FAF2EAF99
:10AD9000289726968EAD9FAD2697049626969FAF50
:10ADA0008EAF269791EC291694E0390609F06BCE08
:10ADB0002496AEADBFAD249714962496BFAFAEAF28
:10ADC00024972296EEADFFAD2297359709F024CE59
:10ADD00080919A1880939B182F962EAD3FAD2F9798
:10ADE000215031092F963FAF2EAF2F97232B09F417
:10ADF000B3C02D963FAD2D9737FDAEC08FAD87FF09
:10AE000047CBAAC0C12CD12CA0E8EA2EA0ECFA2E88
:10AE100099CE412C512CE0E86E2EEFE37E2EB8CE79
:10AE2000812C912C60E8A62E60ECB62ED3CEAE011C
:10AE3000415E5F4FC501B4010E949D4A882309F419
:10AE4000D6CE80912404882321F1B701A60189ED93
:10AE500095E10E9432C54FA158A569A57AA583ED59
:10AE600095E10E9432C54BA15CA16DA17EA189EC48
:10AE700095E10E9432C54F8D58A169A17AA183EC5A
:10AE800095E10E9432C589E20E94C6898AE00E944B
:10AE9000C6899E01215E3F4FAE014D5D5F4FBE01F1
:10AEA000695D7F4FCE018B960E947DB1A0CEC12CF3
:10AEB000D12C40E8E42E40ECF42E0ACF412C512C4A
:10AEC00020E8622E2FE3722E25CF812C912C80E872
:10AED000A82E8FE3B82E3CCFAE01415E5F4FC70175
:10AEE000B6010E949D4A882309F43FCF8091240433
:10AEF000882321F1B701A6018FE995E10E9432C5AF
:10AF00004FA158A569A57AA589E995E10E9432C5A6
:10AF10004BA15CA16DA17EA18FE895E10E9432C595
:10AF20004F8D58A169A17AA189E895E10E9432C5A7
:10AF300089E20E94C6898AE00E94C6899E01215E3C
:10AF40003F4FAE014D5D5F4FBE01695D7F4FCE014A
:10AF50008B960E947DB109CF0E9421B180E090E0E4
:10AF6000A0EAB0E48093BA109093BB10A093BC10F9
:10AF7000B093BD1019821A821B821C829E012F5F22
:10AF80003F4F4AEB50E166EB70E182EB90E10E94AB
:10AF9000A74C80911B0590911C05A0911D05B091B7
:10AFA0001E058093B2109093B310A093B410B09389
:10AFB000B5108091170590911805A0911905B091D1
:10AFC0001A058093B6109093B710A093B810B09361
:10AFD000B91019821A821B821C829E012F5F3F4F7B
:10AFE0004AEB50E166EB70E182EB90E10E94A74CE6
:10AFF0006096FFAD6097F11113C010924904109252
:10B0000048040E94B07680E090E0E7D109C02FADFF
:10B01000F42C052D162DE72C24300CF033CB20CB4F
:10B02000CC5ADF4F0FB6F894DEBF0FBECDBFDF9115
:10B03000CF911F910F91FF90EF90DF90CF90BF9035
:10B04000AF909F908F907F906F905F904F903F90C8
:10B050002F9008951F920F920FB60F9211240BB6E6
:10B060000F922F933F938F939F93EF93FF93209192
:10B07000160F3091170F8091180F9091190F281704
:10B08000390731F4809131018F7D8093310114C0F3
:10B09000E091180FF091190FEA56F14F208180913D
:10B0A000180F9091190F01968F7799279093190F88
:10B0B0008093180F20933601FF91EF919F918F910C
:10B0C0003F912F910F900BBE0F900FBE0F901F90CE
:10B0D00018951F920F920FB60F9211240BB60F9274
:10B0E0002F934F935F938F939F93EF93FF93809151
:10B0F000300182FD1CC02091360180919A0F909101
:10B100009B0F40919C0F50919D0F01968F7799272F
:10B110004817590771F0E0919A0FF0919B0FE65E86
:10B12000F04F208390939B0F80939A0F02C08091E1
:10B130003601FF91EF919F918F915F914F912F91E8
:10B140000F900BBE0F900FBE0F901F901895CF92CF
:10B15000DF92EF92FF920F931F93CF93DF936C01D7
:10B160007A018B01C0E0D0E0CE15DF0581F0D80177
:10B170006D918D01D601ED91FC910190F081E02D52
:10B18000C6011995892B11F02196EECF7E01C701DA
:10B19000DF91CF911F910F91FF90EF90DF90CF90B3
:10B1A00008950E9494ED3FB7F8948091D306909152
:10B1B000D406A091D506B091D60626B5A89B05C0A9
:10B1C0002F3F19F00196A11DB11D3FBFBA2FA92F26
:10B1D000982F8827820F911DA11DB11DBC01CD01A3
:10B1E00042E0660F771F881F991F4A95D1F708958F
:10B1F0002FB7F8946091CF067091D0068091D10658
:10B200009091D2062FBF08951F920F920FB60F9202
:10B2100011242F933F938F939F93AF93BF9380916C
:10B22000CF069091D006A091D106B091D206309170
:10B23000CE0623E0230F2D3720F40196A11DB11D6A
:10B2400005C026E8230F0296A11DB11D2093CE064E
:10B250008093CF069093D006A093D106B093D206E8
:10B260008091D3069091D406A091D506B091D606D0
:10B270000196A11DB11D8093D3069093D406A0938F
:10B28000D506B093D606BF91AF919F918F913F9114
:10B290002F910F900FBE0F901F9018951F920F9235
:10B2A0000FB60F9211240BB60F922F933F934F932B
:10B2B0005F936F937F938F939F93AF93BF93EF931E
:10B2C000FF9380912F0590913005A0913105B091A9
:10B2D0003205892B8A2B8B2B59F190912E05E09109
:10B2E0002C05F0912D0580818927808380912F0581
:10B2F00090913005A0913105B091320518161906CC
:10B300001A061B060CF056C080912F05909130054F
:10B31000A0913105B09132050197A109B10980933F
:10B320002F0590933005A0933105B093320542C0AC
:10B3300080911902E5E5F8E1E4919FEF90931902FD
:10B34000E230C9F050F4EE2399F0E13081F59091AC
:10B350006F009D7F90936F002AC0E43019F1E0F0F8
:10B36000E53029F5909173009D7F909373001FC085
:10B3700010926E001CC0909170009D7F90937000A1
:10B3800091E09093B0009091B100987F9460909379
:10B39000B1001092B3000BC0909171009D7F90930B
:10B3A000710005C0909172009D7F9093720060E0E3
:10B3B0000E94D9B5FF91EF91BF91AF919F918F916D
:10B3C0007F916F915F914F913F912F910F900BBEA5
:10B3D0000F900FBE0F901F90189590934F0480937D
:10B3E0004E0480E00C94FC762F923F924F925F9235
:10B3F0006F927F928F929F92AF92BF92CF92DF9285
:10B40000EF92FF920F931F93CF93DF93CDB7DEB7E9
:10B41000C857D1090FB6F894DEBF0FBECDBFE0917B
:10B420004E07F0914F07EF2B11F00C94B462289661
:10B43000DFAECEAE28976E2C79016A015B01FC016C
:10B4400020813181428153816C962CAF3DAF4EAF4C
:10B450005FAF6C97209196103091971040919810A3
:10B46000509199106C966CAD7DAD8EAD9FAD6C9783
:10B470000E949DE60E94B5ECE0966CAF7DAF8EAF6A
:10B480009FAFE097D5018D919D910D90BC91A02D1E
:10B49000A0968CAF9DAFAEAFBFAFA09720919A1092
:10B4A00030919B1040919C1050919D10BC01CD019A
:10B4B0000E949DE60E94B5ECE4966CAF7DAF8EAF26
:10B4C0009FAFE497D6012D913D914D915C91A4964B
:10B4D0002CAF3DAF4EAF5FAFA49720919E1030913F
:10B4E0009F104091A0105091A110A4966CAD7DAD1D
:10B4F0008EAD9FADA4970E949DE60E94B5ECE896A4
:10B500006CAF7DAF8EAF9FAFE897D7012D913D9186
:10B510004D915C9122962CAF3DAF4EAF5FAF22971D
:10B520002091A2103091A3104091A4105091A51029
:10B5300022966CAD7DAD8EAD9FAD22970E949DE6AB
:10B540000E94B5EC60966CAF7DAF8EAF9FAF6097F9
:10B550008091140783FF1CC060962CAD3DAD4EADAD
:10B560005FAD60972093E9093093EA094093EB09B6
:10B570005093EC0922968CAD9DADAEADBFAD229738
:10B580008093D9099093DA09A093DB09B093DC0981
:10B59000D801BC91B9A7F801F181F9ABD801129695
:10B5A000BC91BEABF801F381FAAF8091B7099091DD
:10B5B000B809891B8F708F3019F40E94FCA0F5CF59
:10B5C0000091B709E9960FAFE9978091B709082F65
:10B5D00010E01CA30BA38091DD099091DE09A091DE
:10B5E000DF09B091E009E0968CAC9DACAEACBFAC8D
:10B5F000E097881A990AAA0ABB0A8091E1099091FA
:10B60000E209A091E309B091E409E4962CAC3DACC9
:10B610004EAC5FACE497281A390A4A0A5B0A80915B
:10B62000E5099091E609A091E709B091E809E8964B
:10B630002CAD3DAD4EAD5FADE897281B390B4A0BE5
:10B640005B0B2DA33EA34FA358A78091E9099091CE
:10B65000EA09A091EB09B091EC0960960CAD1DAD23
:10B660002EAD3FAD6097081B190B2A0B3B0B0DA7A6
:10B670001EA72FA738AB012B022B032B09F4BCC04C
:10B680008091130781114BC0609150047091510457
:10B6900080915204909153040E94C8EB209125029E
:10B6A00030912602621773070CF039C060962CADFA
:10B6B0003DAD4EAD5FAD60972093E9093093EA0947
:10B6C0004093EB095093EC0922968CAD9DADAEAD45
:10B6D000BFAD22978093D9099093DA09A093DB0933
:10B6E000B093DC09E2EFFDE184918F010F5F1F4F02
:10B6F000811103C0E9ECF9E104C00E94C689F80198
:10B70000F3CF84918F010F5F1F4F882321F00E9498
:10B71000C689F801F6CF1DA61EA61FA618AA94E09A
:10B72000699E800111240F5D1D4F6DA57EA58FA51B
:10B7300098A90E943EE6D8012D913D914D915C91D2
:10B740000E949DE66B017C0120E030E0A9010E948F
:10B75000AAEC87FF04C0F7FAF094F7F8F094609130
:10B76000A2107091A3108091A4109091A5100E9436
:10B77000C8EB9B01AC01A8ECB0E00E9464EA0E9417
:10B780003EE6A70196010E9438E687FF39C0609621
:10B790000CAD1DAD2EAD3FAD60970093E909109340
:10B7A000EA092093EB093093EC0922962CAD3DADCC
:10B7B0004EAD5FAD22972093D9093093DA094093BB
:10B7C000DB095093DC09E2EFFDE184918F010F5F0B
:10B7D0001F4F811103C0EAEAF9E104C00E94C68943
:10B7E000F801F3CF84918F010F5F1F4F882321F061
:10B7F0000E94C689F801F6CF1DA61EA61FA618AA8C
:10B80000D501C4018827B7FD83959927AA27BB27AF
:10B81000782E57FE03C0382F3260732E8DA19EA163
:10B82000AFA1B8A5B7FF03C0972D9460792E0DA5E1
:10B830001EA52FA538A937FF03C0172D1860712E3C
:10B8400024E0629E800111240F5D1D4F6DA57EA531
:10B850008FA598A90E943EE6D8012D913D914D916A
:10B860005C910E949DE66B017C0120E030E0A90123
:10B870000E94AAEC87FF04C0C701B601905802C01D
:10B88000C701B60120E030E040E05FE30E9484EAB7
:10B890000E94CDEB6AAB7BAB8CAB9DAB88E60BA17A
:10B8A0001CA1809FF001819FF00D1124ED58FE4EE8
:10B8B0001082EA5BFF4F7082B501A401B7FE07C09A
:10B8C00044275527BA01481959096A097B0988E6AE
:10B8D0000BA11CA1809FF001819FF00D1124ED5858
:10B8E000FE4E458B568B678B708F2C962CAE3DAEE3
:10B8F0004EAE5FAE2C9757FE0DC088279927DC010E
:10B9000082199309A409B5092C968CAF9DAFAEAFEF
:10B91000BFAF2C9728E60BA11CA1209FF001219F0F
:10B92000F00D1124ED58FE4E2C968CAD9DADAEADB4
:10B93000BFAD2C97818F928FA38FB48F0DA11EA1C5
:10B940002FA138A537FF07C0309520951095019598
:10B950001F4F2F4F3F4FE8E67E2EABA1BCA17A9E32
:10B96000F0017B9EF00D1124ED58FE4E058F168FD1
:10B97000278F30A38AA99BA9ACA9BDA981A392A3B3
:10B98000A3A3B4A323964FAF2397752EF62FE72FCB
:10B990002C968CAD9DADAEADBFAD2C974817590719
:10B9A0006A077B0778F429969FAD299723969FAF66
:10B9B00023972A967FAC2A972B96FFAD2B972C9630
:10B9C000EFAD2C9723968FAD2397972DAF2FBE2FDA
:10B9D00080179107A207B30710F4D901C8010AA97B
:10B9E0001BA92CA93DA980179107A207B30710F442
:10B9F000D901C80128E60BA11CA1209FF001219FBD
:10BA0000F00D1124ED58FE4E85A396A3A7A3B0A771
:10BA10000697A105B10508F4A0C5DF01AE59BF4FD7
:10BA200080914604909147048D939C9361A6452B89
:10BA3000462B472B09F05F9888E60BA11CA1809F3D
:10BA4000F001819FF00D1124ED58FE4E818D928DF5
:10BA5000A38DB48D892B8A2B8B2B11F08A98479854
:10BA600088E60BA11CA1809FF001819FF00D11249D
:10BA7000ED58FE4E858D968DA78DB0A1892B8A2B12
:10BA80008B2B31F0809108018170809306014798DB
:10BA90002AA93BA94CA95DA9232B242B252B09F40A
:10BAA00065C580911907882319F081508093190783
:10BAB000611004C0129880E28093190760900F070C
:10BAC0007090100700911107109112079301A801BF
:10BAD00069A579A98EA99AAD0E9438E687FF04C0AE
:10BAE00069A679AA0EAB1AAFC501B4010E943EE661
:10BAF000209163113091641140916511509166114C
:10BB00000E949DE626966CAF7DAF8EAF9FAF2697C5
:10BB1000698B7A8B8B8B9C8BC201B1010E943EE6B4
:10BB200020916711309168114091691150916A110B
:10BB30000E949DE62B013C016D8B7E8B8F8B988F35
:10BB40006DA17EA18FA198A50E943EE620916B1168
:10BB500030916C1140916D1150916E110E949DE6D3
:10BB60004B015C01698F7A8F8B8F9C8F20916F11B5
:10BB7000309170114091711150917211C701B6014D
:10BB80000E949DE66B017C016D8F7E8F8F8F98A345
:10BB900088E60BA11CA1809FF001819FF00D11246C
:10BBA000ED58FE4E258936894789508D2DA33EA339
:10BBB0004FA358A7263031054105510508F4DFC4CD
:10BBC0002896AEADBFAD2897CD90DD90ED90FC905E
:10BBD00020E030E0A901C701B6010E9438E68111DA
:10BBE000EDC426962CAD3DAD4EAD5FAD2697CA0196
:10BBF000B9010E949DE66B017C01A3019201C30182
:10BC0000B2010E949DE69B01AC01C701B6010E94F2
:10BC100084EA6B017C01A5019401C501B4010E9475
:10BC20009DE69B01AC01C701B6010E9484EA0E9417
:10BC3000EFEC28E60BA11CA1209FF001219FF00D45
:10BC40001124ED58FE4E658776878787908B88E6AE
:10BC50000BA11CA1809FF001819FF00D1124ED58D4
:10BC6000FE4E4584568467847088A301920160E08B
:10BC700070E080E89FE30E9460EB64966CAF7DAF5C
:10BC80008EAF9FAF649729A539A94EA95AAD0E94DE
:10BC90009DE64B015C018091B7099091B509891B24
:10BCA0008F7027968FAF2797A501940160E074E20B
:10BCB00084E799E40E9460EB0E94B5EC6B017C0183
:10BCC00027968FAD27978250863008F486C4A50149
:10BCD0009401C301B2010E949DE69B01AC010E9448
:10BCE0009DE668966CAF7DAF8EAF9FAF689788E694
:10BCF000ABA1BCA18A9F80018B9F100D11240D5810
:10BD00001E4E68962CAD3DAD4EAD5FAD6897D80127
:10BD100011962D933D934D935C93149795962D9189
:10BD20003D914D915C9198972EAB3FAB48AF59AF89
:10BD3000CA01B9010E943CE66AAF7BAF8CAF9DAFF0
:10BD40009B01AC01C501B4010E949DE60E944AEB33
:10BD50000E94CDEBA8966CAF7DAF8EAF9FAFA8973A
:10BD6000F801EE5AFF4F60837183828393838E01C3
:10BD70000F5E1F4F2A961FAF0EAF2A970051110971
:10BD800024961FAF0EAF249707EF16E0AC961FAFB7
:10BD90000EAFAC978E010F5D1F4F1AA309A3249617
:10BDA0000EAD1FAD2497AA961FAF0EAFAA97312CE8
:10BDB000212C10E819A70FE309AB2A96AEADBFAD51
:10BDC0002A972D913D914D915D912A96BFAFAEAFCF
:10BDD0002A97C501B4010E949DE66B017C01AA96D9
:10BDE000EEADFFADAA976193719381939193AA965B
:10BDF000FFAFEEAFAA9720E030E0A9010E94AAECC5
:10BE000087FF04C0F7FAF094F7F8F094AC96AEAD63
:10BE1000BFADAC974D905D906D907D90AC96BFAFEF
:10BE2000AEAFAC97A7019601C301B2010E9438E6FC
:10BE300087FD0DC409A11AA12A962EAD3FAD2A9700
:10BE40000217130709F0B9CF20E030E040E85FE3C4
:10BE5000632D722D89A599A90E9438E687FF58C0E5
:10BE60007E0131E1E30EF11C24960EAD1FAD249747
:10BE7000232D322D49A559A9D8016D917D918D9120
:10BE80009C910E949DE6F801619371938193919337
:10BE90008F01EE16FF0661F728E60BA11CA1209F7B
:10BEA000C001219F900D11249C012D583E4E790117
:10BEB00089010E5A1F4FA8966CAD7DAD8EAD9FAD1A
:10BEC000A8970E943CE6232D322D49A559A90E942E
:10BED0009DE60E94CDEBD8016D937D938D939C934D
:10BEE0001397232D322D49A559A9632D722D89A5AC
:10BEF00099A90E949DE668962CAD3DAD4EAD5FAD13
:10BF000068970E949DE6F70161837283838394831F
:10BF10002AAD3BAD4CAD5DAD64966CAD7DAD8EADE7
:10BF20009FAD64970E949DE669A77AA78BA79CA7FF
:10BF30000DA11EA12FA138A5012B022B032B09F067
:10BF40009EC388E62BA13CA1829F8001839F100D98
:10BF500011240D581E4EF801818D928DA38DB48D44
:10BF6000892B8A2B8B2B09F08AC3858D968DA78D03
:10BF7000B0A1892B8A2B8B2B09F081C32091F3066A
:10BF80003091F4064091F5065091F60669A57AA520
:10BF90008BA59CA50E949DE60E944AEB0E94CDEBDA
:10BFA0002B013C01F801E95BFF4F108288E62BA1D1
:10BFB0003CA1829F8001839F100D11240D581E4EBD
:10BFC000F801E25AFF4F4082518262827382C301BC
:10BFD000B2010E943CE629A53AA54BA55CA50E94AA
:10BFE00060EB6AAF7BAF8CAF9DAFD80151966D937C
:10BFF0007D938D939C935497F801E95BFF4F80816B
:10C00000882381F17801B8E4EB0EF11C379620917A
:10C01000E7063091E8064091E9065091EA06608112
:10C020007181828193810E949DE62AAD3BAD4CAD2A
:10C030005DAD0E949DE62091A2103091A310409129
:10C04000A4105091A5100E949DE69B01AC0160E0F8
:10C0500074E284EF99E40E9460EB0E94CDEBF7015B
:10C060007183608388E60BA11CA1809FF001819FF2
:10C07000F00D1124ED58FE4E21813281438154810F
:10C080002C962CAF3DAF4EAF5FAF2C97CA01B901D4
:10C090000E94EFEC362E272E8C0147ED56E062967B
:10C0A0005FAF4EAF62973E0151E1650E711C87EDA7
:10C0B00096E09FAB8EAB24964EAC5FAC24973DA62A
:10C0C0002DA209A719AB1AAAD201CD90DD90ED904F
:10C0D000FD902D0120E030E0A901C701B6010E94CA
:10C0E000AAEC87FF04C0F7FAF094F7F8F094EEA9F1
:10C0F000FFA981909190A190B190FFABEEABA70109
:10C100009601C501B4010E9438E687FDD8C56414C4
:10C110007504D1F627965FAD2797552309F448C6D5
:10C12000C090B909D090BA09E090BB09F090BC0961
:10C130002DEB37E346E855E3C701B6010E9438E628
:10C1400087FD36C6C701B6010E94EFEC6B017C018A
:10C150009B01AC01632D722DC8010E9438E687FD5A
:10C1600003C03C2C2D2C87019601A701632D722D55
:10C17000C8010E9460EB68966CAF7DAF8EAF9FAF39
:10C1800068978DEB99E028969FAF8EAF289720E0B7
:10C1900030E040E85FE32AAB3BAB4CAB5DAB1EAAA3
:10C1A0002896AEADBFAD28972D913D914D915D91F3
:10C1B0002896BFAFAEAF289768966CAD7DAD8EADBB
:10C1C0009FAD68970E949DE64B015C012496EEAD01
:10C1D000FFAD2497C190D190E190F1902496FFAFEC
:10C1E000EEAF2497FEA9FF2391F02AA93BA94CA901
:10C1F0005DA90E949DE64B015C012AA93BA94CA9BF
:10C200005DA9C701B6010E949DE66B017C01A701F3
:10C210009601C501B4010E94AAEC20E030E0A9011A
:10C2200018160CF092C5C701B6010E94AAEC1816A8
:10C230000CF486C520E030E0A901C501B4010E94DC
:10C2400038E687FD7DC52601370177FA709477F8C7
:10C250007094A3019201C501B4010E94AAEC1816C2
:10C2600014F4240135016296AEADBFAD6297CD9056
:10C27000DD90ED90FD906296BFAFAEAF6297A301E7
:10C280009201C701B6010E9438E687FF15C0A301DD
:10C290009201C701B6010E9460EB9B01AC016AA943
:10C2A0007BA98CA99DA90E949DE66AAB7BAB8CAB58
:10C2B0009DABBEA9BF5FBEABEDECF9E028962EADFD
:10C2C0003FAD2897E217F30709F06ACF3EA9332361
:10C2D00061F02AA93BA94CA95DA9632D722DC80163
:10C2E0000E949DE6362E272E8C0124EA30E74DE78A
:10C2F0005FE3632D722DC8010E949DE66B017C01F6
:10C300002091150730911607409117075091180793
:10C310000E9438E687FD42C58DA59DA1A9A5B9A9B2
:10C320008093150790931607A0931707B0931807EB
:10C3300028E64BA15CA1249FC001259F900D1124EC
:10C34000DC01AD58BE4E7D01232D322DA801632D99
:10C35000722DC8010E949DE6F7016187728783876D
:10C3600094876AAD7BAD8CAD9DAD90589B01AC01BF
:10C370000E9484EAD7011D962D913D914D915C91CB
:10C3800050970E949DE69B01AC016BE077ED83E244
:10C390009BE30E9483EA9B01AC018BE097EDA3E253
:10C3A000BBE3F70185839683A783B08710812C9622
:10C3B0006CAD7DAD8EAD9FAD2C970E9438E6181602
:10C3C0000CF4FBC483E0182B88E62BA13CA1829FD0
:10C3D000F001839FF00D1124ED58FE4E108380E193
:10C3E000FE013196ADEBB9E001900D928A95E1F72F
:10C3F0002C968CAD9DADAEADBFAD2C978093B90999
:10C400009093BA09A093BB09B093BC09E0960CAD18
:10C410001DAD2EAD3FADE0970093DD091093DE0911
:10C420002093DF093093E009E4962CAD3DAD4EAD8D
:10C430005FADE4972093E1093093E2094093E3096B
:10C440005093E409E8968CAD9DADAEADBFADE897D5
:10C450008093E5099093E609A093E709B093E80972
:10C4600060960CAD1DAD2EAD3FAD60970093E90910
:10C470001093EA092093EB093093EC096C962CADEC
:10C480003DAD4EAD5FAD6C972093CD093093CE0995
:10C490004093CF095093D009A0968CAD9DADAEAD21
:10C4A000BFADA0978093D1099093D209A093D309EF
:10C4B000B093D409A4960CAD1DAD2EAD3FADA4979D
:10C4C0000093D5091093D6092093D7093093D80942
:10C4D00022962CAD3DAD4EAD5FAD22972093D9098C
:10C4E0003093DA094093DB095093DC099091B70946
:10C4F0008091B809981303C084E68093B409E99643
:10C500008FADE9978F5F8F708093B7098091B709DE
:10C510009091B60981508F70891351C41091B80958
:10C520001BA30091B7090DA728E61BA10DA51013A9
:10C53000D1C4812C912CA12CB12C1DA219A619AA11
:10C540001EAE212C312C00E010E02DA53BA12313C1
:10C55000CEC42114310409F07FC580916F00826040
:10C5600080936F0081E0ECC680E0EAC660900B0724
:10C5700070900C0700910D0710910E07A7CA818DCE
:10C58000928DA38DB48D0697A105B10508F018CB47
:10C59000858D968DA78DB0A10697A105B10508F0F0
:10C5A0000FCB20E030E0A901C701B6010E94AAEC40
:10C5B00087FF04C0F7FAF094F7F8F09488E60BA12F
:10C5C0001CA1809FF001819FF00D1124ED58FE4EBB
:10C5D000C586D686E786F08A3ACB80910707909188
:10C5E0000807A0910907B0910A07C816D906EA06FC
:10C5F000FB0608F06CCB8C199D09AE09BF09BC0184
:10C60000CD01660F771F881F991F27964FAD27977B
:10C61000042F10E020E030E0A90198010E9426EAF2
:10C62000CA01B9010E943CE60E94B5EC6C0D7D1D6B
:10C630008E1D9F1D0E943CE69B01AC0160E074E2F0
:10C6400084E799E40E9460EB4B015C0140CBA701B9
:10C650009601C301B2010E9460EB7B018C019B013A
:10C66000AC01632D722D89A599A90E94AAEC181618
:10C670000CF0E0CB3E2C2F2C09A719ABDBCB0AA981
:10C680001BA92CA93DA9012B022B032B49F02091BA
:10C69000EF063091F0064091F1065091F20608C085
:10C6A0002091EB063091EC064091ED065091EE069C
:10C6B00069A57AA58BA59CA50E949DE60E944AEBE0
:10C6C0000E94CDEB2B013C012AA93BA94CA95DA9F5
:10C6D000232B242B252BC9F020E030E0A901609109
:10C6E000E7067091E8068091E9069091EA060E94BB
:10C6F00038E6882351F081E00DA51EA52FA538A9A5
:10C7000010161106120613060CF080E098E62BA115
:10C710003CA1929F8001939F100D11240D581E4E35
:10C72000180137E4230E311CD1018C93882309F4BE
:10C73000B3C02091CD093091CE094091CF095091DD
:10C74000D0096C966CAD7DAD8EAD9FAD6C970E949F
:10C7500083EA6DA77EA78FA798AB2091D10930916E
:10C76000D2094091D3095091D409A0966CAD7DAD0A
:10C770008EAD9FADA0970E9483EA4B015C01209192
:10C78000D5093091D6094091D7095091D809A4967E
:10C790006CAD7DAD8EAD9FADA4970E9483EA6B0119
:10C7A0007C012DA53EA54FA558A9CA01B9010E943B
:10C7B0009DE66DA77EA78FA798ABA5019401C50143
:10C7C000B4010E949DE69B01AC016DA57EA58FA5DD
:10C7D00098A90E9484EA4B015C01A7019601C70158
:10C7E000B6010E949DE69B01AC01C501B4010E9407
:10C7F00084EA0E94EFEC6B017C012091D909309111
:10C80000DA094091DB095091DC0922966CAD7DADCF
:10C810008EAD9FAD22970E9483EAA70196010E94E8
:10C8200060EB6B017C01F801E25BFF4F6083718379
:10C830008283938320E030E040E450E40E94AAEC3D
:10C8400018161CF4F101108227C02091E7063091E0
:10C85000E8064091E9065091EA06C701B6010E9438
:10C860009DE69B01AC016091E3067091E406809126
:10C87000E5069091E6060E9460EB29A53AA54BA536
:10C880005CA50E949DE60E94CDEB641575058605AA
:10C89000970510F42B013C0180913F1190914011BC
:10C8A000A0914111B09142110EA91FA928AD39AD37
:10C8B00080179107A207B30708F4DFC02DA13EA19E
:10C8C0004FA158A5232B242B252B41F16091431117
:10C8D0007091441180914511909146116415750530
:10C8E00086059705D8F42EA93FA948AD59AD0E94F9
:10C8F00017EA6B017C012DA13EA14FA158A5C301F0
:10C90000B2010E9417EAC616D706E806F90630F407
:10C91000C701B6010E9426EA29013A0188E60BA167
:10C920001CA1809FF001819FF00D1124ED58FE4E57
:10C93000C18CD28CE38CF48CC114D104E104F104D9
:10C9400031F1609147117091481180914911909196
:10C950004A116415750586059705C8F42EA93FA9E7
:10C9600048AD59AD0E9417EA4B015C01A701960141
:10C97000C301B2010E9417EA86169706A806B906F7
:10C9800030F4C501B4010E9426EA29013A0188E683
:10C990000BA11CA1809FF001819FF00D1124ED5887
:10C9A000FE4EC58CD68CE78CF0A0C114D104E104F6
:10C9B000F10431F160914B1170914C1180914D1146
:10C9C00090914E116415750586059705C8F42EA93A
:10C9D0003FA948AD59AD0E9417EA4B015C01A70180
:10C9E0009601C301B2010E9417EA86169706A806AF
:10C9F000B90630F4C501B4010E9426EA29013A01C2
:10CA000088E60BA11CA1809FF001819FF00D1124ED
:10CA1000ED58FE4EC1A0D2A0E3A0F4A0C114D104F1
:10CA2000E104F10409F4C2CA60914F1170915011F0
:10CA300080915111909152116415750586059705E5
:10CA400008F0B4CA2EA93FA948AD59AD0E9417EA13
:10CA50004B015C01A7019601C301B2010E9417EAD4
:10CA600086169706A806B90608F0A0CAC501B40143
:10CA70000E9426EA29013A0199CA2DA13EA14FA19F
:10CA800058A5232B242B252BC9F1609143117091BC
:10CA900044118091451190914611641575058605E4
:10CAA000970560F50E943CE62AAD3BAD4CAD5DAD0F
:10CAB0000E949DE66B017C016DA17EA18FA198A5CE
:10CAC0000E943CE64B015C01C301B2010E943CE6BE
:10CAD000A50194010E949DE69B01AC01C701B6012E
:10CAE0000E9438E687FF0AC0A5019401C701B6017C
:10CAF0000E9460EB0E94CDEB2B013C0188E60BA16C
:10CB00001CA1809FF001819FF00D1124ED58FE4E75
:10CB1000818C928CA38CB48C81149104A104B104F7
:10CB2000B9F160914711709148118091491190912C
:10CB30004A11641575058605970550F50E943CE677
:10CB40002AAD3BAD4CAD5DAD0E949DE66B017C0115
:10CB5000C501B4010E943CE64B015C01C301B20176
:10CB60000E943CE6A50194010E949DE69B01AC0158
:10CB7000C701B6010E9438E687FF0AC0A5019401EB
:10CB8000C701B6010E9460EB0E94CDEB2B013C0176
:10CB900088E60BA11CA1809FF001819FF00D11245C
:10CBA000ED58FE4E858C968CA78CB0A08114910414
:10CBB000A104B104B9F160914B1170914C118091B5
:10CBC0004D1190914E11641575058605970550F528
:10CBD0000E943CE62AAD3BAD4CAD5DAD0E949DE6AA
:10CBE0006B017C01C501B4010E943CE64B015C0174
:10CBF000C301B2010E943CE6A50194010E949DE69A
:10CC00009B01AC01C701B6010E9438E687FF0AC04C
:10CC1000A5019401C701B6010E9460EB0E94CDEB13
:10CC20002B013C0188E60BA11CA1809FF001819F94
:10CC3000F00D1124ED58FE4EC1A0D2A0E3A0F4A047
:10CC4000C114D104E104F10409F4B0C960914F1199
:10CC50007091501180915111909152116415750588
:10CC60008605970508F0A2C90E943CE62AAD3BADB7
:10CC70004CAD5DAD0E949DE64B015C01C701B60164
:10CC80000E943CE66B017C01C301B2010E943CE6BC
:10CC9000A70196010E949DE69B01AC01C501B4016C
:10CCA0000E9438E687FF82C9A7019601C501B40139
:10CCB0000E9460EB0E94CDEB2B013C0177C9FAA9E1
:10CCC000FF2331F1A5019401632D722DC8010E944B
:10CCD0009DE64B015C012DA53DA149A559A9C701C0
:10CCE000B6010E949DE69B01AC01C501B4010E9402
:10CCF00038E687FF22C0A7019601C501B4010E9452
:10CD000060EB6DA77DA389A799AB21E02AABFFC992
:10CD1000A7019601C501B4010E9460EB9B01AC0123
:10CD20006DA57DA189A599A90E949DE66DA77DA30A
:10CD300089A799AB31E03AABEAC941E04AABE7C910
:10CD4000A7019601C501B40113C0C701B6010E9435
:10CD500038E687FD09C020E030E0A901C501B40133
:10CD60000E94AAEC18164CF4A5019401C701B60163
:10CD70000E9483EA2B013C0176CA2401350177FA2F
:10CD8000709477F87094A3019201C701B6010E94D4
:10CD900038E687FD68CA2601370165CA2DA53DA181
:10CDA00049A559A9C701B6010E9438E687FFB4CA50
:10CDB0003DA42DA009A519A9AFCA81E004CBF0902C
:10CDC000B7098FEF8F0D8F708BA3B090B60980914C
:10CDD000B709B81609F454C0C12CD12C0BA10B15FE
:10CDE00009F44EC0602E712C28E6269D8001279DF7
:10CDF000100D11240D581E4ED8018C9183FD2BC0AF
:10CE00000EAF1AAB0115110541F11996BC91BDA7E2
:10CE1000F801F285FDA3D8011B96BC91B9A7F801D2
:10CE2000F485F9ABD80115962D903D904D905C900E
:10CE30001897A20191016DA57DA189A59F2F0E9440
:10CE400038E6811186C1C114D10439F0F601808120
:10CE500080FD7FC102C0CEAEDAAA8BA181508F7057
:10CE60008BA38091B6098B1103C0CEACDAA8B6CFE4
:10CE70000BA10B1529F081E08B0D8F70B82EF1CF2F
:10CE80001091B6091BA3C12CD12C8091B7090BA11D
:10CE9000801709F443CB802E912C28E6289D800131
:10CEA000299D100D11240D581E4ED8018C9183FD23
:10CEB0000AC05801C114D10439F0C6010E94417F53
:10CEC000811102C0C5C156018BA18F5F8F708BA3EA
:10CED0006501DBCF802F81508F70289FF0011124D6
:10CEE000ED58FE4E908193FF24CB8DA71ECB48E6D4
:10CEF000439FC0011124DC01AD58BE4E1D018C9131
:10CF000083FD19C015966D917D918D919C91189717
:10CF10000E94EFECF62EE72ED82EC92E0115110532
:10CF200009F48CC0F801808180FD0AC0D1018C9188
:10CF300080FD06C083C0FDA0E9A4D9A8CEAC83C003
:10CF4000F801808181608083C8010E94417F811146
:10CF500071C0F80161817281838194810E94EFEC3C
:10CF60002B013C019B01AC0160E070E080E89FE395
:10CF70000E9460EB4B015C019B01AC016F2D7E2D8B
:10CF80008D2D9C2D0E949DE669837A838B839C83E3
:10CF90002DA139A549A95EADC501B4010E949DE648
:10CFA000698B7A8B8B8B9C8BAE014F5F5F4FBE0181
:10CFB0006F5E7F4FC8010E9447B8F801E95BFF4FE1
:10CFC00080818823B9F12091E7063091E8064091ED
:10CFD000E9065091EA0637966081718182819381DA
:10CFE0000E949DE62091A2103091A3104091A410C0
:10CFF0005091A5100E949DE64B015C019B01AC0184
:10D00000C301B2010E949DE60E94CDEBF801E65BF0
:10D01000FF4F71836083A50194016F2D7E2D8D2DAF
:10D020009C2D0E949DE60E94CDEBF801E45BFF4F32
:10D0300071836083D8018C918E7F8C938F2C9E2C72
:10D04000AD2CBC2C81018BA18F5F8F708BA3FDA2B7
:10D05000E9A6D9AACEAE79CAF10180818160808328
:10D06000C8010E94417F81116FC0D10111966D915D
:10D070007D918D919C9114970E94EFEC6B017C0146
:10D080009B01AC0160E070E080E89FE30E9460EBF0
:10D090002B013C012DEC3CEC4CE45DE30E949DE651
:10D0A00069837A838B839C839401A501C301B201B8
:10D0B0000E949DE6698B7A8B8B8B9C8BAE014F5FB8
:10D0C0005F4FBE016F5E7F4FC1010E9447B8F10103
:10D0D000E95BFF4F80818823B9F12091E706309109
:10D0E000E8064091E9065091EA0637966081718121
:10D0F000828193810E949DE62091A2103091A3101D
:10D100004091A4105091A5100E949DE64B015C0136
:10D110009B01AC01C701B6010E949DE60E94CDEBC8
:10D12000F101E65BFF4F718360832DEC3CEC4CE436
:10D130005DE3C501B4010E949DE60E94CDEBF101C3
:10D14000E45BFF4F71836083F10180818E7F808378
:10D1500004CA28E6269DF001279DF00D1124ED5804
:10D16000FE4E808181FD43C0C114D10441F0D6013F
:10D170001596CD90DD90ED90FC90189708C08BE04F
:10D18000C82E87EDD82E83E2E82E8BE3F82EB8E682
:10D19000B69DF001B79DF00D1124ED58FE4E81892A
:10D1A0009289A389B489BC01CD0190589B01AC013F
:10D1B0000E9484EAF80125853685478550890E94BA
:10D1C0009DE69B01AC01C701B6010E9483EAE62EF1
:10D1D000872E982EA92E262F372F482F592F6DA531
:10D1E0007DA189A599A90E9438E687FF04C0EDA416
:10D1F0008DA099A4A9A82E2D382D492D5A2DC201F4
:10D20000B1010E9438E6882309F427CEF8E6F69D9E
:10D21000C001F79D900D11249C012D583E4E6901CF
:10D22000D9018C9181608C93C8010E94417F882331
:10D2300029F0F60180818E7F80830FCE8E2D982D70
:10D24000A92DBA2DF60185839683A783B08705CED5
:10D25000D6018C9181FD52C0D60115962D913D913C
:10D260004D915C9118972DA73EA74FA758AB15017C
:10D27000B5E02B0E311CF801458056806780708424
:10D28000A30192016DA57EA58FA598A90E9438E6FD
:10D2900087FF34C0F60181899289A389B489BC01D2
:10D2A000CD0190589B01AC010E9484EAD6011D96E5
:10D2B0002D913D914D915C9150970E949DE69B016F
:10D2C000AC016DA57EA58FA598A90E9483EA6B018C
:10D2D0007C019B01AC01C301B2010E94AAEC1816AB
:10D2E0006CF4D8018C9181608C93C5010E94417FC0
:10D2F0008823E1F0F80180818E7F808318E6189DF5
:10D30000F001199DF00D1124ED58FE4E2185328556
:10D310004385548565817681878190850E9438E6B2
:10D320008111D2CD0BA10093B609CECDD101CD9202
:10D33000DD92ED92FC9213970BA10093B609DECF1C
:10D34000C858DF4F0FB6F894DEBF0FBECDBFDF91D8
:10D35000CF911F910F91FF90EF90DF90CF90BF90F2
:10D36000AF909F908F907F906F905F904F903F9085
:10D370002F9008958091B7099091B809891B8F70FB
:10D380008F3019F40E94FCA0F5CF8091B7098F5F10
:10D390008F70E091B70998E69E9FF0011124ED5837
:10D3A000FE4EDF011D929A95E9F798E09083409137
:10D3B000DD095091DE096091DF097091E009458B2C
:10D3C000568B678B708F4091E1095091E209609113
:10D3D000E3097091E409418F528F638F748F4091FC
:10D3E000E5095091E6096091E7097091E809458FD8
:10D3F000568F678F70A34091E9095091EA096091B7
:10D40000EB097091EC0941A352A363A374A320918B
:10D41000B7099091B809291303C094E69093B40911
:10D420008093B70980916F00826080936F000895A8
:10D430009091B7098091B809981306C080914E0762
:10D4400090914F07892B19F00E94FCA0F1CF08950D
:10D45000CF93DF938B3D9240B1F0EDEDFDE18491F0
:10D46000EF012196882321F00E94C689FE01F7CFA3
:10D47000E4EEF9E18491EF012196882331F00E94D6
:10D48000C689FE01F7CF80E001C081E0DF91CF9136
:10D4900008952F923F924F925F926F927F928F9258
:10D4A0009F92AF92BF92CF92DF92EF92FF920F9333
:10D4B0001F93CF93DF93CDB7DEB7C757D1090FB610
:10D4C000F894DEBF0FBECDBF2DB63EB6A7961FAEF9
:10D4D0001EAEA79784E690E0A9969FAF8EAFA9975E
:10D4E00001E09E012B593F4F44E050E0BE01655AD8
:10D4F0007F4FCE0189599F4F0E94F3CF9E012B5938
:10D500003F4F42E050E0BE0167597F4FCE0189593D
:10D510009F4F0E94F3CF43E050E0BE01655A7F4F1A
:10D520008FED92E00E94EFED892B09F43FC06F96DA
:10D530008FAD6F97882339F08FE36C968FAF6C9720
:10D540006D961FAE6D97E2EFFDE184917F012FEFA5
:10D55000E21AF20A811103C0E7EAFAE104C00E946C
:10D56000C689F701F2CF84917F013FEFE31AF30AF6
:10D57000882321F00E94C689F701F5CFBE01655AC4
:10D580007F4F8EE99AE10E9468C5E0E9FAE1849153
:10D590007F019FEFE91AF90A882321F00E94C689CA
:10D5A000F701F5CF81E080931A0754C5EDB7FEB7B8
:10D5B000E696FFAFEEAFE6976B961CAE1DAE1EAEC5
:10D5C0001FAE6B97A7961FAE1EAEA79701E09E01F8
:10D5D0002B593F4F41E050E0BE0160597F4FCE01D3
:10D5E00089599F4F0E94F3CF80E1EBE5F2E0DE0125
:10D5F000919601900D928A95E1F780E1EBE6F2E0D9
:10D60000DE01519601900D928A95E1F780E1EBE7FA
:10D61000F2E0DE01119601900D928A95E1F7E19614
:10D620004FADE19750E04D5F5F4F440F551F440FE2
:10D63000551F2DB73EB7241B350B0FB6F8943EBFD0
:10D640000FBE2DBF8DB79EB701967C0100E09E01F5
:10D650002B593F4FBC01CE0189599F4F0E94F3CFF8
:10D660009E012B593F4F44E050E067E077E0CE0148
:10D6700089599F4F0E94F3CFE1968FACE197912C8F
:10D6800093E0890E911C880C991C880C991CEDB7AD
:10D69000FEB7E819F9090FB6F894FEBF0FBEEDBF4B
:10D6A0002DB73EB72F5F3F4F69018DB79EB78819E1
:10D6B00099090FB6F8949EBF0FBE8DBFEDB7FEB7A8
:10D6C00031965F019E012B593F4FA401B601CE0157
:10D6D00089599F4F0E94F3CF9E012B593F4FA401C0
:10D6E000B501CE0189599F4F0E94F3CF10911B07BE
:10D6F000112309F4A7C000E09E012B593F4F44E0DD
:10D7000050E06FEE76E0CE0189599F4F0E94F3CF33
:10D710009E012B593F4F44E050E063EF76E0CE018D
:10D7200089599F4F0E94F3CF9E012B593F4F44E0F0
:10D7300050E06BEE76E0CE0189599F4F0E94F3CF07
:10D740009E012B593F4F44E050E06FE077E0CE015F
:10D7500089599F4F0E94F3CF9E012B593F4F44E0C0
:10D7600050E06BE077E0CE0189599F4F0E94F3CFE4
:10D770009E012B593F4F40E150E067ED76E0CE012E
:10D7800089599F4F0E94F3CF9E012B593F4F44E090
:10D7900050E0BE01695A7F4FCE0189599F4F0E94C8
:10D7A000F3CF9E012B593F4F4CE050E06CE375E006
:10D7B000CE0189599F4F0E94F3CF9E012B593F4FB5
:10D7C00044E050E067E371E1CE0189599F4F0E9428
:10D7D000F3CF9E012B593F4F44E050E0BE01695A00
:10D7E0007F4FCE0189599F4F0E94F3CF01E09E01E8
:10D7F0002B593F4F41E050E0BE0161597F4FCE01B0
:10D8000089599F4F0E94F3CF9E012B593F4F41E012
:10D8100050E0BE0162597F4FCE0189599F4F0E944F
:10D82000F3CF11118AC06B968CAD9DADAEADBFAD7F
:10D830006B978093C6109093C710A093C810B093B5
:10D84000C9107BC0E1968FADE19790E0029627EF7B
:10D8500036E0E4963FAF2EAFE497B501DE011196B6
:10D86000E6E98E2EE0E19E2EAE014F5E5F4FF3E5BE
:10D87000AF2EF1E1BF2EE896FFAEEEAEE8977E0147
:10D8800031E2E30EF11C20E030E0821793072CF028
:10D89000E896EEADFFADE89701C0F70140805180FA
:10D8A00062807380F50141925192619271925F01A1
:10D8B0008217930714F0F60101C0FA0140805180ED
:10D8C00062807380F40141925192619271924F0192
:10D8D0008217930734F0FB0140805180628073808F
:10D8E00005C04D905D906D907C901397E496EEADE1
:10D8F000FFADE4974192519261927192E496FFAF2D
:10D90000EEAFE4972F5F3F4F6C5F7F4F1496F4E0CC
:10D91000CF0ED11C4C5F5F4FE896EEADFFADE897A0
:10D920003496E896FFAFEEAFE897F4E0EF0EF11C07
:10D930002430310509F0A9CFDECEE0968FADE09717
:10D94000853099F4AF968FADAF97853071F400E0D4
:10D950009E012B593F4F44E650E06AEC70E1CE0146
:10D9600089599F4F0E94F3CF24C0111102C00E9419
:10D97000AFBDE0968FADE097AF96CFACAF978C9DE3
:10D9800060011124E12CF12CEC14FD0491F000E075
:10D990009E012B593F4F44E050E0BE01695A7F4F32
:10D9A000CE0189599F4F0E94F3CF2FEFE21AF20A5E
:10D9B000EBCF00E09E012B593F4F44E050E0BE0109
:10D9C0006D5A7F4FCE0189599F4F0E94F3CF1AE0C5
:10D9D000115079F000E09E012B593F4F44E050E098
:10D9E000BE01695A7F4FCE0189599F4F0E94F3CFE4
:10D9F000EFCF01E09E012B593F4F41E050E0BE01C7
:10DA000063597F4FCE0189599F4F0E94F3CF9E01EA
:10DA10002B593F4F41E050E0BE0164597F4FCE018A
:10DA200089599F4F0E94F3CF00E09E012B593F4F31
:10DA300044E050E0BE01635C7F4FCE0189599F4FA7
:10DA40000E94F3CF9E012B593F4F44E050E0BE01AE
:10DA50006F5C7F4FCE0189599F4F0E94F3CFAE96E6
:10DA60008FADAE97AD96CFACAD978C9D6001112474
:10DA7000E12CF12C00E09E012B593F4FCE14DF0426
:10DA800071F044E050E0BE01695A7F4FCE018959E0
:10DA90009F4F0E94F3CF3FEFE31AF30AEBCF41E031
:10DAA00050E0BE016F587F4FCE0189599F4F0E94B1
:10DAB000F3CF9E012B593F4F41E050E0BE01655925
:10DAC0007F4FCE0189599F4F0E94F3CF9E012B5962
:10DAD0003F4F44E050E0BE01695A7F4FCE01895963
:10DAE0009F4F0E94F3CF9E012B593F4F44E050E0DF
:10DAF000BE01695A7F4FCE0189599F4F0E94F3CFD3
:10DB00009E012B593F4F44E050E06BE371E1CE01A1
:10DB100089599F4F0E94F3CF9E012B593F4F44E0FC
:10DB200050E0BE01615B7F4FCE0189599F4F0E943B
:10DB3000F3CF9E012B593F4F44E050E0BE01655B9F
:10DB40007F4FCE0189599F4F0E94F3CF9E012B59E1
:10DB50003F4F44E050E0BE01695B7F4FCE018959E1
:10DB60009F4F0E94F3CF10E000E09E012B593F4FE2
:10DB700044E050E0BE01695A7F4FCE0189599F4F62
:10DB80000E94F3CF111110C06B96CCACDDACEEACA3
:10DB9000FFAC6B9720E030E84BE355E4C701B601DA
:10DBA0000E9438E6811103C054E0F52E33C0809105
:10DBB0001B07811108C0C0924007D0924107E09234
:10DBC0004207F092430700E09E012B593F4F44E08B
:10DBD00050E06CE377E0CE0189599F4F0E94F3CF6C
:10DBE0009E012B593F4F44E050E064E477E0CE01C2
:10DBF00089599F4F0E94F3CF9E012B593F4F44E01C
:10DC000050E0BE01695A7F4FCE0189599F4F0E9453
:10DC1000F3CF12C0FA94FF2079F000E09E012B5957
:10DC20003F4F44E050E0BE01695A7F4FCE01895911
:10DC30009F4F0E94F3CFEECF1F5F153009F094CFB6
:10DC400000E09E012B593F4F42E050E0BE016D596C
:10DC50007F4FCE0189599F4F0E94F3CF9E012B59D0
:10DC60003F4F44E050E0BE01695A7F4FCE018959D1
:10DC70009F4F0E94F3CF6B96CCACDDACEEACFFAC0B
:10DC80006B9720E030E84BE355E4C701B6010E94F2
:10DC900038E6882329F180911B07811108C0C092C2
:10DCA0003807D0923907E0923A07F0923B0700E03C
:10DCB0009E012B593F4F44E050E064E377E0CE01F2
:10DCC00089599F4F0E94F3CF9E012B593F4F44E04B
:10DCD00050E060E377E0CE0189599F4F0E94F3CF77
:10DCE00000E09E012B593F4F42E050E0BE016F59CA
:10DCF0007F4FCE0189599F4F0E94F3CF9E012B5930
:10DD00003F4F41E050E0BE016F587F4FCE0189592F
:10DD10009F4F0E94F3CF19E0115000E09E012B5954
:10DD20003F4F112359F044E050E0BE01695A7F4F44
:10DD3000CE0189599F4F0E94F3CFEECF41E050E0D2
:10DD40006EE271E1CE0189599F4F0E94F3CFF12C11
:10DD500000E09E012B593F4F44E050E0BE01695A5C
:10DD60007F4FCE0189599F4F0E94F3CF10911B071F
:10DD7000111110C0F1100EC06B968CAD9DADAEAD03
:10DD8000BFAD6B978093331190933411A0933511ED
:10DD9000B0933611F39485E0F812DACF111102C076
:10DDA0000E94B3C44CE0F42EFA94F11003C03CE09E
:10DDB000F32E0FC000E09E012B593F4F42E050E090
:10DDC000BE01615A7F4FCE0189599F4F0E94F3CF08
:10DDD000EBCFFA9400E09E012B593F4FFF2059F002
:10DDE00044E050E0BE016D5B7F4FCE0189599F4FEB
:10DDF0000E94F3CFEECF46E050E0BE01635C7F4F60
:10DE0000CE0189599F4F0E94F3CF9E012B593F4F5E
:10DE100044E050E067EE76E0CE0189599F4F0E94C2
:10DE2000F3CF9E012B593F4F4CE050E0BE016F5C99
:10DE30007F4FCE0189599F4F0E94F3CF2CE1F22EE4
:10DE4000FA94F11003C094E0F92E1DC000E09E0189
:10DE50002B593F4F44E050E0BE01695A7F4FCE013D
:10DE600089599F4F0E94F3CFEBCF00E09E012B59C1
:10DE70003F4F44E050E0BE01695A7F4FCE018959BF
:10DE80009F4F0E94F3CFFA94F110EFCF8BE0F82E62
:10DE9000FA94FF2079F000E09E012B593F4F44E0B7
:10DEA00050E0BE01695A7F4FCE0189599F4F0E94B1
:10DEB000F3CFEECFA9968EAD9FADA9978456910969
:10DEC000C7DA80931A07882309F1E2EFFDE1849114
:10DED0007F019FEFE91AF90A882321F00E94C68981
:10DEE000F701F5CFA9966EAD7FADA997645671097C
:10DEF00088E89AE10E944FC56BED72E080E89AE1F4
:10DF00000E944FC58AE00E94C68999C0A7962EAD8F
:10DF10003FADA797AB968EAD9FADAB97281739074E
:10DF200009F44BC081E080931A07EDEDFDE1849187
:10DF30007F012FEFE21AF20A811103C0E0E6FAE155
:10DF400004C00E94C689F701F2CF84917F013FEFA0
:10DF5000E31AF30A882321F00E94C689F701F5CF5E
:10DF6000AB966EAD7FADAB9780E090E04AE00E944B
:10DF7000E98CEBE5FAE184917F019FEFE91AF90A58
:10DF8000882321F00E94C689F701F5CFA7966EADD0
:10DF90007FADA79780E090E04AE00E94E98CEBE437
:10DFA000FAE184917F012FEFE21AF20A882309F443
:10DFB00046C00E94C689F701F4CF111142C0E2EFBA
:10DFC000FDE184917F013FEFE31AF30A811103C061
:10DFD0000FED12E004C00E94C689F701F2CFF801EC
:10DFE00081918F01882319F00E94C689F8CFA996E4
:10DFF0006EAD7FADA997645671098EE29AE10E94D9
:10E000004FC5A7964EAD5FADA79760E070E081E287
:10E010009AE10E9415C5EEE1FAE184917F012FEFAC
:10E02000E21AF20A811107C080911A07811109C012
:10E030000E94B4D006C00E94C689F701EECF11231A
:10E0400099F3E6968EAD9FADE6970FB6F8949EBF16
:10E050000FBE8DBF80911B07811102C00E947CBE44
:10E0600090911A0781E089270FB6F8943EBE0FBE43
:10E070002DBEC958DF4F0FB6F894DEBF0FBECDBF1F
:10E08000DF91CF911F910F91FF90EF90DF90CF9094
:10E09000BF90AF909F908F907F906F905F904F90C8
:10E0A0003F902F90089581E080931B07F2D9109242
:10E0B0001B078111EEC90E94EBC281E008958F9287
:10E0C0009F92AF92BF92CF92DF92EF92FF920F9307
:10E0D0001F93CF93DF93CDB7DEB7CA5AD1090FB6DE
:10E0E000F894DEBF0FBECDBFE9961CAE1DAE1EAECE
:10E0F0001FAEE9978091F1039091F203A091F30391
:10E10000B091F403ED968CAF9DAFAEAFBFAFED977E
:10E11000C556DF4F19821882CB59D04084E690E073
:10E12000C356DF4F99838883CD59D04010921A0788
:10E130009E0125563F4F44E050E0BE0167587F4F97
:10E14000CE0183569F4F0E9440D0C356DF4F888137
:10E150009981CD59D0400296C356DF4F9983888369
:10E16000CD59D040C556DF4F19821882CB59D040C7
:10E1700081E0CD55DF4F8883C35AD0409E0125569C
:10E180003F4F41E050E0BE016D557F4FCE018356B9
:10E190009F4F0E9440D09E0125563F4F40E150E0E6
:10E1A00063E571E1CE0183569F4F0E9440D09E01EE
:10E1B00025563F4F44E050E067E077E0CE018356BC
:10E1C0009F4F0E9440D09E0125563F4F40E150E0B6
:10E1D00066E970E1CE0183569F4F0E9440D09E01B8
:10E1E00025563F4F40E150E067EF76E0CE01835681
:10E1F0009F4F0E9440D09E0125563F4F44E050E083
:10E200006FEE76E0CE0183569F4F0E9440D09E0174
:10E2100025563F4F44E050E063EF76E0CE01835651
:10E220009F4F0E9440D09E0125563F4F44E050E052
:10E230006BEE76E0CE0183569F4F0E9440D09E0148
:10E2400025563F4F44E050E06FE077E0CE01835623
:10E250009F4F0E9440D09E0125563F4F44E050E022
:10E260006BE077E0CE0183569F4F0E9440D09E0125
:10E2700025563F4F40E150E067ED76E0CE018356F2
:10E280009F4F0E9440D08AE097EDA3EABCE3E99655
:10E290008CAF9DAFAEAFBFAFE9979E0125563F4F04
:10E2A00044E050E0BE016B587F4FCE0183569F4F34
:10E2B0000E9440D09E0125563F4F4CE050E06CE359
:10E2C00075E0CE0183569F4F0E9440D0809181100F
:10E2D00090918210A0918310B0918410C358DF4FA9
:10E2E00088839983AA83BB83CD57D0409E0125564E
:10E2F0003F4F44E050E0BE0163587F4FCE0183564C
:10E300009F4F0E9440D085E0CC55DF4F8883C45A90
:10E31000D040CB55DF4F8883C55AD0409E0125564B
:10E320003F4F44E050E066EC70E1CE0183569F4FD2
:10E330000E9440D09E0125563F4F41E050E0BE0173
:10E340006C557F4FCE0183569F4F0E9440D09E0157
:10E3500025563F4F41E050E0BE016B557F4FCE0147
:10E3600083569F4F0E9440D09E0125563F4F44E662
:10E3700050E06AEC70E1CE0183569F4F0E9440D07E
:10E38000CF57DF4F188219821A821B82C158D040A2
:10E390009E0125563F4F44E050E0BE016F577F4F2E
:10E3A000CE0183569F4F0E9440D0E9961CAE1DAE11
:10E3B0001EAE1FAEE9971AE0115071F09E0125566E
:10E3C0003F4F44E050E0BE016B587F4FCE01835673
:10E3D0009F4F0E9440D0F0CF83E0CA55DF4F888323
:10E3E000C65AD040C955DF4F8883C75AD040CB5753
:10E3F000DF4F188219821A821B82C558D040C75736
:10E40000DF4F188219821A821B82C958D040E996C0
:10E410001CAE1DAE1EAE1FAEE9979E0125563F4FA6
:10E4200041E050E0BE016A557F4FCE0183569F4FB9
:10E430000E9440D09E0125563F4F41E050E0BE0172
:10E4400069557F4FCE0183569F4F0E9440D09E0159
:10E4500025563F4F44E050E0BE0167577F4FCE0145
:10E4600083569F4F0E9440D09E0125563F4F44E067
:10E4700050E0BE016B577F4FCE0183569F4F0E94E5
:10E4800040D00AE010E00150110971F09E012556BC
:10E490003F4F44E050E0BE016B587F4FCE018356A2
:10E4A0009F4F0E9440D0EFCFC855DF4F1882C85A07
:10E4B000D0408FEFC755DF4F8883C95AD0409E01A7
:10E4C00025563F4F41E050E0BE0168557F4FCE01D9
:10E4D00083569F4F0E9440D09E0125563F4F41E0FA
:10E4E00050E0BE0167557F4FCE0183569F4F0E947B
:10E4F00040D0E9961CAE1DAE1EAE1FAEE9979E0140
:10E5000025563F4F44E050E0BE016B587F4FCE018F
:10E5100083569F4F0E9440D09E0125563F4F44E0B6
:10E5200050E0BE016B587F4FCE0183569F4F0E9433
:10E5300040D09E0125563F4F44E050E06BE371E12F
:10E54000CE0183569F4F0E9440D080918B029091C4
:10E550008C02A0918D02B0918E02C357DF4F888349
:10E560009983AA83BB83CD58D04080918F0290912C
:10E570009002A0919102B0919202CF56DF4F888312
:10E580009983AA83BB83C159D040CB56DF4F1982F0
:10E590001882C559D040C956DF4F19821882C75911
:10E5A000D0409E0125563F4F44E050E0BE016357E6
:10E5B0007F4FCE0183569F4F0E9440D09E0125562B
:10E5C0003F4F44E050E0BE016F567F4FCE0183566F
:10E5D0009F4F0E9440D09E0125563F4F44E050E09F
:10E5E000BE016B567F4FCE0183569F4F0E9440D095
:10E5F00010E0C12C80E8D82E8BE3E82E85E4F82EBD
:10E60000812C912C90E8A92E9FE3B92E111138C0CE
:10E610009E0125563F4F44E050E060E477E0CE0194
:10E6200083569F4F0E9440D09E0125563F4F44E0A5
:10E6300050E06CE377E0CE0183569F4F0E9440D0BC
:10E640009E0125563F4F44E050E064E477E0CE0160
:10E6500083569F4F0E9440D0E9968CAE9DAEAEAEE1
:10E66000BFAEE9979E0125563F4F44E050E0BE0102
:10E670006B587F4FCE0183569F4F0E9440D02AC0D7
:10E68000E996CCAEDDAEEEAEFFAEE9979E01255623
:10E690003F4F44E050E0BE016B587F4FCE018356A0
:10E6A0009F4F0E9440D0E9961CAE1DAE1EAE1FAE1D
:10E6B000E99704E0015071F09E0125563F4F44E078
:10E6C00050E0BE016B587F4FCE0183569F4F0E9492
:10E6D00040D0F0CF1F5F153009F098CF84E190E073
:10E6E000C156DF4F99838883CF59D0409E0125566C
:10E6F0003F4F42E050E0BE0161567F4FCE0183564E
:10E700009F4F0E9440D09E0125563F4F44E050E06D
:10E7100068E377E0CE0183569F4F0E9440D09E0170
:10E7200025563F4F44E050E064E377E0CE01835646
:10E730009F4F0E9440D09E0125563F4F44E050E03D
:10E7400060E377E0CE0183569F4F0E9440D080E285
:10E7500090E0CF55DF4F99838883C15AD0409E0106
:10E7600025563F4F42E050E0BE016F557F4FCE012E
:10E7700083569F4F0E9440D0C655DF4F1882CA5A19
:10E78000D04080E2E3E9F2E0DE019D9601900D9237
:10E790008A95E1F79E0125563F4F41E050E0BE01CA
:10E7A00066557F4FCE0183569F4F0E9440D09E01F9
:10E7B00025563F4F40E250E0BE01635D7F4FCE01E2
:10E7C00083569F4F0E9440D09E0125563F4F41E007
:10E7D00050E06EE271E1CE0183569F4F0E9440D01F
:10E7E00010E011110EC08091331190913411A0915D
:10E7F0003511B0913611E9968CAF9DAFAEAFBFAF7A
:10E80000E9979E0125563F4F44E050E0BE016B580A
:10E810007F4FCE0183569F4F0E9440D01F5F15301F
:10E8200001F7BE01635B7F4F86E1FB0111928A9580
:10E83000E9F79E0125563F4F46E150E0CE01835651
:10E840009F4F0E9440D08CE2E3EBF2E0DE01119694
:10E8500001900D928A95E1F79E0125563F4F4CE2BB
:10E8600050E0BE016F5F7F4FCE0183569F4F0E94E5
:10E8700040D0BE0161597F4F86E0FB0111928A951D
:10E88000E9F79E0125563F4F46E050E0CE01835602
:10E890009F4F0E9440D09E0125563F4F44E050E0DC
:10E8A00067EE76E0CE0183569F4F0E9440D0BE01B6
:10E8B0006D597F4F8CE0FB0111928A95E9F79E011B
:10E8C00025563F4F4CE050E0CE0183569F4F0E94AB
:10E8D00040D0E9961CAE1DAE1EAE1FAEE9971CE1FE
:10E8E000115071F09E0125563F4F44E050E0BE01AB
:10E8F0006B587F4FCE0183569F4F0E9440D0F0CF80
:10E90000E9961CAE1DAE1EAE1FAEE99714E0115085
:10E9100071F09E0125563F4F44E050E0BE016B5818
:10E920007F4FCE0183569F4F0E9440D0F0CFE99693
:10E930001CAE1DAE1EAE1FAEE9971BE0115071F06C
:10E940009E0125563F4F44E050E0BE016B587F4F7B
:10E95000CE0183569F4F0E9440D0F0CF80911A077E
:10E96000811167C0C356DF4FE880F980CD59D04090
:10E97000F4E6EF1AF108C556DF4F88819981CB592B
:10E98000D040C756DF4F99838883C959D04084E669
:10E9900090E0C356DF4F99838883CD59D0409E01C4
:10E9A00025563F4F44E050E06FED72E0CE018356B4
:10E9B0009F4F0E9440D09E0125563F4F42E050E0BD
:10E9C000BE0167567F4FCE0183569F4F0E9440D0B5
:10E9D000E2EFFDE184918F010F5F1F4F882321F04B
:10E9E0000E94C689F801F6CFB7018CE09AE10E9437
:10E9F0004FC5C756DF4F48815981C959D04060E0A3
:10EA000070E08FEF99E10E9415C5ECEFF9E1849178
:10EA10008F010F5F1F4F882321F00E94C689F801E4
:10EA2000F6CFC7010E94286A90911A07892B80931C
:10EA30001A0790911A0781E08927C655DF4F0FB654
:10EA4000F894DEBF0FBECDBFDF91CF911F910F9124
:10EA5000FF90EF90DF90CF90BF90AF909F908F90FE
:10EA60000895FF920F931F93CF93DF938C01EB01D7
:10EA7000F42E80E20E94C6898FEFF81611F084E52B
:10EA800001C082E40E94C6898AE30E94C689F80117
:10EA9000608171818281938142E00E946E8D488104
:10EAA00059816A817B818BE59DE10E9432C562E0DC
:10EAB00070E080E090E0DF91CF911F910F91FF9087
:10EAC0000C940AB78F929F92AF92BF92CF92DF922F
:10EAD000EF92FF920F931F93CF93DF93F0E2FF2EFD
:10EAE000E12CAE2DB0E0BD016F0D711D75956795E0
:10EAF0006E1511F0F6120BC0EEE3FBE16591749117
:10EB0000072E000C880B990B0E943EE662C09B0109
:10EB100021503109220F331F220F331FF901E05416
:10EB2000F54E05911491AB01440F551F440F551F2D
:10EB3000FA01E054F54EC591D4918017910714F471
:10EB4000F62ED1CFC817D90714F4E62ECACFF90193
:10EB5000EE53F54EE590F490FA01EE53F54EC59064
:10EB6000D490BC01601B710B072E000C880B990B15
:10EB70000E943EE64B015C01B6016E197F09072E2B
:10EB8000000C880B990B0E943EE69B01AC01C5016D
:10EB9000B4010E949DE64B015C01C01BD10BBE017C
:10EBA000DD0F880B990B0E943EE69B01AC01C5016D
:10EBB000B4010E9460EB4B015C01B701FF0C880BB4
:10EBC000990B0E943EE69B01AC01C501B4010E9475
:10EBD00084EADF91CF911F910F91FF90EF90DF902A
:10EBE000CF90BF90AF909F908F9008950F931F93F9
:10EBF000CF93DF93CDB7DEB728970FB6F894DEBF7B
:10EC00000FBECDBF60914E0470914F04072E000CD3
:10EC1000880B990B0E943EE66D837E838F839887D5
:10EC20008091500490915104A0915204B0915304EA
:10EC300089839A83AB83BC834DEFBE016B5F7F4FAB
:10EC4000CE0101960EDF6091480470914904072EB1
:10EC5000000C880B990B0E943EE66D837E838F83A8
:10EC6000988780914A0490914B04A0914C04B091F4
:10EC70004D0489839A83AB83BC834FEFBE016B5FE6
:10EC80007F4FCE010196EDDEE3E6FDE184918F0139
:10EC90000F5F1F4F882321F00E94C689F801F6CF2D
:10ECA000E0915207F0E0E05BF84F608170E080E0B7
:10ECB00090E00E94548DEEE5FDE184918F010F5F9D
:10ECC0001F4F882321F00E94C689F801F6CF60917A
:10ECD000510770E080E090E00E94548D28960FB6B6
:10ECE000F894DEBF0FBECDBFDF91CF911F910F9182
:10ECF00008950F930FB70F9300916E000B7F009351
:10ED00006E0078940F930BB70F930CB70F921F926E
:10ED10002F933F934F935F936F937F938F939F9323
:10ED2000AF93BF93EF93FF931124EFD2FF91EF9135
:10ED3000BF91AF919F918F917F916F915F914F9113
:10ED40003F912F911F900F900CBF0F910BBF0F9110
:10ED50000460F89400936E000F910FBF0F91189507
:10ED6000CF92DF92EF92FF92C0904A04D0904B0472
:10ED7000E0904C04F0904D04609148047091490477
:10ED800066507109072E000C880B990B0E943EE615
:10ED90009B01AC01C701B6010E9438E687FF1FC086
:10EDA00020E030E040E050E4C701B6010E9484EA70
:10EDB0000E94CDEB70938A07609389070E94F858F0
:10EDC000DC01CB01805A9541AF4FBF4F809385073F
:10EDD00090938607A0938707B093880708C0109286
:10EDE0008507109286071092870710928807FF9078
:10EDF000EF90DF90CF900895CF92DF92EF92FF9245
:10EE0000C0905004D0905104E0905204F09053040C
:10EE100060914E0470914F0467507109072E000CE9
:10EE2000880B990B0E943EE69B01AC01C701B6011D
:10EE30000E9438E687FF1FC020E030E040E450E445
:10EE4000C701B6010E9484EA0E94CDEB709384074B
:10EE5000609383070E94F858DC01CB01805A9541EA
:10EE6000AF4FBF4F80937F0790938007A093810798
:10EE7000B093820708C010927F071092800710920B
:10EE8000810710928207FF90EF90DF90CF90089556
:10EE90008F929F92AF92BF92CF92DF92EF92FF92AA
:10EEA0000F931F93CF93DF93F0E4FF2EE12CAE2D51
:10EEB000B0E0BD016F0D711D759567956E1511F070
:10EEC000F6120BC0E0EBFCE165917491072E000C8B
:10EED000880B990B0E943EE662C09B0121503109CC
:10EEE000220F331F220F331FF901EE54F44E059108
:10EEF0001491AB01440F551F440F551FFA01EE54F6
:10EF0000F44EC591D4918017910714F4F62ED1CF09
:10EF1000C817D90714F4E62ECACFF901EC54F44E01
:10EF2000E590F490FA01EC54F44EC590D490BC01F5
:10EF3000601B710B072E000C880B990B0E943EE69C
:10EF40004B015C01B6016E197F09072E000C880B7E
:10EF5000990B0E943EE69B01AC01C501B4010E94E1
:10EF60009DE64B015C01C01BD10BBE01DD0F880B80
:10EF7000990B0E943EE69B01AC01C501B4010E94C1
:10EF800060EB4B015C01B701FF0C880B990B0E94F1
:10EF90003EE69B01AC01C501B4010E9484EADF9109
:10EFA000CF911F910F91FF90EF90DF90CF90BF9086
:10EFB000AF909F908F90089560E080919507909119
:10EFC000960780DD6093500470935104809352043F
:10EFD00090935304809193079091940759DF609325
:10EFE0004A0470934B0480934C0490934D04A8956D
:10EFF00010924D0708957F928F929F92AF92BF9289
:10F00000CF92DF92EF92FF920F931F93CF93DF93F4
:10F0100020E030E048E452E46091500470915104E3
:10F0200080915204909153040E94AAEC18164CF45B
:10F03000E6E4FBE1E491C1E001C0CC0FEA95EAF718
:10F0400001C0C0E080E4E82E8BE1F82E06E41BE16D
:10F0500096E0A92E912CD0E0CC24C394D12CF701BA
:10F060007490F801849077FC23C0892D90E0082CDF
:10F0700002C0959587950A94E2F780FD19C0BE01FC
:10F08000082C02C0759567950A94E2F76170B62E58
:10F09000B1946B2D872D0E94D9B56B2D70E0872D13
:10F0A0000E9443B6C60101C0880F8A94EAF7982AE5
:10F0B000AA94FFEFEF1AFF0A0F5F1F4FA110CFCFE7
:10F0C000DF91CF911F910F91FF90EF90DF90CF9044
:10F0D000BF90AF909F908F907F9008950F931F9354
:10F0E00080912F07813019F40E94F85808C0609170
:10F0F0002B0770912C0780912D0790912E0700917E
:10F100005707109158072091590730915A07601BF3
:10F11000710B820B930B28EE33E040E050E00E942D
:10F1200026EA8091530790915407A0915507B0911A
:10F130005607BC01CD01620F731F841F951F1F91DD
:10F140000F91089510922F071092570710925807A9
:10F150001092590710925A0710922B0710922C0701
:10F1600010922D0710922E071092530710925407F9
:10F170001092550710925607089580912F078130FD
:10F18000E1F0823051F4AADF609353077093540783
:10F19000809355079093560701C0D4DF81E0809398
:10F1A0002F070E94F8586093570770935807809371
:10F1B000590790935A0781E0089580E0089580915F
:10F1C0002F07813079F482E080932F070E94F8584E
:10F1D00060932B0770932C0780932D0790932E0735
:10F1E00081E0089580E0089580912F07815082305A
:10F1F00010F080E0089510922F070E94F858609355
:10F200002B0770932C0780932D0790932E0781E096
:10F21000089510924C0780E090E00E94ED59109202
:10F220004904109248049CDDDFDF80E090E00E94FA
:10F23000ED59109250072C981092490410924804EE
:10F24000109251078091020180728093000108950D
:10F25000DF92EF92FF920F931F93CF93DF93F82EDD
:10F26000D62EE72E8A0180912702882309F439C01F
:10F27000EDEDFDE18491EF012196882321F00E94BC
:10F28000C689FE01F7CFED2DFE2D8491EF01219669
:10F29000882321F00E94C689FE01F7CFE1E5FBE15A
:10F2A0008491EF012196882321F00E94C689FE01F6
:10F2B000F7CFF7FC0BC06F2DFF0C770B880B990B6A
:10F2C0000E94548D8AE00E94C6890BC0ECE4FBE1E9
:10F2D0008491EF012196882321F00E94C689FE01C6
:10F2E000F7CF80915B07811108C01092270281E05F
:10F2F00080935B07C8010E94B5A0DF91CF911F9159
:10F300000F91FF90EF90DF9084CFEF92FF920F93D9
:10F310001F93CF93DF9380912A028F37A0F08F57EE
:10F32000909150079093A607992311F02C9A01C051
:10F330002C98209151072093A50790910201222338
:10F3400069F090950BC09091A607891708F02C984A
:10F350009091A507891728F09091020190729093DF
:10F3600000018F5F80932A029091A40781E0892792
:10F370008093A4078091290285301CF4C1E0C80F56
:10F3800001C0C0E0823009F4B4C054F4882301F114
:10F39000813009F0E3C088E080937B0085E4C0C041
:10F3A000843009F4C5C00CF4B7C0853009F0D6C06C
:10F3B0009091A307911102C08093A3078091A307A6
:10F3C00081508093A307882309F4C8C0C5E0C6C054
:10F3D000809128028F5F80311CF480932802BEC088
:10F3E0001092280280914D07811113C080919907D6
:10F3F00090919A079093960780939507809197072D
:10F4000090919807909394078093930781E080935D
:10F410004D078AE0E9E9F7E0DF011D928A95E9F7F7
:10F4200010929807109297070091950710919607F0
:10F4300011950195110980914E0490914F04D1E0EE
:10F44000181619062CF080915007811101C0D0E0E8
:10F450008091360590913705919581959109801796
:10F46000910734F449EE5CE16AE07DE180E0F0DE92
:10F4700080911C0290911D02919581959109081728
:10F48000190744F4DD2331F04CE15DE16DE37DE1EA
:10F4900080E0DEDE809148049091490411E0181666
:10F4A00019062CF080915107811101C010E0E09005
:10F4B0009307F090940780913405909135058E154F
:10F4C0009F0534F049EF5CE16AE07DE18FEFC0DE3B
:10F4D00080911A0290911B02E816F9060CF43EC0C6
:10F4E0001123E1F14CE25DE16DE37DE18FEFB0DEF0
:10F4F00035C080917A0086FD2EC080917800909171
:10F5000079002091990730919A07820F931F909369
:10F510009A078093990722C088E080937B0086E455
:10F5200080937C0080917A00806480937A0016C07A
:10F5300080917A0086FD11C08091780090917900C9
:10F540002091970730919807820F931F9093980707
:10F550008093970703C0C2E001C0C4E0C0932902B2
:10F5600080913B0581110E94BFBD80914E07909113
:10F570004F070097A9F0019790934F0780934E078C
:10F58000892B71F48FE49DE19093A8078093A707DE
:10F59000DF91CF911F910F91FF90EF900C94F28922
:10F5A000DF91CF911F910F91FF90EF9008952F92CF
:10F5B0003F924F925F926F927F928F929F92AF9203
:10F5C000BF92CF92DF92EF92FF920F931F93CF9350
:10F5D000DF9300D01F92CDB7DEB75C017A836983D9
:10F5E0004A01170107FD07C0802F002E000C990B60
:10F5F0009C838B8304C0E1E0F0E0FC83EB83F901A2
:10F6000040805180628073808B819C81880F991F1C
:10F61000880F991F9C838B838557984F7C01A3018A
:10F620009201FC0160817181828193810E9438E6A0
:10F63000882391F0F701408251826282738211E047
:10F6400020E030E0A901C301B2010E94AAEC181623
:10F650000CF010E0F5011083F50180818230D1F0CB
:10F66000833009F45EC0813009F07CC0EB81FC81FD
:10F67000E557F84F2081318142815381F401608147
:10F680007181828193810E9438E687FD6BC082E0A0
:10F69000F50180838B819C818557984F9C838B8358
:10F6A000B60180E090E00E943CE69B01AC01EB815A
:10F6B000FC8160817181828193810E9483EA9B0138
:10F6C000AC01F40160817181828193810E94AAEC76
:10F6D00087FD14C00E94F8586B017C019101A8EECF
:10F6E000B3E00E9474EAC60ED71EE81EF91EE98137
:10F6F000FA81C082D182E282F38234C00E94F8583B
:10F70000E981FA81C080D180E280F380DC01CB0105
:10F710008C199D09AE09BF09B7FD24C083E0F5012E
:10F7200080830F3F19F042EB5CE102C045EC5CE1E5
:10F7300069ED7CE1802F0F900F900F900F90DF917B
:10F74000CF911F910F91FF90EF90DF90CF90BF90DE
:10F75000AF909F908F907F906F905F904F903F9071
:10F760002F9076CD0F900F900F900F90DF91CF914B
:10F770001F910F91FF90EF90DF90CF90BF90AF90CF
:10F780009F908F907F906F905F904F903F902F90C1
:10F7900008954F925F926F927F928F929F92AF9255
:10F7A000BF92CF92DF92EF92FF920F931F93CF936E
:10F7B000DF93CDB7DEB760970FB6F894DEBF0FBE0C
:10F7C000CDBF80914D07811117C060960FB6F89498
:10F7D000DEBF0FBECDBFDF91CF911F910F91FF9084
:10F7E000EF90DF90CF90BF90AF909F908F907F90E1
:10F7F0006F905F904F900895DFDB0E94F8584B01A7
:10F800005C0160914E0470914F04072E000C880B30
:10F81000990B0E943EE669837A838B839C8344E143
:10F82000C42ED12C5CE3E52EF12C00E09E012F5F6D
:10F830003F4F40E554E06BE777E08AE797E0B7DEBB
:10F84000C0905004D0905104E0905204F0905304C2
:10F850006091380570913905072E000C880B990BC3
:10F860000E943EE69B01AC01C701B6010E94AAECD2
:10F8700018160CF009C160911E0270911F02072E2C
:10F88000000C880B990B0E943EE69B01AC01C7015E
:10F89000B6010E9438E687FFF7C000914E04109130
:10F8A0004F04B801012E000C880B990B0E943EE614
:10F8B000A70196010E9483EA2B013C0120ED3CEC5C
:10F8C0004CE45DE3609144077091450780914607E1
:10F8D000909147070E949DE66D837E838F83988772
:10F8E000209171073091720740917307509174070E
:10F8F000C701B6010E9483EA9B01AC016D817E8144
:10F900008F8198850E949DE66D837E838F83988783
:10F9100023E333E343E75FE360916D0770916E0784
:10F9200080916F07909170070E949DE69B01AC014A
:10F930006D817E818F8198850E9484EA6D837E83AC
:10F940008F83988760936D0770936E0780936F071E
:10F9500090937007C0927107D0927207E09273077C
:10F96000F092740720E030E040E251E4C301B201BC
:10F970000E94AAEC18160CF431C220E030E040E2FC
:10F9800051ECC301B2010E9438E687FD2FC2012B62
:10F9900009F42CC280916C0781112CC22091680758
:10F9A0003091690740916A0750916B0729873A8720
:10F9B0004B875C8720914007309141074091420777
:10F9C00050914307C301B2010E949DE66B017C0187
:10F9D000A301920169857A858B859C850E9484EAC2
:10F9E00069877A878B879C8760936807709369071C
:10F9F00080936A0790936B0720913C0730913D07F5
:10FA000040913E0750913F070E949DE6A701960155
:10FA10000E9484EA2D813E814F8158850E9483EAAD
:10FA20006B017C0120E030E04FE753E40E94AAEC38
:10FA300020E030E0A90118160CF4E3C1C701B601BB
:10FA40000E9438E687FD07C0C701B6010E94C8EBD7
:10FA5000759567951AC020E030E0A901C301B20195
:10FA60000E9438E687FF10C0A301920169857A855C
:10FA70008B859C850E9483EA609368077093690771
:10FA800080936A0790936B0760E0609350078091C2
:10FA90007F0790918007A0918107B091820700971E
:10FAA000A105B10521F1A5019401281B390B4A0BD1
:10FAB0005B0B57FD1CC0609183077091840780E049
:10FAC00090E00E943CE69B01AC0160915004709173
:10FAD000510480915204909153040E9438E687FFAC
:10FAE00082C141E95BE163EA7BE180E0B1DB8091C7
:10FAF000480790914907A0914A07B0914B07A5018B
:10FB00009401281B390B4A0B5B0B57FD0FC073DAAE
:10FB1000D501C4018C53964FAF4FBF4F8093480718
:10FB200090934907A0934A07B0934B0780918507AC
:10FB300090918607A0918707B09188070097A1054B
:10FB4000B10511F1881A990AAA0ABB0AB7FC1CC0B0
:10FB50006091890770918A0780E090E00E943CE6FE
:10FB60009B01AC0160914A0470914B0480914C045C
:10FB700090914D040E9438E687FF20C14FE65BE17B
:10FB800062E87BE18FEF64DB609148047091490487
:10FB9000072E000C880B990B0E943EE669837A833E
:10FBA0008B839C8395E0C92ED12C24E1E22EF12C8D
:10FBB0000FEF9E012F5F3F4F4AE454E065E777E087
:10FBC00089E797E0F4DCC0904A04D0904B04E090C1
:10FBD0004C04F0904D0420E030E040EA50E4C701CE
:10FBE000B6010E94AAEC87FDE5C020E030E04CEDB4
:10FBF00052E4C701B6010E9438E618160CF4DAC0C8
:10FC00006091480470914904072E000C880B990BF1
:10FC10000E943EE6A70196010E9483EA4B015C0127
:10FC2000209138073091390740913A0750913B07AE
:10FC30000E949DE669877A878B879C87209164075D
:10FC4000309165074091660750916707C501B4017F
:10FC50000E9484EA6D837E838F8398876093640714
:10FC60007093650780936607909367072091340728
:10FC70003091350740913607509137070E949DE635
:10FC80006D877E878F87988B20ED3CEC4CE45DE39D
:10FC9000609130077091310780913207909133075E
:10FCA0000E949DE62B013C01209160073091610785
:10FCB0004091620750916307C701B6010E9483EA31
:10FCC0009B01AC01C301B2010E949DE62B013C01E6
:10FCD00023E333E343E75FE360915C0770915D07E3
:10FCE00080915E0790915F070E949DE69B01AC01A9
:10FCF000C301B2010E9484EA2B013C0160935C07BE
:10FD000070935D0780935E0790935F07C0926007D2
:10FD1000D0926107E0926207F09263072D853E85DD
:10FD20004F85588969857A858B859C850E9484EAF0
:10FD3000A30192010E9483EA6B017C0120E030E084
:10FD40004FE753E40E94AAEC20E030E0A901181626
:10FD5000C4F5C501B4010E94AAEC181684F4A501EB
:10FD600094016D817E818F8198850E9483EA6093E2
:10FD700064077093650780936607909367076FE742
:10FD80001AC020E030E0A901C501B4010E9438E6A4
:10FD900087FF10C0A50194016D817E818F819885B8
:10FDA0000E9483EA609364077093650780936607F7
:10FDB0009093670760E06093510707CD0E94B0768B
:10FDC000E3CEC701B6010E9438E687FDDACFC7014E
:10FDD000B6010E94C8EB75956795EDCF81E08093E1
:10FDE0006C076FE752CE80E007D881CE81E0809328
:10FDF0006C074ACE10926C0719861A861B861C86E1
:10FE0000D9CDC301B2010E94AAEC181654F7A30180
:10FE1000920169857A858B859C850E9483EA60932F
:10FE200068077093690780936A0790936B076FE781
:10FE30002CCE90916F00292F227091FF05C09091D8
:10FE40006F009D7F90936F0034E0839FC001112469
:10FE5000FC01EA57FF4E4081518162817381FC01B0
:10FE6000E15EF84F408351836283738381E0809326
:10FE70001E07222329F080916F00826080936F001B
:10FE80000895BC0120911C0730911D0740911C076B
:10FE900050911D072417350711F09A01F7CF81E023
:10FEA0002617370709F080E008958F929F92AF924E
:10FEB000BF92CF92DF92EF92FF921F93CF93DF9387
:10FEC000C82F87ED9BE09093B3098093B2091092FD
:10FED000F30B82E090E0A0E0B0E08093DC0B909325
:10FEE000DD0BA093DE0BB093DF0B1092B1091092E3
:10FEF000AD091092AE091092AF091092B0098FEFC0
:10FF00009FEFDC018093A9099093AA09A093AB0904
:10FF1000B093AC09CC2379F1C53008F0F8C040E0CB
:10FF200060E070E0CB010E949CD1882309F4EFC00F
:10FF300020E1C29FC00111248756984FFC01E25472
:10FF4000FE4F20812F7709F0E2C03C96408151811D
:10FF500062817381443651056105710508F4D7C08B
:10FF60003497C080D180E280F380C114D104E104D1
:10FF7000F10421F4CCC0C12CD12C760140E0C701A2
:10FF8000B6010E949CD1182F882309F4C0C080912B
:10FF9000B4079091B5078115924009F0B8C0A091BF
:10FFA000B907AA2309F4B3C06091B7077091B807E5
:10FFB0006115710509F4ABC02091B607222309F43D
:10FFC000A6C0A093EE0B2093E00B80E030E041E070
:10FFD00050E0C82FFA01082E02C0EE0FFF1F0A944E
:10FFE000E2F72E173F0739F08F5FC83091F789E0AD
:10FFF0008093E90B8CC08093E90B2091BF0730916F
:020000021000EC
:10000000C0072115310519F040E050E008C02091EB
:10001000CD073091CE074091CF075091D007209364
:10002000E10B3093E20B4093E30B5093E40B46015A
:100030005701860E971EA11CB11C8092EF0B909267
:10004000F00BA092F10BB092F20BE091BA07F09195
:10005000BB07F093F50BE093F40BB0E00E9464EA69
:10006000860E971EA81EB91E8092F60B9092F70B73
:10007000A092F80BB092F90B85E0EE0FFF1F8A9566
:10008000E1F7E150FE4FEF2FFF27E6958E0E9F1E02
:10009000A11CB11C8092EA0B9092EB0BA092EC0B8E
:1000A000B092ED0B2091BC073091BD0721153105B1
:1000B00021F0A90160E070E008C04091C9075091AB
:1000C000CA076091CB077091CC07D701C601881988
:1000D0009909AA09BB09840F951FA61FB71F04C061
:1000E000B695A79597958795CA95D2F78093E50B16
:1000F0009093E60BA093E70BB093E80B853F2FE0BE
:100100009207A105B10528F48CE08093F30B10E071
:100110001AC0853F9F4FA105B10510F480E111C0C1
:100120008091D5079091D607A091D707B091D807B5
:100130008093F60B9093F70BA093F80BB093F90B09
:1001400080E28093F30B812FDF91CF911F91FF907D
:10015000EF90DF90CF90BF90AF909F908F900895D9
:10016000682F8EE99FE00C94DA4ACF92DF92EF92EB
:10017000FF921F93CF93DF931092360A8091690A02
:10018000882321F086E69AE00E94D9981092DB0B32
:100190001092D80B85E38093D70B0E94F858EB019F
:1001A000A89561E08091D70B0E9407B687ED9BE090
:1001B0000E943A9A2398229A219A209A289A85E0B6
:1001C0008093D90B82E58CBD1DBC1AE08FEF0E9495
:1001D0003F9A1150D9F720E030E0A90160E087EDA7
:1001E0009BE00E94449A182F8093DA0B813049F0EB
:1001F0000E94F8586C1B7D0B613D774060F381E0F5
:1002000054C02AEA31E040E050E068E087ED9BE02E
:100210000E94449A82FF03C01093DB0B0EC014E0CF
:100220000E94529F8093DA0B1150D1F78A3A11F055
:1002300082E03BC082E08093DB0B8091DB0B82305D
:1002400021F0C12CD12C760105C0C12CD12CE12C80
:1002500080E4F82E20E030E0A90167E387ED9BE021
:100260000E94449AA701960169E287ED9BE00E94F3
:10027000449A8093DA0B882349F00E94F8586C1B4B
:100280007D0B613D774030F38AE00FC08091DB0B3E
:10029000823011F520E030E0A9016AE387ED9BE0B0
:1002A0000E94449A882351F088E08093D80B87ED10
:1002B0009BE00E943A9AE2EFFDE119C00E94529F32
:1002C000807C803C19F483E08093DB0B0E94529F7A
:1002D0000E94529F0E94529F87ED9BE00E943A9A93
:1002E0001092D90B81E0E1DD811131C015C08491FC
:1002F000EF012196882321F00E94C689FE01F7CFE5
:10030000E4EEFDE18491EF012196882309F454C0C5
:100310000E94C689FE01F6CF80E0C7DD811117C0BB
:10032000EDEDFDE18491EF012196882321F00E94FB
:10033000C689FE01F7CFE9ECFDE18491EF0121963A
:10034000882309F439C00E94C689FE01F6CF6CEDFE
:100350007BE086E69AE00E948698811116C0EDED5A
:10036000FDE18491EF012196882321F00E94C68946
:10037000FE01F7CFE8EBFDE18491EF0121968823A0
:10038000D9F00E94C689FE01F7CF81E08093360A3A
:10039000E2EFFDE18491EF012196882319F0F6D771
:1003A000FE01F8CFECEAFDE18491EF01219688236C
:1003B00019F0ECD7FE01F8CF8BE1E6E6FAE0A5E80C
:1003C000BAE001900D928A95E1F78091640A9091CC
:1003D000650A9093840A8093830ADF91CF911F91DD
:1003E000FF90EF90DF90CF9008958091430E823080
:1003F00039F487E99DE19093A8078093A707F2D786
:100400000E94F8586093470E7093480E8093490EEF
:1004100090934A0E8091360A882319F081E08093E8
:10042000350A81E08093430E0895CF93DF931092B5
:10043000350A83E08093430E8091900E8823B1F0BB
:10044000EFE8FDE18491EF01882341F0082E000CD4
:10045000990B86DE2196FE018491F6CF8DE090E027
:100460007FDE8AE090E0DF91CF917ACEE3E9FDE193
:100470008491EF01882391F3082E000C990B70DE14
:100480002196FE018491F6CF8F929F92AF92BF92F8
:10049000CF92DF92EF92FF920F931F93CF93DF9350
:1004A00000D01F92CDB7DEB7FC018381813079F592
:1004B000818181FF2CC081899289A389B489892B8C
:1004C0008A2B8B2B09F448C07F0140E050E0BA0131
:1004D000CF010E94EF978823D1F0F7018588968895
:1004E000A788B08CC18CD28C82E090E0A0E0B0E014
:1004F000F60180839183A283B3839E012F5F3F4FD8
:10050000B501A401C6010E9465D2811102C080E03C
:100510003CC000E010E09801B501A401C6010E94B2
:10052000D4D18823A1F389809A80AB80BC80F60166
:100530008789803141F4F8EF8F16FFEF9F06A10401
:10054000B10460F4DACF88EF88168FEF9806A8061A
:100550008FE0B80618F4D1CF81E017C0F701158AF3
:10056000168A178A108E118A128A138A148A818138
:1005700080688183C7010E94B3D3882341F240E0A1
:1005800050E0BA01C7010E94EF970F900F900F90B3
:100590000F90DF91CF911F910F91FF90EF90DF901F
:1005A000CF90BF90AF909F908F9008951092380A8F
:1005B0001092350A8091010C882321F08EEF9BE088
:1005C0000C94D99808952F923F924F925F926F9218
:1005D0007F928F929F92AF92BF92CF92DF92EF92D3
:1005E000FF920F931F93CF93DF93CDB7DEB7C25720
:1005F000D1090FB6F894DEBF0FBECDBF8C013B0111
:100600004A014DB75EB7E1965FAF4EAFE197AD9649
:100610001FAEAD971B0154E0250E311C7E018FE506
:10062000E80EF11C9DEE492E92E0592EE0E4F0E038
:10063000EC0FFD1F3496E396FFAFEEAFE397F301A7
:100640008781823008F45AC184859585A685B7854F
:100650008F719927AA27BB27892B8A2B8B2B09F00F
:100660004DC11092460A46E45AE0BE016F5F7F4FCB
:10067000C1010E944BD318160CF040C18C85982FF5
:100680009871903129F42091B30C2150223078F4E4
:100690002981222309F432C1253E89F22E3279F2D2
:1006A0002091460A2E3259F28A7049F6B4C04DB7ED
:1006B0005EB7AF965FAF4EAFAF97BE016F5F7F4F34
:1006C000C7010E9446D10115110521F0F801808172
:1006D000811197C021E081E090E0F70101900020B6
:1006E000E9F73197EE19FF098E0F9F1F02964DB75C
:1006F0005EB7481B590B0FB6F8945EBF0FBE4DBFD7
:100700008DB79EB701965C01211102C0B80102C0ED
:1007100062E273E0C5010E94E8EDB701C5010E94E5
:10072000C9ED62E273E0C5010E94C9ED25961FAED6
:10073000259728961FAE289724961FAE1EAE2497A5
:1007400022965FAE4EAE229721E0A701B101E3965B
:100750008EAD9FADE3970E94659E811126C080916A
:10076000B30C811122C0E2EFFDE184916F019FEF94
:10077000C91AD90A882319F009D6F601F6CFEBE792
:10078000FDE184916F012FEFC21AD20A882319F07C
:10079000FDD5F601F6CF6701F60181916F0188233F
:1007A00011F0F4D5F9CF8AE0F1D58BE1FE01EC5BD5
:1007B000FF4FDE01959601900D928A95E1F7249600
:1007C0008EAD9FAD24979CA38BA35AA249A240E073
:1007D00050E0BE016F5D7F4FC501F5DECE01819611
:1007E0000E9492A0CE01805C9F4F0E9492A0AF9683
:1007F0004EAD5FADAF970FB6F8945EBF0FBE4DBF65
:100800001ECFF80101900020E9F73197CF01801B3E
:10081000910B20E062CF81E0903109F080E080937D
:10082000370A903141F08985873409F008CF8A85ED
:100830008E3709F404CF8091B30C813029F08230D7
:10084000B9F18111FCCE0AC08091B40C9091B50C25
:1008500001969093B50C8093B40CF1CEBE016F5FFE
:100860007F4F89E39AE00E9446D10115110529F4D2
:1008700089E3C82E8AE0D82E08C06801F60181916C
:100880006F018823A9F382D5F9CFF60181916F0119
:10089000882311F07BD5F9CF80E278D56D8D7E8DE0
:1008A0008F8D98A14AE00E94E98C8AE06FD5C7CE6F
:1008B000BE016F5F7F4F89E39AE00E9446D18114A9
:1008C000910441F069E37AE0C4010E94B6ED892BFE
:1008D00069F414C0AD96FFADAD978F2F90E02091D5
:1008E000C00F3091C10F8217930741F0AD962FAD25
:1008F000AD972F5FAD962FAFAD97A1CEE1968EADA0
:100900009FADE1970FB6F8949EBF0FBE8DBFCE5836
:10091000DF4F0FB6F894DEBF0FBECDBFDF91CF9192
:100920001F910F91FF90EF90DF90CF90BF90AF900D
:100930009F908F907F906F905F904F903F902F90FF
:1009400008950F931F93CF93DF93CDB7DEB76F97C3
:100950000FB6F894DEBF0FBECDBF8B0122E020930F
:10096000B30C9093C10F8093C00F85E89AE00E946A
:10097000369A8BE1E5E8FAE0DE01159601900D92DA
:100980008A95E1F78091830A9091840A9C838B83F6
:100990008DEE92E09A838983A801BE016F5F7F4F3D
:1009A00080E090E010DECE0101960E9492A06F964A
:1009B0000FB6F894DEBF0FBECDBFDF91CF911F9170
:1009C0000F9108952F923F924F925F926F927F9274
:1009D0008F929F92AF92BF92CF92DF92EF92FF924F
:1009E0000F931F93CF93DF93CDB7DEB76F970FB6FB
:1009F000F894DEBF0FBECDBF6C012DB63EB61D8292
:100A000018861C821B828DEE92E09A838983FB01FB
:100A100080819E012F5F3F4F39018F3241F081E885
:100A20009AE0F60191838083F62E172F62C082E64A
:100A30009AE0F601918380838B010F5F1F4F0115B0
:100A4000110509F454C04DB65EB66FE270E0C801FE
:100A50000E94D4ED4C010817190708F046C07C012C
:100A6000E01AF10AFF24C70101962DB73EB7281BF3
:100A7000390B0FB6F8943EBF0FBE2DBF8DB79EB792
:100A800001965C01A701B8010E94FDEDF501EE0D94
:100A9000FF1D1082F601608171816115710511F0F1
:100AA0006C5F7F4F21E0A501CE0105960E94659EF7
:100AB00081110FC0B50187E69DE10E9468C58EE2F5
:100AC00065D48AE063D40FB6F8945EBE0FBE4DBE07
:100AD0000EC0F6017182608284010F5F1F4F0FB656
:100AE000F8945EBE0FBE4DBEAACFF02E02C0F12C10
:100AF00010E0C3010E9492A08F2D912F0FB6F894A1
:100B00003EBE0FBE2DBE6F960FB6F894DEBF0FBE71
:100B1000CDBFDF91CF911F910F91FF90EF90DF90AC
:100B2000CF90BF90AF909F908F907F906F905F908D
:100B30004F903F902F9008959091C310E92FF0E0CF
:100B4000E85BFA4F80839F5F943018F49093C31052
:100B500002C01092C3108091C4108F5F8093C410A4
:100B60000895CF93FC0120812B33A1F02091C41074
:100B7000243080F4C62FBC018091C310F0E68F9F13
:100B8000C0011124835B9A4F0E94E8ED8C2FD4DFC3
:100B900081E001C080E0CF9108952F923F924F9263
:100BA0005F926F927F928F929F92AF92BF92CF92FD
:100BB000DF92EF92FF920F931F93CF93DF9300D0BA
:100BC00000D0CDB7DEB79A8389830E94F858E981B7
:100BD000FA81C680D780E084F184C114D104E10495
:100BE000F10409F0ACC22485222309F469C33285DB
:100BF0002150248721E0230F22874585241301C03B
:100C00001286E981FA8124E0329FE00DF11D112462
:100C1000C684D784E088F188E981FA81C282D382D0
:100C2000E482F582DC01CB018C0D9D1DA11DB11D5F
:100C300086839783A087B18784819581892B09F466
:100C40003FC3FFB7FD83F894E981FA8122803380A6
:100C50002101612C712C04811581809119028F3141
:100C600021F08F3F09F068C205C0E5E5F8E1249165
:100C70002E83DAC08FE180931902E5E5F8E18491D3
:100C80008E838F3F09F458C2823009F469C030F571
:100C9000882309F44CC0813009F0C6C0109280004E
:100CA0001092810080918100886080938100809102
:100CB0008100816080938100E9E5F4E2E491F0E055
:100CC000EE0FFF1FEA5FFB4D85919491EFE9F4E28F
:100CD000E491E093C50FE1E0EE8330C19E81943052
:100CE00009F482C008F460C0953009F09DC01092EC
:100CF00020011092210180912101886080932101BF
:100D000080912101816080932101E9E5F4E2E49181
:100D1000F0E0EE0FFF1FEA5FFB4D85919491EFE944
:100D2000F4E2E491E093C20F95E09E8307C114BC06
:100D300015BC84B5826084BD85B5816085BDE9E55B
:100D4000F4E2E491F0E0EE0FFF1FEA5FFB4D8591C6
:100D50009491EFE9F4E2E491E093C60F1E82ABC2F6
:100D60001092B0001092B1008091B0008260809328
:100D7000B0008091B10081608093B100E9E5F4E2B8
:100D8000E491F0E0EE0FFF1FEA5FFB4D8591949137
:100D900090932D0580932C05EFE9F4E2E491E09324
:100DA0002E05F2E0FE8387C210929000109291000F
:100DB0008091910088608093910080919100816082
:100DC00080939100E9E5F4E2E491F0E0EE0FFF1F7B
:100DD000EA5FFB4D85919491EFE9F4E2E491E093B1
:100DE000C40F23E02E83AAC01092A0001092A1008D
:100DF0008091A10088608093A1008091A100816012
:100E00008093A100E9E5F4E2E491F0E0EE0FFF1F2A
:100E1000EA5FFB4D85919491EFE9F4E2E491E09370
:100E2000C30F84E08E838AC0EE81E7FD85C161E057
:100E30008FE10E9407B68E818D7F09F083C0480143
:100E4000A12CB12C60E072E18AE790E0A501940149
:100E50000E9448EA29833A834B835C8369017A01C3
:100E6000F1E0CF1AD108E108F1082FEFC216D10442
:100E7000E104F10409F008F44EC060E472E48FE08C
:100E800090E0A50194010E9448EA69017A0181E09D
:100E9000C81AD108E108F1089E81923009F5EFEFF8
:100EA000CE16D104E104F10409F008F4CBC160E9E5
:100EB00070ED83E090E0A50194010E9448EA690189
:100EC0007A01F1E0CF1AD108E108F1082FEFC2163C
:100ED000D104E104F10411F008F041C183E027C01E
:100EE0008FEFC816D104E104F104B9F0B0F068E462
:100EF00078EE81E090E0A50194010E9448EA690142
:100F00007A0191E0C91AD108E108F108EE81EE23D7
:100F100009F49AC163C181E001C082E09E81911110
:100F200006C095B5987F892B85BD7AC085E09091E4
:100F3000B100987F892B8093B10072C061E08FE18E
:100F40000E9407B64801A12CB12C60E072E18AE74B
:100F500090E0A50194010E9448EA69017A01E1E06C
:100F6000CE1AD108E108F108C114D104F1E0EF066E
:100F7000F10488F068E478EE81E090E0A501940146
:100F80000E9448EA69017A0181E0C81AD108E108A3
:100F9000F10883E001C081E09E81913071F490916D
:100FA0008100987F892B8093810045284628472817
:100FB000D9F52FEF3FEFA90168C0EE81E33071F45E
:100FC00090919100987F892B809391004528462825
:100FD000472851F52FEF3FEFA90179C0FE81F4308A
:100FE00071F49091A100987F892B8093A1004528EE
:100FF00046284728C9F42FEF3FEFA9017AC02E8178
:10100000253071F490912101987F892B80932101E3
:1010100045284628472841F42FEF3FEFA9017BC020
:1010200045284628472869F0D801AA0FBB1F91011F
:101030000E9474EA28EE33E040E050E00E9426EA85
:1010400003C02FEF3FEFA9018E81823081F12CF494
:10105000882361F08130C9F06FC09E81943009F41B
:1010600048C0ACF1953009F456C066C0C7BC2093A7
:10107000D70F3093D80F4093D90F5093DA0F809148
:101080006E00826080936E0057C0D0928900C0923B
:1010900088002093D30F3093D40F4093D50F5093F3
:1010A000D60F80916F00826080936F0045C0C09220
:1010B000B30020932F0530933005409331055093B2
:1010C00032058091700082608093700035C0D092AC
:1010D0009900C09298002093CF0F3093D00F409387
:1010E000D10F5093D20F8091710082608093710074
:1010F00023C0D092A900C092A8002093CB0F3093B8
:10110000CC0F4093CD0F5093CE0F80917200826030
:101110008093720011C0D0922901C09228012093BF
:10112000C70F3093C80F4093C90F5093CA0F8091D7
:101130007300826080937300ED81EFBFC1C0DC015A
:10114000CB018C199D09AE09BF09B7FDB9C04698FE
:10115000E981FA811682178210861186B1C068E48F
:1011600078EE81E090E0A50194010E9448EA6901CF
:101170007A01F1E0CF1AD108E108F1082FEFC21689
:10118000D104E104F10441F138F164E274EF80E04C
:1011900090E0A50194010E9448EA69017A01F1E01A
:1011A000CF1AD108E108F1082FEFC216D104E104EB
:1011B000F10409F008F4BACE62E17AE780E090E049
:1011C000A50194010E9448EA69017A0181E0C81AE8
:1011D000D108E108F10819C084E0A9CE2FEFC216AA
:1011E000D104E104F10409F008F463C062E17AE794
:1011F00080E090E0A50194010E9448EA69017A012B
:10120000F1E0CF1AD108E108F1082FEFC216D1049E
:10121000E104F104A9F0A0F089819A81AB81BC813D
:101220002AE0B595A795979587952A95D1F76C01F2
:101230007D01F1E0CF1AD108E108F10887E077CE0F
:1012400086E075CE82E073CEEFEFCE16D104E104D6
:10125000F10469F160F162E17AE780E090E0A501D4
:1012600094010E9448EA69017A0181E0C81AD10814
:10127000E108F1089FEFC916D104E104F104A9F0D7
:10128000A0F089819A81AB81BC813AE0B595A795A0
:10129000979587953A95D1F76C017D01E1E0CE1ADB
:1012A000D108E108F10885E03CCE84E03ACE83E045
:1012B00038CE84E033CE61E08FE10E9407B6BFCD27
:1012C00026960FB6F894DEBF0FBECDBFDF91CF914B
:1012D0001F910F91FF90EF90DF90CF90BF90AF9054
:1012E0009F908F907F906F905F904F903F902F9046
:1012F00008950F931F93CF93DF93CDB7DEB72C974D
:101300000FB6F894DEBF0FBECDBFE6E3F4E08085F4
:101310009185A285B385448155816681778100815D
:1013200011812281338109831A832B833C834D836E
:101330005E836F83788789879A87AB87BC87AE0186
:10134000475F5F4FBE016B5F7F4FCE0101960E94EA
:10135000C2BC22E434E0AE01475F5F4FBE016B5F69
:101360007F4FCE0101960E941DC82C960FB6F894AF
:10137000DEBF0FBECDBFDF91CF911F910F910895BA
:10138000FC01238121110C94D99808959091C000FB
:1013900095FFFCCF8093C6000895EF92FF921F93B4
:1013A000CF93DF937C0160E0DCDB182F882399F07A
:1013B000E2EFFDE18491EF012196882319F0E6DF49
:1013C000FE01F8CFB70188EF9DE10E9468C582E277
:1013D000DDDF8AE0DBDF812FDF91CF911F91FF906E
:1013E000EF900895DF92EF92FF920F931F93CF93A8
:1013F000DF93CDB7DEB76E970FB6F894DEBF0FBEA2
:10140000CDBF6091A7077091A8076115710541F1E3
:101410004DE150E0CE0101967C010E94E1E51E8E77
:10142000F7018F010E191F09D190DD2019F09AE004
:10143000D912F7CFF701E00FF11F1082C701ADDF1E
:10144000882371F0DD20A9F00F5F1F4F8091A7075F
:101450009091A807080F191F1093A8070093A707DA
:1014600081E02091A7073091A807232B29F480E081
:1014700003C000E010E0F0CF6E960FB6F894DEBF28
:101480000FBECDBFDF91CF911F910F91FF90EF90D5
:10149000DF9008953F924F925F926F927F928F926A
:1014A0009F92AF92BF92CF92DF92EF92FF920F93F3
:1014B0001F93CF93DF931F92CDB7DEB793DF8111D8
:1014C00075C28091C410843008F048C00E94A34BBC
:1014D000AC0197FF7CC142C08E3409F0D9C101151F
:1014E000110509F4D5C16BE27FE1C8010E94F0E566
:1014F0007C01892B09F48EC16EE470E0C80104966A
:101500000E94D4ED009709F485C14AE050E060E004
:1015100070E001960E948CE36093DB0F7093DC0F08
:101520008093DD0F9093DE0F8090C2189090C318C7
:10153000A090C418B090C5182FEF821A920AA20A80
:10154000B20A681579058A059B0509F465C1EF287B
:1015500009F062C188EF9EE10E9426D78091350A8A
:10156000882309F423C28091C410811102C0109213
:101570004110EE24E3944091AF0C5091B00C609177
:10158000B10C7091B20C8091AB0C9091AC0CA0910D
:10159000AD0CB091AE0C481759076A077B0708F4E9
:1015A000E12C00E010E09924939480E6882E90E3EB
:1015B000A92E9FE1B92E2DE8322E8091C4108430DF
:1015C00008F0F4C1E110F2C1809141108111EEC127
:1015D0008091060C9091070CA091080CB091090C19
:1015E0008093AF0C9093B00CA093B10CB093B20C5D
:1015F00041E050E0BE016F5F7F4F8EEF9BE00E94A5
:10160000599B019719F4898190E002C08FEF9FEFF9
:10161000F82E4090AF0C5090B00C6090B10C7090D0
:10162000B20C4091AB0C5091AC0C6091AD0C709130
:10163000AE0CEE24E394441655066606770608F4CD
:10164000E12C4416550666067706B0F4019609F4B7
:101650006AC08AE0F81609F489C09DE0F91609F419
:1016600085C023E2F21619F08AE3F81296C0809141
:101670004010811192C06FC00E94186A8EEF9BE0EB
:101680000E94D9988091190C882359F18150809338
:10169000190C389EC001112441E061E0825E934F35
:1016A0000E9486D5E091190C94E0E99FF001112485
:1016B000E65EF34F40815181628173814093AF0CAC
:1016C0005093B00C6093B10C7093B20C8EEF9BE012
:1016D0000E94EF978091360A8823A9F09092350AEC
:1016E00012C01092350A0E94A4B70E94F4780E949A
:1016F0006E786D3371058105910528F0B092A807C9
:10170000A092A7076FDE8091350A811128C0E3E41B
:10171000FFE184916F012FEFC21AD20A8823D9F01A
:1017200035DEF601F6CFEDEDFDE184916F019FEF1F
:10173000C91AD90A882319F029DEF601F6CFE4E3A5
:10174000FFE184916F012FEFC21AD20A882319F0AA
:101750001DDEF601F6CF83E2F81208C005C023E2D1
:10176000F21221C100E010E090924110109240105E
:101770000115110519F40E94C97B0CC08091C3109A
:10178000889E000D111D1124F801E35BFA4F1082B1
:1017900080E0D2D900E010E010CF0F35110508F03D
:1017A0000CCF9BE3F91202C0909240108091401040
:1017B000811103CF8091C310F801889EE00DF11DC7
:1017C0001124E35BFA4FF0820F5F1F4FF6CE982F84
:1017D0002091C0183091C1188A3019F09D3009F05D
:1017E000B0C010923F102115310519F40E94C97B39
:1017F00068CEF901E152F04F10821092C118109298
:10180000C0180FED1FE0F8018191803209F064CE1D
:101810008F01F9CFC80179CE6AE270E0C8010E9459
:101820000CEE9C01009701F1982F901BF12C99234D
:1018300039F09150F801E90FF11D8081F826F7CFBA
:101840004AE050E060E070E0C90101960E948CE33C
:10185000CF2CD12CE12CF12C6C157D058E059F052C
:1018600031F089ED9EE178CE8FEA9EE175CE8091D0
:10187000DB0F9091DC0FA091DD0FB091DE0F809314
:10188000C2189093C318A093C418B093C5180EC083
:101890008091330A882351F065EF73E0C8010E94FC
:1018A000DFED892B19F085E89EE156CE8091270265
:1018B000811126C067E470E0C8010E94D4ED009752
:1018C000F9F04AE050E060E070E001960E948CE39D
:1018D00097FD16C064307105810591052CF06530C7
:1018E00071058105910561F4EEE0FEE184917F01CF
:1018F0009FEFE91AF90A882319F048DDF701F6CFBE
:1019000069EF73E0C8010E94DFED892B11F410929A
:1019100020026EEF73E0C8010E94DFED892B21F4F5
:1019200085E09EE10E94B5A063E074E0C8010E94DA
:10193000DFED892B09F42AD261E08FED9FE011D908
:10194000C0CD2F3531050CF0BCCD9C35C1F40E94C3
:10195000A34B97FDB6CD20913F102111B2CD209120
:10196000C0183091C118A9014F5F5F4F5093C11843
:101970004093C018F901E152F04F8083A2CD9B3310
:1019800019F481E080933F1080913F10811199CD2F
:10199000C90101969093C1188093C018F901E152D2
:1019A000F04F40838ECD10924010E5CE0F90DF9126
:1019B000CF911F910F91FF90EF90DF90CF90BF904C
:1019C000AF909F908F907F906F905F904F903F90DF
:1019D00008958F929F92AF92BF92EF92FF920F93D2
:1019E0001F93CF93DF93CDB7DEB7A0970FB6F894D0
:1019F000DEBF0FBECDBF611571058105910589F16F
:101A000000E0842E912CA12CB12C102FEE24E39415
:101A1000F12CEC0EFD1EE00EF11C07FDFA94A50161
:101A200094010E9426EAF7016083B901CA010F5FA1
:101A3000611571058105910541F71F3F21F1E1E035
:101A4000F0E0EC0FFD1FE10FF11D17FDFA9580810D
:101A50008A3010F097E301C090E3890F97DC1150B2
:101A6000ECCF80E3A0960FB6F894DEBF0FBECDBFDB
:101A7000DF91CF911F910F91FF90EF90BF90AF90AA
:101A80009F908F9083CCA0960FB6F894DEBF0FBEC8
:101A9000CDBFDF91CF911F910F91FF90EF90BF903D
:101AA000AF909F908F900895CF92DF92EF92FF9228
:101AB0006B017C0197FF0AC08DE268DCF094E09432
:101AC000D094C094C11CD11CE11CF11C4AE0C70198
:101AD000B601FF90EF90DF90CF907BCF8F929F92D7
:101AE000AF92BF92CF92DF92EF92FF92CF936B01B2
:101AF0007C01B42E20E030E0A9010E9438E687FF87
:101B000006C08DE243DCF7FAF094F7F8F094C0E0F9
:101B100060E070E080E09FE3CB1541F02DEC3CEC01
:101B20004CEC5DE30E949DE6CF5FF6CF9B01AC01DC
:101B3000C701B6010E9484EA6B017C010E94CDEBD3
:101B40004B015C014AE045DFCC2379F1C501B401CA
:101B50000E943CE69B01AC01C701B6010E9483EAEA
:101B60006B017C018EE212DC20E030E040E251E4C7
:101B7000C701B6010E949DE64B015C010E94C8EBC3
:101B80006B01770FEE08FF08C701B6018DDFC701B3
:101B9000B6010E943EE69B01AC01C501B4010E9462
:101BA00083EA6B017C01C150F9F6CF91FF90EF9071
:101BB000DF90CF90BF90AF909F908F900895CF927D
:101BC000DF92EF92FF920F931F93CF93DF9388E5FD
:101BD0000E94484CD82E89E40E94484CC82E882385
:101BE00019F00E94E14B1CC0DD20C1F00E94114C95
:101BF00020E030E040E251E40E9483EA20E030E05F
:101C000048EC51E40E9484EA2AE037ED43EA5CE3C1
